:020000040800F2
:1000000000000420E58C0008CD320008D132000841
:10001000D5320008D9320008DD32000800000000A7
:1000200000000000000000000000000085490108F9
:10003000E132000800000000114A0108714A01087D
:10004000358D0008358D0008358D0008358D000888
:10005000358D0008358D0008E53200083D33000875
:10006000358D0008358D000809100008891D00082D
:10007000B11D0008D91D0008358D0008011E0008BB
:100080000D1E0008358D0008358D0008358D0008DF
:10009000358D0008358D0008358D0008B93600080B
:1000A000358D0008358D0008358D0008358D000828
:1000B000358D0008358D0008358D0008D51C0008E9
:1000C000E11C0008ED1C0008F91C0008051D0008D3
:1000D000111D0008358D00081D1D0008358D000814
:1000E00055330008358D0008358D00089D33000814
:1000F000B5330008CD330008358D0008351E0008E3
:1001000000000000358D0008358D0008358D000891
:100110000000000000000000358D0008358D00084B
:100120005D1E0008691E00089D1E0008E1330008DE
:10013000358D0008358D0008358D0008358D000897
:10014000358D0008358D0008358D0008358D000887
:10015000358D0008ED330008A91E0008391D000880
:10016000358D0008358D00080000000000000000FB
:10017000000000000000000000000000000000007F
:10018000358D0008358D00080000000000000000DB
:10019000358D0008358D00080000000000000000CB
:1001A000000000000000000000000000000000004F
:1001B000358D00080000000000000000358D0008AB
:1001C000358D000810B5034B0360044614F07EF92A
:1001D000204610BD9897010810B5054B03600446F2
:1001E00014F074F92046082115F0D2FE204610BD07
:1001F0009897010810B5064A064B0260044640F87D
:10020000783F14F063F9204614F09CFA204610BDA4
:10021000B49701089897010810B5064A064B02608A
:10022000044640F8783F14F051F9204614F08AFA59
:10023000204610BDB49701089897010890F8BE3584
:1002400010B5044623B1D0F8B80508B115F0A2FEE8
:1002500094F8AE3523B1D4F8A80508B115F09AFE8C
:1002600094F89E3523B1D4F8980508B115F092FEA4
:1002700094F88A3423B1D4F8840408B115F08AFEC6
:10028000204610BD08B5274C2368BFF35B8FD90704
:1002900012D5254C2368BFF35B8FDA072FD5234C8B
:1002A0002368BFF35B8FDB0717D5214B01221A7040
:1002B00015F094FA04F044FC204600F0BDFC002840
:1002C000E7D01C4800F098FB1B4A1C49194800F075
:1002D000BFFC204600F0B6FCDBE7204600F0ACFC9B
:1002E0000028E2D01349164800F0ACF9124A15492B
:1002F000134800F0ADFC204600F0A4FCD5E72046F2
:1003000000F09AFC0028CAD00A490F4800F098F87B
:10031000094A0E490C4800F09BFC204600F092FC74
:10032000BDE700BF18040020900200200802002052
:1003300078D901201C040020790C00083D02000837
:100340000C0200201902000894020020F5010008A8
:1003500010B5094A094B0260044640F8783F14F092
:10036000B5F8204614F0EEF920464FF4C27115F0AE
:100370000FFE204610BD00BFB497010898970108F2
:1003800010B5084A084B0260044640F8783F14F064
:100390009DF8204614F0D6F92046842115F0F8FD8A
:1003A000204610BDB49701089897010808B5044687
:1003B0000021204614F060FA78B9204614F06AFA59
:1003C00006280ED1D4F88000032102F081FC002120
:1003D000204614F051FA0028EFD0022003F070FA02
:1003E000E6E704F0ADFB00BF70B5541A82B00F2CE5
:1003F0000E460194054611D8012C006808D10B78EF
:100400000370019C28686C600023035502B070BD26
:100410005CB900236C60035502B070BD002201A9D5
:1004200015F0BCFD019B2860AB602246314618F0F8
:1004300087FA019C28686C600023035502B070BDE8
:1004400070B5114A86B0044602AE68460D46A2F168
:100450000A010096FFF7C8FF032369464FF4806244
:10046000204614F0EDF90098B04203D00299013112
:1004700015F08EFD054B2360C4F88051204614F022
:1004800025F9204606B070BDCA970108609801089A
:100490002DE9F041D0F88051284600F00FFB421EB4
:1004A00018BF012206460321284602F047FC3246C7
:1004B0000121284602F042FC05F5987003F0E2F8AD
:1004C0000FF0AAFB4A480EF0EBFC4A4808227821BC
:1004D0000FF0D8F948481E2278210FF0D3F9474889
:1004E0000EF0DEFC012E79D004200EF0BDFC444855
:1004F000502278210FF0C6F9301E18BF012080006D
:100500000EF0B2FC6E2278213E48DFF8F4803D4FB9
:100510000FF0B8F900200EF0A7FC3B489622782196
:100520000FF0B0F901220021284602F007FC00215B
:10053000284602F021FD022804460DD0042831D0BF
:10054000012813D0FA2004F033FB0021284602F0E2
:1005500013FD02280446F1D1FA2004F029FB2846B5
:10056000314600F0AFFA3046BDE8F08100220321A9
:10057000284602F0E3FB22462146284602F0DEFB35
:1005800000200EF071FC5022782140460FF07AF9DD
:1005900004200EF069FC6E22782138460FF072F9C3
:1005A0002646CFE701220321284602F0C7FB00229E
:1005B0000121284602F0C2FB20460EF055FC5022D5
:1005C000782140460FF05EF900200EF04DFC6E22BF
:1005D000782138460FF056F90026B3E700200EF0D8
:1005E00043FC0748502278210FF04CF9042087E79C
:1005F00008E70108CC970108E4970108F0D6010844
:10060000FC970108149801082C98010830B595B0A2
:100610000446FFF73DFF03220223CDE900230546F0
:10062000062369462046029314F040F964212046CF
:1006300014F032F9D4F88001294600F0C7FA15B059
:1006400030BD00BF70B5114A86B0044602AE6846A0
:100650000D46A2F10E010096FFF7C6FE0223694681
:100660004FF40072204614F0EBF80098B04203D02B
:100670000299013115F08CFC054B2360C4F88050C1
:10068000204614F023F8204606B070BD56980108A5
:100690007498010802484FF4DC310FF013BF00BF1B
:1006A000E81100204FF0C043C0B21880704700BF6F
:1006B0004FF0C0435880704741B100EB41014FF00B
:1006C000C04230F8023B53808142FAD1704700BFEC
:1006D00041B100EB41014FF0C042538820F8023B8A
:1006E0008142FAD1704700BF30B50024A1B0214645
:1006F000682206A80194029403940494059418F0C7
:100700008BF823462246134913480FF0E9F9F022EB
:100710000546114620460DF065F9F02211462046A7
:100720000DF048F9204603210EF0B6FC01A9284639
:100730000DF0DFF8094A0A4B0A4C1194CDE90E235B
:10074000094A1592094B0A4A06A928460DF0EFF806
:1007500021B030BD10F501085CF30108A5060008C2
:10076000B1060008B9060008D1060008F9D2000851
:100770005DCC000810B58AB01E4B00220192196BA7
:1007800041F008011963186B00F00800019001980E
:100790000292186B40F040001863186B00F04000A4
:1007A000029002980392186B40F0200018631B6BB4
:1007B0001148069203F020030393022304A94FF487
:1007C00000620793012304920593039C04F09CFCB0
:1007D00004A9082200230948CDE9042304F094FC6D
:1007E00020220123064804A9CDE9042304F08CFC4F
:1007F0000AB010BD00380240000C02400018024050
:100800000014024008B5FFF7B5FF1F480122202160
:1008100004F0ACFD00224FF400611C4804F0A6FD7A
:10082000052004F0C5F901224FF40061174804F0D7
:100830009DFD0A2004F0BCF900224FF4006113482A
:1008400004F094FD142004F0B3F901224FF4006188
:100850000E4804F08BFD0A2004F0AAF90C4B5B68EB
:100860009847852807D00B4B5B6898474FF6FF7376
:10087000984204D008BDBDE8084002F021B9BDE8A7
:10088000084001F03FBE00BF00140240000C0240CF
:100890004000002004000020012908B503D1FFF723
:1008A000B1FF002008BD4FF0FF3008BD00F26444E6
:1008B00080B50546052301220221204600F00EFBEB
:1008C00005F27C46204600F049FB0221304600F04C
:1008D00001FC104F05F5B565204600F065FB20468C
:1008E00000F06AFB012238464FF4806104F03EFDBF
:1008F0000121204600F084FB40F3CF11284600F090
:1009000003FA47F6FF7382B20221304600F0F8FB8B
:10091000E2E700BF0000024080B5DFED308A9FEDC6
:1009200030AADFED30AADFED309A9FED309A82B029
:100930000746B0EE68BA00F5B56900F2D458B7EED4
:10094000008A002568EE0A7AD7F84006FDEEE77ABD
:1009500017EE903A19B208F0ADFDBEEEC98A4846CE
:1009600018EE103A1CB2214600F0CEF9C0EB00118F
:10097000090144BF01F57F41FF3106460914D7F84C
:10098000440608F097FD2A46CDE90056184923464B
:10099000404617F007FF01354146002004F078F883
:1009A000B5F5817F09D178EE8B8A0025F4EEEA8ACD
:1009B000F1EE10FAC8BFDFED098A0EF0B5FB68EE64
:1009C000A97A87EE890A07EE905AF8EEE77A20EEC8
:1009D000270A15F027FBB0EE408AB3E70000C842B3
:1009E0000000704200007A44DB0FC94000007A45E5
:1009F000809801080000000030B56021044689B0ED
:100A000001F06CFA002504F29443294AC4F88434B6
:100A10008121A4F88814C4F88C34C4F89034C4F844
:100A200098254FF40053A4F89C15C4F8A02504F5AC
:100A3000B361C4F8A42584F88A5404F2844284F88B
:100A40009E5504F5B56000F019F92846C4F83856EB
:100A5000C4F83C5603F01EFF2946204600F026FC51
:100A60002046012100F03CFC2046012100F042FC20
:100A7000104B01951A6B104842F001021A631B6B70
:100A80009FED097B03F001030193002202A90223D9
:100A9000CDE904238DED027B019B04F035FB20465C
:100AA00009B030BDAFF30080000400000100000079
:100AB0005C9901080038024000000240032102F066
:100AC00079BA00BF0A46032102F06ABAF0B5D0F83D
:100AD0003C5685B004460E462DB1284605B0BDE80B
:100AE000F04009F0DCB909F0B3FC4FF4087303934C
:100AF00002230193F0231A460090294602952846C6
:100B000009F090F82A46C4F83C066FF07F4109F0DE
:100B1000DDF82C49D4F83C06012209F0D7F803226D
:100B20002949D4F83C0609F0D1F8D4F83C06012153
:100B300009F0E9F8334604F24C624FF4F0714FF4D7
:100B40007F0008F07DFC334604F60C22C4F8400612
:100B50004FF4F0714FF4004008F072FCD4F8407686
:100B6000C4F8440606463946D4F83C0609F06AF84B
:100B700038463C2108F0B9FCD4F83C06314609F06F
:100B800061F83046B42108F0B0FC1423012211466C
:100B9000184608F049FBB7EE000AC4F8480608F00A
:100BA00071FBD4F84816D4F83C0609F06DF8D4F877
:100BB0003C0600952B462A46142109F0BCF805B0E6
:100BC000F0BD00BF808080004040400008B5054671
:100BD0000C46C0F83816B1B90FF01EF8114920467E
:100BE00003F056FF1049204603F052FF0F485022F1
:100BF00078210EF047FE0E486E2278210EF042FE5C
:100C00002846FFF753FE4FF4F071FFF75FFF0949E5
:100C1000002003F03DFF0449002003F039FF28467F
:100C2000FFF77AFE98980108B8980108FC98010827
:100C300018990108389901080078B0FA80F0400945
:100C4000704700BF01230370704700BF704700BFAB
:100C500000207047704700BFFEE70000044A0549C6
:100C60001368002B08BF0B461844106018467047E5
:100C7000E8C901209818022000207047F8B50D46F9
:100C80008979044616461F46C1B92B680360836004
:100C9000C360AB8881718380B3791BBBB288A375B5
:100CA0003368A2822361A361E361AA882785930840
:100CB00002F00302236262622046F8BDA888400069
:100CC00015F06AF9AB79AA882060A060E060A37192
:100CD000A280002BE0D02968520017F031FEB379D2
:100CE000002BDBD0B088400015F056F9B379B288FC
:100CF0002061A061E061A375A282002BD5D031688C
:100D0000520017F01DFED0E72DE9F84FC3690469C2
:100D1000D0F800A0D0F820B09A1CC2611980B0F8B9
:100D200014C004EB4C018A424FEA4C0C14BFC26958
:100D30002246ACF1020CC2610646A4440AEBCB0E7B
:100D400052460020002133F90289B2F90070B2F94D
:100D500002509C4294BF9946E146C8FB870139F98D
:100D60000239B2F904704C4594BFC846E046C3FB53
:100D7000850138F90299B2F90650444594BF4346BB
:100D80006346C9FB870133F9027908329C4288BF68
:100D900063469645C7FB8501D5D1726AB3614FEAB8
:100DA0008B0B82B15A440AEB420A1A463EF9025BA7
:100DB00032F9027994428CBF63461346F245C7FB71
:100DC0008501F2D1B361B6F92820D31716F0F8FAED
:100DD00000B2BDE8F88F00BF10B5034B03600446B6
:100DE00013F0D4FB204610BD689A010810B5054BDE
:100DF0000360044613F0CAFB2046082115F0C8F82A
:100E0000204610BD689A010870B5044640F80C1BD6
:100E1000022388B0A36008220021606017F0FCFC68
:100E200000251E4B00951A6B257542F002021A63CD
:100E30001A6B1B4E02F002020092009A01951A6B87
:100E400042F004021A631B6B03F0040301930122B6
:100E50000123CDE9022302A9019B30460022002391
:100E6000CDE9042304F050F90E4B0F481022CDE9D0
:100E7000022302A902230122CDE9042304F044F94C
:100E80002A4609210A2003F0B7FE01223046114606
:100E900004F06CFA204608B070BD00BF0038024074
:100EA00000040240000021100008024070B5054611
:100EB0000C46164622460021286800F095F90022CB
:100EC0002868114600F090F980B204B970BDB042B4
:100ED0004FF00A00FAD003F06BFEEBE7F8B51746C7
:100EE000002204460E46006811461D4600F07CF9BB
:100EF00000221146206800F077F945F206521146AB
:100F00002046FFF7D3FF43F64B020021206800F094
:100F10006BF9760200221146206806F47E4600F046
:100F200063F906F14D020021206800F05DF900220E
:100F30001146206800F058F905EB4712D2B21202B0
:100F40004E320021206800F04FF90022206811463F
:100F500000F04AF901232375F8BD00BF10B540F237
:100F60004F3204460021006800F03EF9002211468D
:100F7000206800F039F94FF44C5211462046FFF733
:100F800095FF45F2055211462046FFF78FFF0448B2
:100F900013F026FB034B4FF480621A6010BD00BFB4
:100FA000F0C9012000E100E002484FF0FF3113F0EA
:100FB00009BB00BFF0C9012010B588B00F490191ED
:100FC00005A9044603AA032303910068029301A91B
:100FD000049300F035F9039B2068596801F0F0FF95
:100FE0006268039B000A10609968206801F0E8FFBE
:100FF0006368000A586008B010BD00BF709A01080D
:10100000436853F82100704700B5102083B004F006
:10101000BBF90A4801A913F0F1FA019B012B09D190
:101020004FF0E0234FF08052C3F8042DBFF34F8FF1
:10103000BFF36F8F03B05DF804FB00BFF0C9012060
:1010400070B588B01F4B204E002500951A6B0160CB
:1010500042F002021A631A6B02F002020092009A36
:1010600001951A6B42F004021A631B6B03F0040330
:101070000193164B4FF48042CDE902230446019BB5
:101080001348022302A90122CDE9042304F03CF80D
:101090002A460921282003F0AFFD01220123CDE9D2
:1010A000022302A9022300223046CDE9042304F0E2
:1010B0002BF801223046114604F058F9204608B0BA
:1010C00070BD00BF0038024000080240000021103F
:1010D0000004024010B5032384B0C94319408022A4
:1010E0008DF806208DF8051000688DF8043001ACED
:1010F00002AA0121CDE9024300F0B6F804B010BD08
:1011000010B584B01344303103220292C3F3072C8C
:101110008DF80C1000688DF80DC003AC01AA0121F8
:1011200001948DF80E3000F09FF804B010BD00BFA0
:101130000160704710B5064C00220121204613F0D3
:1011400067FA2046034A0449BDE81040FFF780BD16
:10115000F0C90120790C0008D90D000810B5054C24
:10116000204654F808391B6898472046FFF734FE9C
:1011700010BD00BFA0CF012010B5054C204654F88B
:1011800008391B6898472046FFF726FE10BD00BFB0
:1011900090CF012010B5054C204654F808391B6843
:1011A00098472046FFF718FE10BD00BF80CF0120F2
:1011B00010B5054C204654F808391B68984720465E
:1011C000FFF70AFE10BD00BF70CF012038B5054CF7
:1011D000A4F1280554F8083D1B6820469847AC4206
:1011E000F8D138BD68CF012000B585B0019271B942
:1011F00001A9042303AA0E4806F02EFF4FF0FF3189
:101200000C4813F0DFF9039805B05DF804FB01A961
:101210000222094806F0B0FE41F234234FF0FF31BC
:101220000648039313F0CEF9039805B05DF804FB6C
:1012300010D00120B0CF0120B8CF0120A8CF0120CD
:1012400008B50AC99B009BB21268054806F004FF66
:10125000BDE8084003484FF0FF3113F0B3B900BFB9
:1012600010D00120B0CF012008B559B911680B4842
:10127000928806F081FEBDE8084009484FF0FF3132
:1012800013F0A0B911680748928806F075FEBDE812
:10129000084005484FF0FF3113F094B910D00120F9
:1012A000B0CF0120B8CF0120A8CF012038B5094820
:1012B000094C0A4A0B464FF48061C55CD25C20465B
:1012C00004F054F82A4620464FF40051BDE8384057
:1012D00004F04CB8E49A010800140240E89A0108AE
:1012E0000A1E034818BF0122202104F03FB800BFA6
:1012F000001002400A1E034818BF0122402104F0DA
:1013000035B800BF0010024000B58BB0264B27480F
:1013100000220092196B41F008011963196B01F06A
:101320000801009100990192196B41F010011963B5
:10133000196B01F01001019101990292196B41F0B2
:1013400020011963196B01F02001029102990392A7
:101350001A6B42F040021A631B6B03F040030393C5
:101360004FF440520123CDE9042304A900220023B5
:10137000CDE90623039B03F0C7FE04A960230C48B4
:10138000049303F0C1FE04A942F20C4309480493FC
:1013900003F0BAFE4FF498430748049304A903F0FE
:1013A000B3FE0BB05DF804FB00380240000C0240B5
:1013B0000010024000140240001802402DE9F04FD6
:1013C00091B00026AF4C0396236BAF48AF4D43F06E
:1013D00001032363236B03F001030393039B049630
:1013E000636C43F480536364636C03F48053A02202
:1013F000022704930AA94FF003094FF0050A049B42
:101400000A924FF00108CDE90C790B97CDF838A07E
:1014100003F07AFE102212239B48CDF830800AA9EF
:10142000CDE90A2303F070FE402397480A930AA9E6
:101430000C9603F069FE4FF482736B604FF48023C7
:10144000AB610823EB610A23EB622846904BAE6048
:10145000EE602E61C5F814802E626E62AE622B6063
:1014600006F048FD002840F00A810590236B894E64
:1014700043F480032363236BF06003F4800305933C
:10148000059B70614023B36003F1804303F519337A
:1014900033604FF0806373604FF4806333614FF4C7
:1014A0000033B061F061F062306333623046042390
:1014B000C6F82890736203F021FC0246002840F031
:1014C000DE80414601903A20DFF8E8B103F094FB5A
:1014D0003A2003F0CFFB019ACBF80820CBF80C2080
:1014E000CBF81420CBF81820CBF81C20CBF82C20FC
:1014F000CBF83020684ACBF8002004234FF0C062BC
:10150000CBF82430CBF804204FF480634FF4403202
:101510005846AE64B563CBF81030CBF82890CBF8C2
:10152000202003F0EBFB0646002840F0A88002468E
:101530004146382003F060FB382003F09BFB324625
:1015400039462320C5F84CB0CBF8385003F054FB93
:10155000232003F08FFB0696236B5048504D43F039
:1015600002032363236B03F002030693069B079693
:10157000236B43F004032363236B03F004030793FB
:10158000079B0896236C43F480432364236C0B97DA
:1015900003F48043082208930AA90A92089BCDF815
:1015A00038A0CDE90C7903F0AFFD4FF400533D486E
:1015B0000A930AA90C96CDF838A003F0A5FD1223D2
:1015C0003848CDF838A04FF480520AA9CDE90A2353
:1015D000CDF8308003F098FD4FF482736B604FF4C8
:1015E0008023AB610823EB610A23EB622E4B2B6057
:1015F00028464FF40043EE602F616E612E626E62EA
:10160000AE62AB6006F076FC002838D10990236BFF
:1016100043F400132363236B244C03F40013099356
:10162000099B60604023A3604FF4806323614FF403
:1016300000332362E0601E4B6061A061E061606284
:10164000E06220632046C4F82890236003F056FB34
:101650000646A0B9414602460F20AC64A56303F0DC
:10166000CBFA0F2003F006FB32463946242003F064
:10167000C3FA242003F0FEFA11B0BDE8F08F03F0A6
:101680005FFA00BF003802400000024010D0012085
:1016900000300140E0CD012010640240000802400B
:1016A000B8CF0120000402400038004020CC0120C7
:1016B0007060024080CD01202DE9F04F8FB0894C41
:1016C000894D8A48002603960A96236C43F400133A
:1016D0002364236C03F400130393039B0496236C8D
:1016E00043F480032364236C03F480030493049B7A
:1016F0000596236B43F002032363236B03F002037D
:101700000593C02212234FF0020A4FF0040908A9E2
:10171000CDE90823CDF82CA0059BCDF8309003F03F
:10172000F3FC734B2B60734B6B606E274FF480435D
:101730002846AE606E61AE61EE612E62EF602B6195
:1017400004F06AF8002840F0CB800690236BDFF8A5
:10175000C881694A43F400132363236BC8F8080067
:1017600003F400130693069BC8F80C00C8F8140095
:10177000C8F81800C8F81C00C8F82400C8F80020F1
:101780004FF480334FF000724FF480664046C8F843
:101790000420C8F81060C8F8203003F0AFFA834680
:1017A000002840F09D80C5F83880C8F83850DFF830
:1017B0006C8102460C210B2003F01EFA4F4AC8F838
:1017C00004B0C8F80CB0C8F814B0C8F818B0C8F81D
:1017D0001CB0C8F820B0C8F824B040464FF0400B09
:1017E000C8F80020C8F81060C8F808B003F086FAFE
:1017F0000246002874D101900D210C20C5F83480D8
:10180000C8F8385003F0F8F912233848099308A9AA
:1018100001230A93CDF82CA0CDF83090089603F060
:1018200073FC4FF40073364D3048089308A9092320
:101830000C9303F069FC2F4B6B604FF48043019ACB
:101840002B6128462F4BEF60AA606A61AA61EA61AA
:101850002A622B6003F0E0FF002841D10790236B40
:1018600043F400132363236B274C03F40013079303
:10187000079BA0604FF480332362244BE0606061DB
:10188000A061E06160624FF060682046C4E9003802
:10189000266103F033FA074610BBAC63A5631C4C0A
:1018A00002460C210D2003F0A7F91A4BC4F804805E
:1018B0002046C4F808B0E76026616761A761E76168
:1018C00027626762236003F019FA024640B90C21CF
:1018D0002F206C63A56303F08FF90FB0BDE8F08F84
:1018E00003F02EF9003802404CCA012000040240E7
:1018F00000540040801A0600106002402860024038
:10190000F8C9012000580040A0CA012040600240F0
:1019100000CB0120B860024060CB0120C0CB012089
:101920002DE9F0418AB000253F4E0195336B3F48C9
:101930003F4C43F001033363336B03F00103019326
:10194000019B0295336C43F400333364336C03F42E
:10195000003302930C220223CDE904230122032346
:10196000CDE9062304A907230893029B03F0CCFBCF
:10197000304AA5604FF4E133C4E9002320460C232C
:10198000E56025616361A561E56106F0B7FF0028A8
:1019900047D10390336B284D43F400133363336B0B
:1019A000A86003F400130393244BE8606861A86106
:1019B000E861286268624FF0006828464FF480674B
:1019C000C5E90038039A2F6103F098F9064640BB39
:1019D00002460D2110206563AC63194D03F00CF92C
:1019E000102003F047F94023AB602846154BC5F89B
:1019F0000480EE602F616E61AE61EE612E626E62F8
:101A00002B6003F07BF9024658B90D2111202563A4
:101A1000AC6303F0F1F8112003F02CF90AB0BDE833
:101A2000F08103F08DF800BF003802400000024052
:101A300040CD01200044004080CC0120886002405D
:101A4000E0CC0120A06002402DE9F0478AB0604E52
:101A50006048614D00240094336B43F0040333630A
:101A6000336B03F004030093009B0194336B43F04A
:101A700040033363336B03F040030193019B0294F3
:101A8000736C43F020037364736C03F02003082726
:101A90000293402202234FF001084FF0030904A9EA
:101AA000CDE90423CDE90689029B089703F02CFBBE
:101AB0004FF4007202234948089704A9CDE9042392
:101AC000CDE9068903F020FB4FF440520223CDE913
:101AD0000423424808970022032304A9CDE90623E2
:101AE00003F012FB3E4A3F4BAC60C5E900234FF4C4
:101AF00000434FF44072EB6128460C23AA61EC606E
:101B00002C616B6106F0FAFE00285FD10390336B05
:101B1000354C43F480033363336BA06003F48003DC
:101B20000393324BE0604FF02069C4E900396061F3
:101B3000A061E061E06220634FF4003320464FF47F
:101B4000806A4FF004080227039AC4F810A02362A9
:101B5000C4F82480A76203F0D1F80646002835D1E6
:101B60000246062139206C63A563214C03F044F83A
:101B7000392003F07FF840231E4AA36020464FF42B
:101B80008033E6606661A661E661E6622663C4F8BA
:101B90000490C4F810A0C4F82480A76222602362D5
:101BA00003F0ACF8064688B90246062146202C63AD
:101BB000A56303F021F8462003F05CF832460A21C1
:101BC000472003F019F80AB0BDE8F08702F0B8FF2B
:101BD000003802400008024000CF012000180240F7
:101BE0000014014080841E0040CE01202864024081
:101BF000A0CE0120B864024030B5044683B001F0A5
:101C00007DFD40F20E2204F5AA700021C4F8502197
:101C1000C4F84C01012516F0FFFD02F08FFF1549B5
:101C20000095802304F55972002002F04FFF002830
:101C300011DA2046FFF768FB2046FFF7BFFB20467E
:101C4000FFF73AFD2046FFF76BFE2046FFF7FCFE4C
:101C5000204603B030BD08490095802304F5797211
:101C6000284602F033FF0028E3DB0449002002F09D
:101C70000FFFDEE77C9A01088C9A01089C9A010804
:101C8000026808491368884223F04003136003D0B8
:101C9000054B984203D07047044801F001BB04484B
:101CA00001F0FEBA10D00120B8CF0120B0CF012042
:101CB000A8CF0120054B984200D070470268044825
:101CC000136823F04003136001F0EABA10D001203A
:101CD000B0CF0120014804F017BA00BF4CCA012060
:101CE000014804F0FFBE00BF4CCA0120014804F0C7
:101CF0000BBA00BFF8C90120014804F0F3BE00BFD1
:101D0000F8C90120014806F04BBB00BF10D00120EC
:101D1000014806F045BB00BFB8CF012008B5044814
:101D200006F066FEBDE80840024801F0B9BA00BFFF
:101D300040CD012098CF012070B5104C94F83A5056
:101D400094F83930EDB22046DEB206F051FE222D75
:101D50000BD0212E00D070BD94F83930202BFAD151
:101D6000BDE87040064801F09BBA94F83A30202B49
:101D7000F1D1BDE87040034801F092BA00CF0120D4
:101D800090CF012088CF012010B5074C204603F0EA
:101D9000E1F894F83530012B00D010BDBDE81040BB
:101DA000024801F07DBA00BF60CB012078CF01204E
:101DB00010B5074C204603F0CDF894F83530012BD0
:101DC00000D010BDBDE81040024801F069BA00BF64
:101DD000C0CB012080CF012010B5074C204603F076
:101DE000B9F894F83530012B00D010BDBDE8104093
:101DF000024801F055BA00BFA0CA012068CF0120F7
:101E0000014803F0A7B800BF20CC012010B5074C53
:101E1000204603F09FF894F83530012B00D010BD18
:101E2000BDE81040024801F03BBA00BF80CC012061
:101E300098CF012010B5074C204603F08BF894F89A
:101E40003530012B00D010BDBDE81040024801F034
:101E500027BA00BF00CB012070CF0120014803F05A
:101E600079B800BF80CD012010B5094C204603F0A1
:101E700071F894F83530012B00D010BD054B0648A1
:101E80002022BDE8104083F8392001F009BA00BFD4
:101E900040CE012000CF012088CF0120014803F06F
:101EA00059B800BFE0CD012010B5094C204603F021
:101EB00051F894F83530012B00D010BD054B064881
:101EC0002022BDE8104083F8392001F0E9B900BFB5
:101ED000A0CE012000CF012090CF012010B50446F4
:101EE000FFF78AFE214604F26440FEF78DFF21468B
:101EF00004F27C40FFF7A4F8214604F59060FFF758
:101F000017F9204610BD00BF38B500220121304826
:101F1000304C12F07DFB304A30492D48FEF798FED8
:101F2000002201212E4812F073FB2B4A2B492C482A
:101F3000FEF78EFE002201212A4812F069FB0022E2
:101F40000121294812F064FB234A28490020FEF7AA
:101F50007FFE00220121264812F05AFB00220121B7
:101F6000244812F055FB1C4A23490020FEF770FE5E
:101F700000220121214812F04BFB002201212048C0
:101F800012F046FB144A1F490020FEF761FE0022B2
:101F900001211D4812F03CFB002201211B4812F0D8
:101FA00037FB0D4A1A490020FEF752FE04F12805BE
:101FB000204600220121083412F02AFBAC42F7D15E
:101FC000BDE83840044A13490020FEF741BE00BF77
:101FD000B0CF012040CF0120790C0008D90D0008B6
:101FE000A8CF012098CF0120A0CF01205D110008CB
:101FF00088CF012090CF01207911000878CF0120EF
:1020000080CF01209511000868CF012070CF0120FA
:10201000B1110008CD110008B420704710B4B328E6
:10202000144C94BF84464FF0000CA4F800C0B329B0
:10203000114C94BF8C464FF0000CA4F800C014184B
:10204000B42CDCBF02F1FF32801803EB0102D4BFD5
:1020500080B2B320B42ADCBF03F1FF33C918074CA8
:10206000074B2080D4BF89B2B3215DF8044B19809F
:10207000704700BF6AD0012068D001200200002014
:102080000000002008B501F0C9FC4FF6FF7008BD44
:10209000B420704708B5292001F04CFDBDE8084088
:1020A000382001F047BD00BF08B5282001F042FDEF
:1020B000142001F04BFD102001F03CFDBDE808406C
:1020C000962001F043BD00BFF0B5C0B283B000223E
:1020D00000F11E04A0F12F032A208DF805400F46C1
:1020E0008DF804208DF806208DF8073001F022FDD0
:1020F00001AC02AE254615F8010B01F015FDB54205
:10210000F9D1F9B2A1F14D032B208DF805108DF80E
:10211000073001F00FFD14F8010B01F005FDB4428A
:10212000F9D103B0F0BD00BF38B5D50802F478434B
:1021300005F0FC051D441446ADB2FFF7C5FF2C2089
:1021400001F0F8FC284601F0EFFCE00200F47840D2
:10215000BDE8384001F0E8BC2DE9F8430546C60A61
:1021600005F01F08F60008461F4606EBC826C5F313
:10217000451311464FEAC80805F4784505EB830579
:1021800008EB8328FFF7A0FF2C20B6B2ADB21FFAF0
:1021900088F801F0CFFC8FB107F1FF390024284601
:1021A00001F0C2FC304601F0BFFC4C45404601D076
:1021B00001F0BAFC0234A4B2A742F0D8BDE8F8831B
:1021C00038B504460D46FFF77FFF29462046FFF746
:1021D0007BFF2E2001F0AEFC01F0B2FC01F0B0FC60
:1021E000044601F0ADFCC4F38502C0F3C42303EB45
:1021F000421304F47844181980B238BD2DE9F04F29
:102200000446151983B02C200F46994601F092FC24
:10221000A54219DD254EDFF89C80DFF89CA0244AFA
:102220004FF0000B3188A1420AD8B8F80010B9422B
:1022300006D8BAF80010A14202D31188B94206D2DA
:102240000234A4B2AC42EDDB03B0BDE8F08F39F844
:102250001B10C80800F0FC0001F4784108444FEA64
:102260004B03023380B2019301F05EFC019B39F80D
:102270001B0039F80310C002C90A00EBC10080B28C
:1022800001F052FC691EA142094A0BF1020BD7D0A2
:10229000019B39F80310C800C0B2490900EB812046
:1022A00080B201F041FC024ACAE700BF6AD00120B7
:1022B0000000002068D0012002000020364B2DE9EC
:1022C000F04F364C1B8824885588958801331B1B9A
:1022D000334C1FFA83FE334BB4F800C01B880CF15B
:1022E000010CACEB030C5389948911FA8CFC9BB262
:1022F0008C4589B043EA04434BD9D718C3B203F1E4
:102300001E0A2F3BDBB20CF1FF395FFA8AFA019308
:102310004FEA4E031FFA89F602934FF0000808AD0A
:10232000CDF80CE0CDF810A005908B46049B8DF8FD
:102330001D302A20019B8DF81C808DF81E808DF8A1
:102340001F3001F0F7FB07ACA2461AF8010B01F0B1
:10235000EBFB5545F9D1F2B28DF81D202B204D3AFB
:102360008DF81F2001F0E6FB14F8010B01F0DCFBF7
:10237000A542F9D1029A05983B4631461744039A83
:10238000FFF73CFF013ED945B6B202D909F1FF394A
:10239000CCE709B0BDE8F08F020000206AD0012030
:1023A0000000002068D001202DE9F04F01EB030B65
:1023B000594589B0894643D2C3B203F11E0A2F3B67
:1023C000DBB25FFA8AF10193129E029153000393EC
:1023D000002708AD04900592029B8DF81D302A203D
:1023E000019B8DF81C708DF81E708DF81F3001F068
:1023F000A1FB0DF11C081FFA89F4C2461AF8010B63
:1024000001F092FBAA45F9D15FFA89F28DF81D20FF
:102410002B204D3A8DF81F2001F08CFB18F8010B92
:1024200001F082FBA845F9D1039A0498334621466E
:1024300009F101091644059AFFF7E0FED945CBD30F
:1024400009B0BDE8F08F00BF2DE9F04F0C4687B012
:102450001146054620469A461646FFF735FE2C20C3
:1024600001F068FBBAF1000F48D0EB0805F47842A0
:1024700003F0FC031344E4B2ED029BB204F11E0B23
:1024800001932F3CABB24D3E02930027E3B2F6B26C
:102490005FFA8BFB0393B94606AD039B8DF814904E
:1024A0002A208DF815B08DF816908DF8173001F0B0
:1024B00041FB05ACA04618F8010B01F035FB454582
:1024C000F9D106F14D032B208DF815308DF81760EA
:1024D00001F030FB14F8010B01F026FBA542F9D105
:1024E0002C2001F027FB019801F01EFB0137029818
:1024F00001F01AFB01365745F6B2CED107B0BDE860
:10250000F08F00BF70B582B001F088FA352001F07D
:1025100011FB002001F008FB3A2001F00BFB062024
:1025200001F002FBB02001F005FB012001F0FCFAF4
:10253000FE2001F0F9FAB12001F0FCFADE2001F0F2
:10254000F3FA212001F0F0FAB72001F0F3FA0520A8
:1025500001F0EAFA332001F0E7FAB82001F0EAFAD4
:10256000052001F0E1FA332001F0DEFAC82001F085
:10257000E1FA042001F0D8FA032001F0D5FAC920CD
:1025800001F0D8FA5E2001F0CFFA082001F0CCFA71
:10259000CA2001F0CFFA0A2001F0C6FA0C2001F09F
:1025A000C3FA022001F0C0FACC2001F0C3FA0320E4
:1025B00001F0BAFA042001F0B7FAD02001F0BAFA1B
:1025C0000C2001F0B1FAB32001F0B4FA022001F0BE
:1025D000ABFAC02001F0AEFA532001F0A5FAC520F5
:1025E00001F0A8FA002001F09FFA452001F09CFAC2
:1025F000C22001F09FFA032001F096FA122001F0A8
:1026000093FADD2001F096FA002001F08DFAB42053
:1026100001F090FA112001F08DFA962001F096FA5F
:102620001C4B01932A2001F085FA01AC02AE25462D
:1026300015F8010B01F078FAB542F9D10022B32365
:102640002B208DF805208DF8073001F073FA14F86F
:10265000010B01F069FAB442F9D1362001F06AFAAF
:10266000832001F061FA292001F064FA382001F09A
:1026700061FA2C2001F05EFA4BF6D854002001F0EC
:1026800053FA013CFAD1142002B0BDE8704001F0C9
:102690005DBA00BF001E00D1F020704710B4EF28D3
:1026A000144C94BF84464FF0000CA4F800C0EF29EE
:1026B000114C94BF8C464FF0000CA4F800C01418C5
:1026C000F02CDCBF02F1FF32801803EB0102D4BF13
:1026D00080B2EF20F02ADCBF03F1FF33C918074CAA
:1026E000074B2080D4BF89B2EF215DF8044B1980DD
:1026F000704700BF6ED001206CD001203E0000204A
:102700003C000020F020704708B501F087F9042054
:1027100001F010FA01F014FA01F012FAC0B208BD8B
:1027200008B5292001F006FABDE80840112001F0A3
:1027300001BA00BF08B5BD2001F0FCF9FE2001F090
:10274000F3F9102001F0F6F9BDE808400A2001F085
:10275000FDB900BFF0B5C3B283B00022A3F11104EC
:102760002A208DF807400F468DF804208DF805309B
:102770008DF8062001F0DEF901AC02AE254615F811
:10278000010B01F0D1F9B542F9D1F9B2A1F1110370
:102790002B208DF805108DF8073001F0CBF914F8D7
:1027A000010B01F0C1F9B442F9D103B0F0BD00BF93
:1027B00010B51446FFF7CEFF2C2001F0BBF92046E0
:1027C000BDE8104001F0B0B970B5064608461146A4
:1027D0001D46FFF7BFFF2C2001F0ACF935B10024F6
:1027E0003046013401F0A0F9AC42F9D170BD00BF10
:1027F0002DE9F04F0446151983B02C200F46994659
:1028000001F098F9A54219D9124EDFF84C80DFF893
:102810004CA0DFF84CB000233288A2420BD8B8F8A5
:102820000020BA4207D8BAF80020A24203D3BBF86E
:102830000020BA4205D20134A542EDD803B0BDE86C
:10284000F08F39F81300019301F06EF9019B013309
:10285000F1E700BF6ED001206CD001203E000020C7
:102860003C000020354B2DE9F04F354C1B88248867
:102870005588958801331B1B324C1FFA83FE324B5F
:10288000B4F800C01B880CF1010CACEB030C5389AD
:10289000948911FA8CFC9BB28C4589B043EA0443BD
:1028A00048D902EB0308C2B20CF1FF3BA2F1110AB6
:1028B0004FEA4E035FFA8AFA1FFA8BF701934FF043
:1028C000000908AECDF808E0039204900591039B3F
:1028D0008DF81C902A208DF81D308DF81E908DF8F3
:1028E0001FA001F027F907AC254615F8010B01F0F0
:1028F0001BF9AE42F9D1FAB28DF81D202B20113A06
:102900008DF81F2001F016F914F8010B01F00CF9F5
:10291000A642F9D1019A0498434639469044029A56
:10292000FFF766FF059B013F9B45BFB202D90BF144
:10293000FF3BCCE709B0BDE8F08F00BF3E000020B0
:102940006ED001203C0000206CD001202DE9F04F1A
:1029500001EB030C614589B08B4642D2C1B2A1F1B3
:10296000110A5300129F01935FFA8AFA4FF0000890
:1029700008AECDF808C0039104900592039B8DF832
:102980001C802A208DF81D308DF81E808DF81FA028
:1029900001F0D0F807AD1FFA8BF4A94619F8010B26
:1029A00001F0C2F8B145F9D15FFA8BF28DF81D2024
:1029B0002B20113A8DF81F2001F0BCF815F8010BFF
:1029C00001F0B2F8B542F9D1019A04983B4621468C
:1029D0001744059AFFF70CFF029B0BF1010B9B4577
:1029E000CCD309B0BDE8F08F38B504460D46FFF7EB
:1029F000B1FE29462046FFF7ADFE2E2001F09AF8E1
:102A000001F09EF801F09CF8044601F099F8C4F337
:102A10008502C0F3C42303EB421304F4784418196D
:102A200080B238BD2DE9F04F85B08946009011463F
:102A300048469A461446FFF78DFE2C2001F07AF89E
:102A4000BAF1000F39D05FFA89F9A9F1110B113CE5
:102A50005FFA8BF300270193E6B2B84604AD019B01
:102A60008DF80C802A208DF80D908DF80E808DF851
:102A70000F3001F05FF803ACA3461BF8010B01F027
:102A800053F85D45F9D106F111032B208DF80D3077
:102A90008DF80F6001F04EF814F8010B01F044F8C6
:102AA000A542F9D12C2001F045F80137009801F03A
:102AB0003BF801365745F6B2D1D105B0BDE8F08FED
:102AC00070B584B000F0AAFF102001F033F80A209E
:102AD00001F03CF8012001F02DF8C82001F036F893
:102AE000112001F027F8782001F030F8362001F0AD
:102AF00021F8002001F018F83A2001F01BF8052019
:102B000001F012F8212001F015F84FF06F432A2050
:102B1000009301F00FF801AD6C4614F8010B01F0C1
:102B200003F8AC42F9D12B2001F004F86C4614F8FC
:102B3000010B00F0F9FFAC42F9D1332340F60C420F
:102B4000B220ADF800208DF803308DF8043000F08D
:102B5000F1FF0DF105056C4614F8010B00F0E4FFE0
:102B6000A542F9D1B72000F0E5FF352000F0DCFFE9
:102B7000BB2000F0DFFF1F2000F0D6FFC02000F0D8
:102B8000D9FF2C2000F0D0FFC22000F0D3FF01209D
:102B900000F0CAFFC32000F0C7FFC42000F0CAFF46
:102BA000202000F0C1FFC62000F0C4FF0F2000F07D
:102BB000BBFFD02000F0BEFFA42000F0B5FF2248EC
:102BC0002249234A0292CDE9000142F62953E0202E
:102BD000ADF80C3000F0AEFF0DF1FF340DF10D0635
:102BE000254615F8010F00F09FFFAE42F9D140F2E3
:102BF00006631022ADF8043040F6513344218DF8BD
:102C00000220ADF80830162243F22F13E1208DF890
:102C100007108DF80A20ADF80C3000F08BFF14F887
:102C2000010F00F081FFA642F9D1292000F082FFB8
:102C3000112000F07FFF352000F07CFF002004B061
:102C4000BDE8704000F070BFD00811080C15393392
:102C50005036131430B5012883B00BD002280BD0A6
:102C60006024362000F066FF204603B0BDE8304007
:102C700000F05ABF0024F4E70D4A009200233320ED
:102C8000ADF8043000F056FF6C460DF1060514F85F
:102C9000010B00F049FFA542F9D1372000F04AFFAF
:102CA000002000F041FF502000F03EFFC024D8E794
:102CB000000001F038B5054CA4F1280554F8083D92
:102CC0001B6820469847AC42F8D138BD60D101203E
:102CD00010B5E9B1012926D0164C174A002332F865
:102CE0001110E1604FF44862204662602361A360E6
:102CF00005F06EFD0246D0B90E212C2001F07CFFBC
:102D0000204605F01FFCBDE810402C2001F0B2BFAA
:102D1000032000F0C9FD2C2001F0BAFFBDE81040EF
:102D2000044805F01FBC032000F0B2FDF3E701F0FA
:102D300007FF00BFE4D10120009B01080329F8B57B
:102D400015460EDD224C234F04F1100654F8042BD7
:102D5000012D134610D1B85C00F09AFDB442F5D1B4
:102D6000F8BD012A2ED0022A26D04AB9194B585C48
:102D7000BDE8F84000F098BD022D164F02D075B1A5
:102D800001F0DEFEF85C00F09BFDA642E8D054F8AE
:102D9000043BF85C00F094FDA642F8D1F8BDF85C65
:102DA00000F082FDA642DBD054F8043BF85C00F052
:102DB0007BFDA642F8D1F8BD064B585CBDE8F84053
:102DC00000F07EBD034B585CBDE8F84000F060BDEC
:102DD000EC9A0108FC9A0108F0B44FF060434FF000
:102DE000E025D3F8000ED5F8FC4D154E154F44F0F4
:102DF0008074C5F8FC4D4FF0010C134CC3F8B04F74
:102E00000CFA02F2114C20EA0200002501394FF0C1
:102E1000020CC3F8000E0243C3F8805E0C48C4F8ED
:102E2000F0C021614FF48071C3F8405E3760C4F890
:102E30000413C3F8800EF0BCC3F8002E704700BF27
:102E4000001000E0FE03004055CEACC5000004E0D9
:102E50000D000100F0B5A5B0364A374B00240194AF
:102E6000106C40F080501064126C02F0805201929D
:102E7000019A02941A6842F440421A601B68119148
:102E800003F440430D204FF4A021022402930425B3
:102E90000123CDE908014FF4800608A8CDE90E46CC
:102EA000CDE91245029A0A930D931095149404F0FB
:102EB00019FD00283BD14FF48053059007900F2750
:102EC000032103A806930397049404F0DDFA034654
:102ED00068BB032218921D934FF4807222936823DB
:102EE0001C9215934FF00062482315A8199416956B
:102EF0001F92179304F0AAFB0446C0B9314602465C
:102F000004F038FA04F086FA04F058FB0B4BA3FBEC
:102F10000030800901F0CAFE284601F0E3FE224697
:102F200039464FF0FF3001F067FE25B0F0BD01F0EB
:102F300007FE00BF0038024000700040D34D621011
:102F400038B505462D200C4601F0A2FE002001F008
:102F5000A1FC44B930BF2D2001F08CFEBDE8384003
:102F6000012001F097BC0121002003F09BFE6021AD
:102F70002846FFF76FFFEEE738B5FFF7E1FF074D93
:102F800001242846002111F01DFB083520B9013429
:102F9000052CF6D1062038BD204638BD40D1012091
:102FA000132908B501D9022008BD04F0DBFE00207A
:102FB00008BD00BF132901D90020704704F0D8BE16
:102FC00008BA704730B589B0194C1A4800250095E9
:102FD000236B43F010032363236B03F01003009370
:102FE0000F22012302A9CDE9022301220023CDE90A
:102FF0000423009B02F088F8284600F055FC0120CD
:1030000000F052FC022000F04FFC032000F04CFCCA
:103010000195236C084A094943F080032364236C1B
:10302000116003F080030193019B09B030BD00BF24
:103030000038024000100240E4D10120001C004092
:103040002DE9F0438BB03D4B002500951A6B42F003
:1030500002021A631A6B02F002020092009A0195B2
:103060001A6B42F020021A631A6B02F020020192DE
:10307000019A02951A6B42F040021A631A6B02F031
:1030800040020292029A03959A6B42F002029A63FE
:103090009B6B03F002030446002603270393C02220
:1030A00027484FF0090904A90223CDE904234FF072
:1030B0000A08039BCDF82090CDE9066702F024F8BA
:1030C0004FF4407202231E48CDF8208004A9CDE9B8
:1030D0000423CDE9066702F017F8042202231948F9
:1030E000CDF8209004A9CDE90423CDE9066702F0CC
:1030F0000BF8402202231448CDF8208004A9CDE922
:103100000423CDE9066701F0FFFF04230F49A36301
:103110001022172321636563E26323646564A56459
:10312000E564256504F1300003F082FE20B901F06A
:1031300081F90BB0BDE8F08301F002FD00380240D8
:10314000001402400004024000180240001000A0D9
:1031500000B583B00B4B002201925A6B42F0400243
:103160005A635B6B084A40F87C2F03F040030193DD
:10317000019B04F06FFD10B903B05DF804FB01F092
:10318000DFFC00BF003802400008065070B588B070
:103190000026184B02961A6C174C42F480721A647F
:1031A0001B6C03F480730D46029301A903A8029BD4
:1031B00004F02AFA04F008FA104A226040F2E732DA
:1031C000E2600F4A26614300A2FB03239B0C013BF4
:1031D00020466360A66005F0FBFA042229462D20F4
:1031E00001F00AFD2D2001F045FD204605F0AAF969
:1031F00008B070BD0038024060D1012000200040BE
:1032000083DE1B4338B504460D4601F00FFB214B0E
:103210001A6842F400721A601A6842F480621A60F6
:103220001A6842F480721A60032001F0D3FC0F2167
:103230002046FFF7ABFF29462046FFF70BFE04F0C0
:10324000E9F8002208212046FFF7C6FD012000F022
:1032500043FB2046FFF7B6FE2046FFF7F1FE20466F
:10326000FFF776FF0C4A0D480121C2F83C1E0023EF
:103270007F21FF22C4E90003A160E2602361636152
:10328000A361204604F002FD08B9204638BD01F0D4
:1032900057FC00BF003C02400000474200280040AD
:1032A00000B583B001A911F0A9F958B1019B4BB148
:1032B0004FF0E0234FF08052C3F8042DBFF34F8F3F
:1032C000BFF36F8F03B05DF804FB00BFFEE700BFE4
:1032D000FEE700BFFEE700BFFEE700BFFEE700BF5E
:1032E000704700BF70B5124D012002F04DF800F09C
:1032F0007FFB2B68BFF35B8FDB07044608D50D4EC1
:1033000030680D4BBDE8704003EBC000FFF7C8BF4D
:103310002846FDF791FC074E0028F1D0003C18BF6D
:103320000124A40028463460FDF78CFCE8E700BFC8
:1033300070D0012074D0012038D1012008B50220BE
:1033400002F022F8BDE808400148FFF7A9BF00BF1E
:1033500040D1012008B50E4B5B695A0404D40C4BD4
:103360005B691B040BD408BD4FF4804002F00CF8DD
:103370000848FFF795FF064B5B691B04F3D54FF434
:10338000004002F001F8BDE808400348FFF788BF9D
:10339000003C014050D1012048D1012008B503482C
:1033A00005F000F9024B01221A7008BDA4D10120DA
:1033B000A0D1012008B5044805F0F4F8BDE80840A4
:1033C000032000F07DBA00BFE4D1012008B5034816
:1033D00005F0E8F8BDE8084001F0D8BB60D1012055
:1033E000014801F0B7BD00BF78D00120014801F0CD
:1033F000B1BD00BFD8D0012038B5094C04F1280573
:10340000204600220121083411F002F9AC42F7D124
:10341000BDE83840034A04490020FDF719BC00BF4D
:1034200038D10120790C0008B52C000810B54FF6F2
:10343000FF7000F087FD002000F06EFC4FF6FF707B
:1034400000F070FC084800F073FC084A0123642176
:10345000002000F0F3FCBDE81040054A012378216C
:10346000002000F0EBBC00BF800000200C9B010896
:10347000189B010870B504460D4603E0237883B11C
:1034800001F096FB204601F099F803466420002BDA
:10349000F6D1002DF2D0012DF2D12378013B012B82
:1034A000EED801F07FFB86B2204601F087F80028B5
:1034B000FAD175B92378013B012B0FD901F072FBCA
:1034C0006438B0424FF0640010D9BDE8704001F09C
:1034D0006FBB012DF2D12378002BEFD1642001F0D6
:1034E00067FBBDE87040642001F062BB01F060FB47
:1034F000DAE700BFF8B5174C34F811500446002045
:103500001E46174600F008FC29461422284600F003
:10351000CFFD4FF6FF7000F0FFFB0A222946284638
:1035200000F0C6FD20460121FFF7A4FF63883B8021
:10353000E388338000212046FFF79CFF4FF6FF70A1
:1035400000F0EAFB294628461422BDE8F84000F0C6
:10355000AFBD00BF989B010838B500210446C06884
:10356000FFF728FD00283ED0030C6082A382E068AC
:1035700001210125FFF71EFD00283BD12046FFF762
:1035800055FF00F0B9FB054600F0BEFB012281B2F9
:10359000A8B200F0E7FF0546002833D123460146D4
:1035A00003F8140B04F112022046FFF7A3FF638A0D
:1035B000A28AE06843EA02422946FFF7F1FC23466B
:1035C00004F1160203F8185B01212046FFF792FF71
:1035D000E38A228BE06843EA02420121FFF7E0FC24
:1035E0000120207438BD05460121E068FFF7E2FCA8
:1035F0000028C3D0030CE0822383002DBED001201D
:10360000207438BD4FF6FF7000F08CFB4FF478400B
:1036100000F082FB164A01239121002000F00EFCED
:10362000144A0123A021002000F008FC012D17D02E
:10363000022D0AD000F068FBA0F141010E4A0123DF
:1036400089B2002000F0FAFBCAE700F05DFBA0F1B0
:1036500041010A4A012389B2002000F0EFFBBFE7D5
:10366000074A2B46AF21002000F0E8FBB8E700BF77
:10367000249B01082C9B0108809B01086C9B01087E
:10368000509B010838B5054600F0E6FD0CF0FEFA47
:1036900000F032FB044600F037FB022281B2A0B2F8
:1036A00000F060FF00B138BD2846FFF755FFBDE8C8
:1036B000384001F01DB800BF10B50E4B5C6982B0F8
:1036C000202001F061FEA30601D402B010BD0A481B
:1036D00001A910F093FF019B012BF6D14FF0E023DD
:1036E0004FF08052C3F8042DBFF34F8FBFF36F8F9D
:1036F00002B010BD003C014024D2012010B582B0C0
:103700000446FFF77FFD00210B4B01911A6B84F8F3
:10371000401142F48052C4F83C411A631B6B03F41D
:1037200080530193019B10F0B9FE042006F068FC61
:10373000204602B010BD00BF0038024010B5064C54
:1037400000220121204610F063FF2046034A04496D
:10375000BDE81040FDF77CBA24D20120790C0008A6
:10376000D90D000830B5474B474C83428BB04FF022
:10377000000545D00295236B444843F002032363C0
:10378000236B03F0020302934FF480621223CDE90E
:10379000042300220223CDE9062304A9042308936D
:1037A000029B01F0B1FC4FF4007304A90493374865
:1037B0000923089301F0A8FC0395236C43F48003CC
:1037C0002364236C03F480030393039B236A43F471
:1037D00080032362236A23F4800323622A460F2195
:1037E000212001F009FA212001F044FA2A460F2194
:1037F000222001F001FA222001F03CFA0BB030BD8A
:103800000095236B214843F002032363236B03F0ED
:103810000203009340221223CDE904230022022355
:10382000CDE9062304A904230893009B01F06CFC56
:1038300004A980231548049301F066FC0195236CCC
:1038400043F400132364236C03F400130193019BDE
:10385000236A43F400132362236A23F400132362D0
:103860002A460F211F2001F0C7F91F2001F002FA9C
:103870002A460F21202001F0BFF9202001F0FAF99B
:103880000BB030BD2CD201200038024000040240B1
:103890000246034B034833F82210002201F066BDB4
:1038A000C49B0108001002400246034B034833F852
:1038B0002210012201F05ABDC49B010800100240F1
:1038C0000246034B034833F8221001F053BD00BFFA
:1038D000C49B0108001002402DE9F04702228CB081
:1038E0000223DFF808813D4D3D4FCDE90823064610
:1038F00008F105094446A4EB0803032B60D8DFE870
:1039000003F041341D02374B002204921A6B42F03F
:1039100020021A631B6B03F020030493049B37F807
:10392000023B0693DEB1012E39D001344C4505F13E
:103930000405E0D100200CB0BDE8F087294B00223F
:1039400003921A6B42F020021A631B6B03F02003F0
:103950000393039B37F8023B0693002EE3D12868BC
:10396000079606A901F0D0FBDFE71E4B002202926A
:103970001A6B42F040021A631B6B03F04003029380
:10398000029BCCE7174B002201921A6B42F0010216
:103990001A631B6B03F001030193019BBFE7124BFA
:1039A0002868079306A901F0AFFB94F900A0002254
:1039B00050460F2101F020F9504601F05BF9B4E7C1
:1039C000084B002205921A6B42F040021A631B6BEF
:1039D00003F040030593059BA1E700BFB09B0108DE
:1039E000A49B010800380240000011109C9B0108B4
:1039F00070B5084E084D002435F8021B56F8040B2C
:103A000001F0AEFC20B90134052CF5D1204670BD83
:103A1000E0B270BDB09B0108A49B010810B53D4900
:103A2000AEB04FF02040CDE91A010222022324213A
:103A30000124CDE90E23CDE916230C9100230920A2
:103A40001021CDE91C33CDE92033CDE922330A9092
:103A50001F91CDE9124407204FF480412E4A149063
:103A600026914FF480504FF4001110931593189342
:103A70001E932593279328932B93299301932490A6
:103A80000B940D942A91916B244821439163916B7F
:103A90002140019101990293116B41F008011163DA
:103AA000116B01F00801029102990393116B41F02F
:103AB00010011163116B01F010010391039904933C
:103AC000136B43F020031363136B079403F020037D
:103AD000049302230693032308930C2305A9099357
:103AE0004CF2B373049A059301F00EFB4FF680730A
:103AF00005A90B48059301F007FB05A909480594A2
:103B000001F002FB12AA0AA91AA804F0EDFC2EB0DB
:103B100010BD00BF040100A000380240000C0240AC
:103B200000100240001402404FF0C0435880BFF321
:103B30004F8F70474FF0C0431880BFF34F8F7047CF
:103B40004FF0C043588880B2704700BF01F030B8D2
:103B500010B50E4C204603F0A1F80346A0B90C485E
:103B60000C49A360C4E900014FF480422046E360A1
:103B700022616361A361E3612362FFF7F3FD2046E5
:103B8000BDE8104001F048BE10BD00BF2CD201209E
:103B900000540040A086010010B586B04FF47A733F
:103BA000174C0293944601230A4601460DF1170073
:103BB0000090019320468DF817C001F00FFF08B95F
:103BC00006B010BD204601F0EFFE204603F066F877
:103BD00003460028F4D10B490B48A360C4E9000157
:103BE0004FF480422046E36022616361A361E36198
:103BF0002362FFF7B7FD204601F00EFE06B010BDB0
:103C00002CD20120A08601000054004030B587B0BE
:103C10001A4C0A46002101234FF47A758DF81710CB
:103C200001460DF11700009002950193204601F026
:103C30007DFF18B99DF8170007B030BD204601F090
:103C4000B3FE204603F02AF803460028F2D10C49BF
:103C50000C48A360C4E900014FF480422046E360B1
:103C600022616361A361E3612362FFF77BFD20466C
:103C700001F0D2FD9DF8170007B030BD2CD2012015
:103C8000A08601000054004030B5184D85B04FF4B7
:103C90007A74CDE9002302940A460123014628469E
:103CA00001F044FF044610B9204605B030BD284657
:103CB00001F07AFE284602F0F1FF03460028F3D116
:103CC0000B490C4AAB60C5E9001228464FF480420C
:103CD000EB602A616B61AB61EB612B62FFF742FD28
:103CE000284601F099FD204605B030BD2CD20120B8
:103CF00000540040A086010008B5024B1B689B6A77
:103D0000984708BD80D2012008B5024B1B68DB6ACA
:103D1000984708BD80D20120014B1860704700BF52
:103D200088D20120014B5860704700BF88D2012023
:103D3000014B9860704700BF88D201202DE9F04FF9
:103D40003C4B9C6887B0B4F804A00491A2F1200316
:103D50000AF10701E28805904FEAE10C02FB03F348
:103D6000CAEBCC0120680CFB03F3C9B2002A53D084
:103D7000013901EB0A09DFF8C0B0039218440021B1
:103D800007E0BAF1000F4CD1039B01318B42604434
:103D900042D0049BBCF1010F03EB0107BFB23ED040
:103DA000BCF1020FEDD10678437846EA032676BAD5
:103DB000B6B2059CCDF800C000254FF00108019176
:103DC00002900BE05B693946204613B1194A12880C
:103DD0009847013501345545A4B214D2A9EB050327
:103DE00008FA03F33342DBF80030EBD15B6920467D
:103DF0003946002BEDD00F4A01359288984701349F
:103E00005545A4B2EAD30199039BDDF800C002989E
:103E100001318B426044BCD107B0BDE8F08F067819
:103E2000C7E746780378360246EA034683781E439E
:103E3000BFE700BF88D2012080D201202DE9F047E2
:103E4000174612F8014B064688461D461CB110461F
:103E500014F084FD441CDFF88C90DFF88CA0D9F8B6
:103E600000309B6A9847DAF80830012D9B88B0FB38
:103E7000F3F030D0022D04D1001B10FB03F39B1B89
:103E80009EB233B2002B07F1FF37D8BF01260024C2
:103E900009E03A78FFF752FFDAF808309B880134DE
:103EA0003344A4B29EB2D9F8003017F8015F9B6A80
:103EB000003D18BF01259847DAF80820928803468C
:103EC00002FB14339BB293423046414601D3002D8E
:103ED000DFD1BDE8F087001B00FB03F306EB5303C3
:103EE0009EB2CEE780D2012088D201202DE9F04792
:103EF000DFF84CA0DAF800502C6A074688461646D0
:103F000044B10E4A33461088A4460A463946BDE8F5
:103F1000F04760477AB1DFF8249001E0DAF800500A
:103F20006B693819414680B2013413B1B9F80020E9
:103F30009847A642F2D1BDE8F08700BF88D20120A1
:103F400080D201202DE9F041DFF838800C4ED8F8FE
:103F500000303768DB6A30609847054660B100245E
:103F6000D8F800309B6A9847A1B20246013400207D
:103F7000FFF7BCFFAC42F3D1BFB23760BDE8F081C0
:103F800088D2012080D201202DE9F04F530087B064
:103F9000C3F10303CDE90001424C434F0293924623
:103FA0004FF000090CE0029BA9EB0A020A330AF168
:103FB000FF3A09F1010903EB8203CA4502936ED36C
:103FC0003B6822685B69002B5CD0009901981FFA5E
:103FD00089F51FFA8AF601EB050BA0EB06081FFA1C
:103FE0008BFB1FFA88F892B24146584698473B68C7
:103FF00000995B694A1B92B210462288002B41D07F
:1040000041460390984700993B6872181FFA82FC5A
:10401000019A5B69511B6046228889B2002B31D01E
:104020000591CDF810C098473B6800995B692288DC
:10403000A1EB06081FFA88F823B305994046984774
:104040003B68019A5B691644B6B22288D3B15846E0
:10405000314698473B6822885B699BB1039831469B
:1040600098473B68019A5B691544ADB222884BB111
:104070000498294698473B6822885B6913B1294612
:1040800040469847094BA360029B002B8BDA06330E
:1040900003EB890309F10109CA45029390D207B0E5
:1040A000BDE8F08F88D2012080D201207800002066
:1040B0002DE9F04FDFF8C49083B0B9F80030C9F8AB
:1040C0000030550082468846C5F103051646002497
:1040D0000192D6B99CBB002D05F106034BDBA31B57
:1040E0000A3505EB8305013E0134A642F1D2DDF825
:1040F00004B0B9F80030C9F800305A46414650467D
:1041000003B0BDE8F04FFFF73FBFB7B2A3B2AAEBD1
:1041100007007F0008EB03011FFA80FBBFB23A469D
:1041200089B258460093FFF7E1FE009BA8EB03011C
:104130003A4689B25846FFF7D9FE002CCBD0A7B239
:10414000B3B2AAEB07007F00A8EB03011FFA80FBC4
:10415000BFB23A4689B258460093FFF7C7FE009BAC
:1041600003EB08013A4689B25846FFF7BFFE002D1F
:1041700005F10603B3DA03EB8405B5E788D2012025
:104180009FED2B7B70B52C4D2C4BAB6085ED007BF0
:104190000446FCF7EFFA2A482A4E0122202101F0BA
:1041A000E5F800224FF40061274801F0DFF8052010
:1041B00000F0FEFC01224FF40061234801F0D6F824
:1041C0000A2000F0F5FC00224FF400611E4801F0C7
:1041D000CDF8142000F0ECFC01224FF400611A48E5
:1041E00001F0C4F80A2000F0E3FC736898478528C2
:1041F00010D0164C636898474FF6FF73984201D071
:10420000012070BD124A236814609847114BAB60BF
:10421000002070BD0E4A3368166098470CB1022C1E
:10422000F4D12046FEF716FDF0E700BFAFF30080A3
:1042300000000000FFFF000088D20120880000205D
:104240000014024040000020000C02400400002046
:1042500080D20120780000200220FFF791BF00BF2C
:1042600030B595B09FED127B052400220346012155
:1042700006944FF080701024CDE90E20CDE9122273
:10428000CDE902410D920B921192009201914FF4EF
:1042900080756A4606A908480C958DED047B02F0EE
:1042A0009DFE003818BF012015B030BDAFF300806F
:1042B000000000000000400094D201200000000037
:1042C00010B594B04FF48071062200230C91069231
:1042D00019480D9341F2883206A9CDE90E33CDE994
:1042E00012330B93119302F019FE10B1012014B098
:1042F00010BD9FED0F7B0223CDE900330124102276
:10430000052303940292069306A94FF0807441F2AC
:1043100088336A4608480F948DED047B02F05EFEF8
:10432000003818BF012014B010BD00BFAFF30080EB
:10433000000000000000400094D20120F0B58BB0D6
:10434000384B394D3948002400949A6B42F00202F0
:104350009A639A6B02F002020092009A9A6942F004
:1043600002029A619A6922F002029A6101941A6B20
:1043700042F040021A631A6B02F040020192019A65
:1043800002941A6B42F002021A631A6B02F00202E4
:104390000292029A03941A6B42F020021A631B6B7A
:1043A00003F02003039340220223CDE904230A27CC
:1043B0000122039B089704A90323CDE906230926BC
:1043C00000F0A2FE04A90423194804930694089659
:1043D00000F09AFE04A928464FF4807304930897CE
:1043E00000F092FE04A928464FF400730493089746
:1043F00000F08AFE802304A928460493089600F062
:1044000083FE402304A928460493089600F07CFE0E
:1044100022460F215C2000F0EFFB5C2000F02AFC1C
:104420000BB0F0BD003802400014024000180240FA
:104430000004024070B5494C494B236090B02046BF
:1044400002F058FD054610B1012010B070BD0146C4
:104450002046FFF773FF04221023A260E36065602B
:104460004FF0807696FAA6F3B3FA83F3013B4FF44C
:104470008062204623616261A561E561256202F0E8
:10448000D7FC0028E0D1CDE90A00CDE90E004FF4B9
:1044900080756623099007900D9041F2883202A939
:1044A00020460895029302F039FD10B1042010B0A7
:1044B00070BD992341F2883202A92046029302F08E
:1044C0002DFD0028F2D141F28830FFF7C9FE002807
:1044D000ECD18523CDE90A06CDE90E0002930990BF
:1044E000012307900D9041F2883202A920460895D9
:1044F0000C9302F013FD0028D8D141F288320DF15F
:104500000701204602F0AEFE0028CFD1FFF7D8FE0B
:104510000028CBD181230293F02292FAA2F29DF8D7
:1045200007300A20B2FA82F200FA02F203F00F0317
:10453000134302A941F2883220468DF8073002F079
:10454000EDFC0028B2D141F288320DF1070120467E
:1045500002F008FE00283FF478AFA7E794D20120CC
:10456000001000A070B5114C114E2368307815462C
:104570009847636870209847CD2801D0032070BD0C
:104580008DB1022D0CBF08210C210A4A0A4DA368E7
:104590001170702030702C6098472B683078DB6881
:1045A0009847002070BD0621EFE700BF940000206F
:1045B000F0D2012090000020F4D201202DE9F04F2C
:1045C000DFF8D4B0314ADBF8003005461B691078BB
:1045D00083B09847287000284FD06946DFF8BC8028
:1045E0002B4F01AEAA464FF000090C46DBF8003015
:1045F000264A5B691078214632469847254B1A783F
:1046000010073ED420883388910703D5C0F1EF000E
:1046100080B22080520703D5C3F1EF039BB23380F1
:10462000D8F800C0396860458CBFA0EB0C02ACEB39
:1046300000028B428CBFA3EB010EA1EB030E92B2E2
:104640001FFA8EFE7244052AD2BF1FFA8CF0C8F8FA
:1046500000003B602AF8020FD8BF8BB2AAF80430E2
:104660002B7809F101094B4504F1020406F1020619
:1046700008F1040807F10407B8D8002003B0BDE82A
:10468000F08F2388308820803380BDE7F0D201206E
:10469000E0D2012090000020F4D20120E8D20120D5
:1046A00000B589B0104B1148002201921A6B42F0FC
:1046B00040021A631B6B9FED0A7B03F040030193DA
:1046C0000122022302A9CDE904238DED027B019B87
:1046D00000F01AFD09B05DF804FB00BFAFF30080E5
:1046E00020000000000021100038024000180240A5
:1046F00008B5FFF7D5FF0F210022172000F07CFA44
:10470000172000F0B7FA044B044A1B6810789B6925
:104710009847002008BD00BFF4D20120F0D201204C
:10472000704700BF0020704710B50446FFF710FA2D
:10473000A821E0B2FFF76AFA10BD00BF10B582B041
:1047400000240221C0B28DF80740FFF75FFA8DF810
:1047500007009DF8073003F00F038DF807309DF830
:104760000730022B88BF8DF807409DF80710044BD7
:104770009DF80700597000229A7002B010BD00BF6A
:10478000F8D2012070B5164C1546A37862789A428B
:1047900082B00E461FD903B3012B0CBF09210021A3
:1047A00004230DEB0302C0B2FFF76EFA9DF804304C
:1047B0009DF805209DF807101B0203F470631A434F
:1047C0009DF8063032801B02A27803F4706319430F
:1047D000531C2980A37002B070BD0321E0E700BF25
:1047E000F8D201200122A421C0B2FFF7D5B900BF41
:1047F0000022A421C0B2FFF7CFB900BF064A137848
:10480000834204D05178884201D013B101B170477E
:104810000123D054FFF79CB9FCD20120704700BFA0
:104820000022A421C0B2FFF7B7B900BF10B4174AE5
:10483000116885B04FF0E023490400910099D3F846
:10484000244D2143C3F8241D116889040191019965
:10485000D3F8244D2143C3F8241D12680C491201DA
:104860000292029AD3F8144D2243C3F8142D0A6819
:104870006FEAC2020392039AD3F8141D0A40C3F8E8
:10488000142D05B05DF8044B704700BFC000002038
:10489000BC000020012882B00BD00B4B1B684FF0EE
:1048A000E022DB430093009B11690B40136102B0CF
:1048B0007047064B4FF0E0221B680193019B116982
:1048C0000B43136102B07047BC000020C000002001
:1048D0002DE9F041C46887680546164600202B691B
:1048E000A7EB040C9C4203F1FF3328BFDB19B4454E
:1048F00028BFB4461B1B9C4528BF9C4660446B6880
:10490000A6EB0C0604EB0C08BCF1000F09D0013C2F
:1049100023448C4411F801EB03F801EF8C45F9D1E5
:10492000AF68B84514BF44460024EC60002ED6D1D1
:10493000BDE8F08170B4C5688668731B93420ED9D8
:104940004368AE1842B1013D2B440A4411F8014BB3
:1049500003F8014F9142F9D1C66070BC70474468BA
:10496000C3B105F1FF3C0B44A44411F8014B0CF812
:10497000014F9942F9D144682A44961BECD0621E3B
:104980009C1913F8011B02F8011FA342F9D1C6605C
:1049900070BC70470B46EFE710B5154A154C16482A
:1049A0001649C4E906204FF48060206214489FED48
:1049B0000E7BC4E91820102000230422A066E01D0D
:1049C000A3626362E3622367E366636784ED047B4B
:1049D00013F0B6FF0B4B93E803002022A271206076
:1049E000A18010BDAFF300800300000003000000B1
:1049F000D8C9010810D7012010D30120E4C901084B
:104A000000D30120E8C9010838B5204B00EB400471
:104A100003EBC40E0130DEF82C4000EB4000012C0B
:104A20008C46154603EBC00005D0022C2AD0B4B149
:104A30000024204638BDDEF82830DEF82440A342AA
:104A40009CBFDEF820105B18013B1C1B944228BF62
:104A5000144622466146FFF76DFF204638BDDEF85A
:104A60002830DEF8242093429CBFDEF820105B182B
:104A7000013B9A1A9542DCD82A466146FFF75AFF55
:104A80002C46D6E7BDE83840FFF722BF10D70120FB
:104A9000F8B5054608460C4613F060FF0A4B1B7834
:104AA00006466BB1EFF311874FF0200181F31188B7
:104AB000324621462846FFF7A7FF87F31188F8BD45
:104AC000FFF76AFFEEE700BF10D701202DE9F041A4
:104AD000194D1E462B7804468846174633B32B697A
:104AE000A34226D9EFF3118C4FF0200181F31188F6
:104AF00054B92246131905EBC305069BEB628CF3F0
:104B000011880020BDE8F081601C00EB4000C0006F
:104B100004EB440305EBC30345F80080284400215F
:104B2000476062001E6299625962E3E7FFF734FF53
:104B3000D5E74FF0FF30E5E710D70120FFF72CBF96
:104B4000FEE700BF38B50E4A0E4B12781B680546CB
:104B50004FF47A70B0FBF2F0B3FBF0F000F0A6F87F
:104B6000044608B90F2D01D9012038BD0246294657
:104B70004FF0FF3000F040F8034B20461D6038BD79
:104B8000C4000020CC000020C8000020034A044BD1
:104B900011681B780B441360704700BFB8D7012021
:104BA000C4000020014B1868704700BFB8D701202F
:104BB00038B50446FFF7F6FF631C054602D0044BE8
:104BC0001B781C44FFF7EEFF401BA042FAD338BD10
:104BD000C40000200749CA6803024FF6FF0003F42F
:104BE000E0630240134343F0BF6343F40033CB6000
:104BF000704700BF00ED00E01C4BDB68C3F30223ED
:104C000000B5C3F1070EBEF1040F03F1040C28BF79
:104C10004FF0040EBCF1060F1BD9033B4FF0FF3CD5
:104C20000CFA03FC22EA0C024FF0FF3C0CFA0EFCDB
:104C300021EA0C019940002841EA02010CDB00F155
:104C40006040090100F56140C9B280F800135DF8C9
:104C500004FB00221346E7E7054B00F00F000901B3
:104C60000344C9B219765DF804FB00BF00ED00E013
:104C7000FCEC00E0002807DD4109044A00F01F00B9
:104C80000123834042F82130704700BF00E100E07B
:104C9000002808DD4309044900F01F0001222033E9
:104CA000824041F82320704700E100E00138B0F174
:104CB000807F10B403D301205DF8044B70474FF0A0
:104CC000E023074C58614FF0F00C84F823C0002219
:104CD000072110469A615DF8044B1961704700BFC7
:104CE00000ED00E04FF0E022042813690CBF43F010
:104CF000040323F004031361704700BF38B5044672
:104D0000FFF750FF0546002C74D02368022284F878
:104D100035201A68002122F0010284F834101A604C
:104D200005E0FFF73FFF431B052B39D823681A68BE
:104D3000D107F6D4A0686268E168256902430A4396
:104D40006169A0692A430A43E1691D6802430A4375
:104D500032492940256A2A430A43616A042926D038
:104D60001A605A6922F007021143D8B22C4A5961DD
:104D70001038A2FB005212092A4923F47F73895C80
:104D8000E16523F003035F2888BF04333F228A4094
:104D9000A36500209A600123606584F8353038BD32
:104DA000032320226265184684F8353038BDE56A51
:104DB000216B2943114319605969A26A21F0070147
:104DC000114341F00401002DCFD028B9012A21D090
:104DD00032F00202C9D106E0B0F5005F0CD0022A21
:104DE00003D9032AC1D1EA01BFD54022012362655C
:104DF00084F83530012038BD032AB6D801A050F818
:104E000022F000BFEB4D0008E74D0008EB4D000815
:104E1000154E0008B5F1C07FA7D1E6E73F8010F03E
:104E2000ABAAAAAAF0C9010870B490F83440856D05
:104E3000012C0AD090F835404FF0010C644580F801
:104E400034C005D0002380F83430022070BC704795
:104E5000022680F83560046800264665266826F438
:104E60008026266063608368402B0EBFA260A1602D
:104E7000E260C26D08BFE1603F239340AB602368EE
:104E8000026C43F0160323601AB1236843F0080351
:104E90002360236843F001030020236070BC704747
:104EA00070B50446866DFFF77DFE94F83530022B11
:104EB000054606D080220023626584F83430012044
:104EC00070BD23681A6822F016021A605A6922F02F
:104ED00080025A61226C32B31A6822F008021A600A
:104EE0001A6822F001021A6005E0FFF75BFE431B1F
:104EF000052B0FD823681B6813F00103F5D1E16D72
:104F00003F228A400121B260184684F8343084F888
:104F1000351070BD032020220023626584F83430F0
:104F200084F8350070BDA26C002AD5D1D8E700BF47
:104F300090F83530022B03D0802343650120704761
:104F40000268052380F83530136823F00103002040
:104F500013607047F0B583B0674A876D1668002309
:104F60000193C36D3D6808229A402A42044603D04B
:104F700001680868400778D401229A402A4203D089
:104F80002168496908066AD404229A402A4203D05B
:104F90002168096889075CD410229A402A4203D00C
:104FA00021680868000741D420229A402A4214D080
:104FB00021680868C00610D5BA6094F83520052A23
:104FC00063D00B6813F4802F0B687ED0190340F177
:104FD0008980E36B0BB120469847636D23B3636D03
:104FE000DA071AD522684549052384F83530136855
:104FF000A1FB061623F00103B60A136002E0136852
:10500000DB0704D5019B0133B3420193F7D900229A
:10501000012384F8342084F83530E36C23B1204632
:1050200003B0BDE8F040184703B0F0BDBA600A68AD
:1050300012F4802F0A6822D1D20503D40A6822F024
:1050400008020A60226C002AAED020469047E36D29
:10505000AAE7BA60626D42F0040262659CE7BA603A
:10506000626D42F0020262658EE7086820F004007B
:105070000860BA60626D42F0010262657CE711036C
:10508000E0D5A26C002AE0D18EE70A6822F0160271
:105090000A604A6922F080024A61226C3AB30A68C7
:1050A00022F008020A603F2202FA03F3216DBB607E
:1050B0000022012384F8342084F835300029B3D04D
:1050C000204603B0BDE8F040084713F4807380D158
:1050D0000A6822F010020A60012284F8343084F851
:1050E000352076E7636C002B7FF475AF75E7A26C13
:1050F000002AD4D1D7E700BFCC000020B5814E1BD9
:1051000090F83500704700BF2DE9F04F85B00022C0
:105110000D688B4F019113464FF0010805E00133F4
:10512000102B02F1020200F09B8008FA03F636EA27
:10513000050406EA050CF2D101994C6824F0100E22
:105140000EF1FF39B9F1010F40F28D808E68D0F871
:105150000CE0032101FA02F996402EEA090E46EA14
:105160000E06C6606FEA0906D0F800E00EEA060EE9
:1051700004F00306964046EA0E060660E600CED529
:10518000704E002103913146766C46F480464E64A1
:105190004E6C06F480460396039E23F0030606F148
:1051A000804603F003090F2106F59C364FEA890972
:1051B00001FA09FA6449D6F808E088422EEA0A0E94
:1051C00023D001F58061884200F097805F498842D2
:1051D00000F09A80DFF878A1504500F09C80DFF85D
:1051E00074A1504500F09E80DFF86CA1504500F09E
:1051F000A080DFF868A150450CBF4FF0060A4FF0C1
:10520000070A0AFA09F94EEA090EC6F808E03E68EC
:105210006FEA0C0EE10354BF0EEA06064CEA0606DE
:105220003E607E68A10354BF0EEA06064CEA0606FD
:105230007E60BE68E10254BF0EEA06064CEA06062E
:10524000BE60FE68A10203F1010354BF0EEA060628
:105250004CEA0606102BFE6002F102027FF465AFF5
:1052600005B0BDE8F08F0199D0F808B0C96801FA1F
:1052700002FA032101FA02F92BEA090B4AEA0B0AA6
:10528000C0F808A0D0F804A001992AEA060A260965
:105290009E4046EA0A064660C668896826EA090A08
:1052A0006FEA090601FA02F949EA0A09BEF1020F9A
:1052B000C0F80C907FF458AF01994FEAD30E0969FA
:1052C00000EB8E0E03F0070C4FEA8C0CDEF82090FA
:1052D00001FA0CFA0F2101FA0CFC29EA0C094AEA3E
:1052E0000909CEF82090D0F800C004F003049440DF
:1052F00006EA0C063443046011E74FF0010A0AFA8B
:1053000009F94EEA090E80E74FF0020A0AFA09F994
:105310004EEA090E79E74FF0030A0AFA09F94EEA54
:10532000090E72E74FF0040A0AFA09F94EEA090E6B
:105330006BE74FF0050A0AFA09F94EEA090E64E72D
:10534000003C0140003802400000024000080240DA
:10535000000C0240001002400014024000180240FD
:105360000369194214BF01200020704702B90904E3
:1053700081617047436931EA030308BF0904816111
:10538000704700BF704700BF044A5169014208B529
:1053900000D108BD5061FFF7F5FF08BD003C01409A
:1053A0002DE9F8430D46814617461E464FEA11483F
:1053B000D9F8002001E0731C13D1B8F1010F0BBF25
:1053C0005369946925EA030C25EA040C1FFA8CFC46
:1053D000BCFA8CFC4FEA5C1CBC45ECD00020BDE85C
:1053E000F883FFF7DFFB089BC01AB04201D8002EFC
:1053F000DED100222023C9F8302089F83D3089F819
:105400003E20D9F8403089F83C2043F02003C9F809
:1054100040300120E3E700BF2DE9F84381460E4606
:1054200017469846D9F8004004E065696A0509D432
:105430007B1C21D1606926EA000080B20028F4D1EB
:10544000BDE8F883236843F400732360002220231F
:105450006FF480616161C9F8302089F83D3089F8C6
:105460003E20D9F8403043F00403C9F8403000230F
:1054700089F83C300120E3E7FFF794FBA0EB08003C
:10548000B84201D8002FCDD100232022C9F83030F6
:1054900089F83D2089F83E30D9F840301343C9F8E7
:1054A0004030E4E7F8B506460D463468636913F00A
:1054B000400317461DD16269D2061CD4FFF772FB68
:1054C000C01BA8420ED900232022336386F83D205A
:1054D00086F83E30336C13433364002386F83C3047
:1054E0000120F8BD002DEED03468636913F040034D
:1054F000E1D00020F8BD6FF010012022616133631C
:1055000086F83D2086F83E30336C3364002386F8FD
:105510003C300120E5E700BFF8B505460E461746CA
:105520002C6801E0731C1AD1636913F0800314D155
:1055300060694205F6D56FF48061202261612B63BA
:1055400085F83D2085F83E302B6C43F004032B6436
:10555000002385F83C300120F8BD0020F8BDFFF79E
:1055600021FBC01BB04201D8002ED9D1002320223C
:105570002B6385F83D2085F83E302B6C13432B645C
:10558000E6E700BFF8B505460E4617462C6801E071
:10559000731C1AD1636913F0040314D160694205C6
:1055A000F6D56FF48061202261612B6385F83D2080
:1055B00085F83E302B6C43F004032B64002385F800
:1055C0003C300120F8BD0020F8BDFFF7EBFAC01B0E
:1055D000B04201D8002ED9D1002320222B6385F8B8
:1055E0003D2085F83E302B6C13432B64E6E700BF6B
:1055F0002DE9F0479946036882B090461A680A9DE3
:105600000B9F42F4807206468A461A605C69E10785
:105610000ED50AF0FE021A612F493B462A46304653
:10562000FFF7FAFE38B30124204602B0BDE8F08748
:105630006A1CEBD0FFF7B6FAC01B854202D30DB14E
:105640003368E3E700232022336386F83D2086F8A1
:105650003E30326C316842F0200232640A6886F8CB
:105660003C30D00502D54FF4007333640324204648
:1056700002B0BDE8F08733680190596901919B69D8
:1056800001933A4629463046019BFFF745FF044601
:10569000C8B9B9F1010F07D133685FFA88F2204623
:1056A0001A6102B0BDE8F08733684FEA182018612C
:1056B0003A4629463046FFF72FFF20B932685FFA95
:1056C00088F31361B0E7336C042BACD132681368F4
:1056D00043F400731360A6E7020001002DE9F047D0
:1056E0009946036890461A6842F480621A601A6804
:1056F00084B042F480720C9D0D9F1A6006468A4663
:105700005C69E1070FD50AF0FE021A6140493B4689
:105710002A463046FFF780FE5FFA8AFA18B3012066
:1057200004B0BDE8F0876A1CEAD0FFF73BFAC01B63
:10573000854202D30DB13368E2E7002320223363B0
:1057400086F83D2086F83E30326C316842F0200207
:1057500032640A6886F83C30D00502D54FF40073F5
:1057600033640320DCE733680390596903919B6934
:1057700003933A4629463046039BFFF7CDFE40BBD4
:10578000B9F1010F2ED133685FFA88F21A613A46F7
:1057900029463046FFF7C0FED8B902463068016896
:1057A00041F4807101602B4600974FF001113046A3
:1057B000FFF7F6FD30BB326815494AF0010313616B
:1057C00030463B462A46FFF727FE003818BF012027
:1057D000A6E7336C042BA2D13268136843F400733C
:1057E00013609CE733684FEA18221A6129463A464B
:1057F0003046FFF791FE0028EBD132685FFA88F35C
:105800001361C4E733681B68DB05AAD5A6E700BFB0
:1058100002000100704700BF70B50446002800F088
:105820009D8090F83D3003F0FF02002B00F098803F
:105830002368242284F83D201A6822F001021A60AD
:105840001A6842F400421A601A6822F400421A6090
:1058500001F0BAFE65684E4B9D424FD84D4B9842C1
:105860007CD922684C4B5168A3FB003C21F03F01DE
:1058700041EA9C415160116A4FEA9C4E0EF1010EC3
:1058800021F03F0141EA0E011162D169431E6D0012
:1058900040F6FC70B3FBF5F3013321F44F410342B2
:1058A00021F0FF0161D104230B43D3611168206A09
:1058B000E36921F0C00103430B4313609168E06882
:1058C000236921F40341034321F0FF010B4393605B
:1058D000D168A069636921F0FF0103430B43D360E2
:1058E0001168002341F0010120201160236484F835
:1058F0003D002363184684F83E3070BD274B984224
:105900002CD92268244B5168254EA3FB003C21F082
:105910003F0141EA9C4151604FEA9C434FF496712C
:1059200001FB03F3A6FB0363116A9B0921F03F010E
:1059300001330B431362D169A36821F44F4121F075
:10594000FF01ABB9431E05EB4505B3FBF5F301338E
:10595000C3F30B03D3B143F40043A5E7012070BDAB
:1059600080F83C20FFF756FF62E7C3F30B039BE789
:1059700005EB8505431E05EB8505B3FBF5F3013308
:10598000C3F30B0313B143F440438DE701238BE7CB
:10599000A08601007F841E0083DE1B43FF083D00BC
:1059A000D34D6210704700BF10B50446A0B1026825
:1059B000242380F83D30136823F001031360FFF7C0
:1059C000F1FF0023236484F83C3084F83D3018460E
:1059D000236384F83E3010BD012010BD2DE9F04F47
:1059E000044683B09946BDF834A00E9E0F469046FB
:1059F000FFF7D8F894F83D30202B054608D0022058
:105A000003B0BDE8F08FFFF7CDF8401B19286FD821
:105A1000206883696FEA030C1CF0020BF3D094F842
:105A20003C30012BEBD003680122DB0784F83C20DB
:105A30006CD53946076827F4006707600C986062E8
:105A400021200195009684F83D00402084F83E0016
:105A500000202064A4F82AA0608D20853248E062EE
:105A60004B4642462046FFF7C3FD00285AD1238DFE
:105A70005BB32A4631462046FFF74EFD002849D148
:105A8000676A2068B4F828C039460CF1FF3211F873
:105A9000013B0361638D013B9BB26385D0F814E049
:105AA000616293B21EF0040F2385E1D06BB17A7866
:105AB0000261628DACF1020C013A1FFA8CF30237DD
:105AC00092B2676223856285D2E72A463146204634
:105AD000FFF758FDF0B922681368202143F40073E2
:105AE000136084F83D1084F83C0084F83E0087E79A
:105AF0002023C4F830B084F83D3084F83EB0236CE5
:105B000084F83CB043F02003236478E70368134330
:105B100003608EE7236C042B04D12268136843F4DE
:105B20000073136001206BE70000FFFF2DE9F04FC9
:105B3000044687B09946BDF844A0129E0F46904691
:105B4000FFF730F894F83D30202B05460AD04FF08F
:105B50000208404607B0BDE8F08FFFF723F8401B6E
:105B600019284AD8206883696FEA030C1CF0020BDD
:105B7000F3D094F83C30012BE9D003680122D90717
:105B800084F83C2047D53946076827F4006707604A
:105B90001098606222200195009684F83D00402014
:105BA00084F83E0000202064A4F82AA0608D20859F
:105BB0008448E06242464B462046FFF78FFD804610
:105BC000A8B9238D5BBB236802905A6902929A6937
:105BD0000292029A1A6842F400721A60002320228C
:105BE00084F83D2084F83C3084F83E30B1E74FF033
:105BF0000108404607B0BDE8F08F2023C4F830B05C
:105C000084F83D3084F83EB0236C84F83CB043F017
:105C1000200323649BE7036813430360B3E7012B6E
:105C200000F0BF80022B00F084802268059051694B
:105C3000059192690592059A634F032B4DD8012B6C
:105C400000F0A280022B009533464FF00002394647
:105C500020467ED0FFF7A4FB02460028C7D1236868
:105C6000196821F4806119601969636A1970616AA1
:105C7000638D01316162013B218D9BB263854B1EB7
:105C800023853946009533462046FFF789FB0028D7
:105C9000ADD12368616A1A6842F400721A601B6908
:105CA0000B70638D626A2168013B9BB26385531C54
:105CB00009696362238D013B23855170238D628DB9
:105CC000616A013B013A01319BB292B26162238564
:105CD0006285002B82D0032BB1D92A46314620465B
:105CE000FFF7E0FB002882D12268636A12691A700C
:105CF000628D2068238D616A013A92B262854269A1
:105D0000013B9BB201F1010C52072385C4F824C06A
:105D1000DFD503694B70628D238D013A92B26285A3
:105D2000626A013B9BB2013223856262002BD2D1B1
:105D300054E72268116821F480611160116841F410
:105D40000061116004905169049192690492049A6F
:105D500072E7FFF725FB00287FF449AF2368616AEB
:105D60001A6842F400721A601B690B70638D626AD4
:105D7000013B9BB26385238D013B23852368511C26
:105D80001B6961625370C6E72A4631462046FFF719
:105D900089FB00287FF42BAF23681A69636A1A70A5
:105DA000B9E72268116821F480611160039051699C
:105DB0000391916903910399116841F40071116095
:105DC0003AE700BF0000FFFF04000100704700BF7A
:105DD000704700BF704700BF704700BF704700BFEB
:105DE000704700BF704700BF90F83D20016D10B5AF
:105DF0000346D2B259B9C26C0168012A826C29D01B
:105E0000C2F307220A61026D0132026510BD016D05
:105E1000012925D0016D0229F8D1222A2CD0418DEB
:105E200089B229BB418D89B20029EFD1212AEDD158
:105E30000268546824F4E0645460146844F4007404
:105E400014602022016380F83D2080F83E10FFF7A7
:105E5000C9FF10BDD2B20A61026D0232026510BDE7
:105E6000826C0168D2B20A61026D0132026510BD16
:105E7000212A07D05B8D10BD0268136843F480733C
:105E8000136010BD416A026811F8010B10615A8D50
:105E90005962013A92B25A8510BD00BF704700BFE7
:105EA000704700BF704700BF70B53A4B3A4A1B6855
:105EB000806B82B0DB080021A2FB032301911B0A47
:105EC00090F83D10026803EB8303C3EBC303C9B230
:105ED000019305E0019B013B019313689B0506D5E7
:105EE000019B002BF6D1036C43F020030364446B49
:105EF0004CB3836B0025E563F3B11668DD6326F4CC
:105F0000806616604585256500241C65136823F0AE
:105F10000103136090F83D30602B2AD001F0280176
:105F2000282919D02022002380F83D2080F83E3017
:105F3000FFF7B6FF02B070BD156825F480651560E7
:105F400043852365E2E7836BF3B11568DC6325F4D1
:105F5000806515604485D7E7136843F0010313603B
:105F60001368002443F480631360046380F83D10D9
:105F7000DEE70023202280F83D2080F83E300364D5
:105F8000FFF790FF02B070BD146824F480641460C1
:105F90004385BBE7CC00002089B5F81490F83D207C
:105FA00090F83E30102B10B5D2B20446D9B238D09A
:105FB000402936D002F0280128293DD023685968AD
:105FC000080507D4602A05D02021002284F83D105E
:105FD00084F83E20002222635A6812F4006234D111
:105FE00094F83D10602975D05A69500605D5626A4B
:105FF0001B691370636A013363622046FFF750FF29
:10600000236C190704D02268536823F4E0635360BB
:1060100094F83D30226C5207DBB201D5282B2FD0EB
:1060200010BD222AC6D123681A6822F400621A60C1
:106030005A681205C8D5CDE700232363236884F886
:106040003D105A6812F40062CAD05A68606B22F49C
:1060500000625A6090F83530012B1ED0284B036542
:10606000FEF766FF0028CBD02268606B1368202102
:1060700023F001031360036D84F83D109847BFE7D8
:1060800000232049E16220222363204684F83D203A
:1060900084F83E30FFF7A4FE10BDA06B184B0365DB
:1060A000FEF746FF0028ABD023685A69510606D593
:1060B000626A1B691370626A2368013262621A683D
:1060C000A06B22F0010220211A60036D84F83D10BC
:1060D000984795E7202184F83D1022645A695206BA
:1060E00006D5626A1B691370626A236801326262B4
:1060F0001A6822F0010220461A60FFF7D3FE7FE7FC
:10610000A95E00080000FFFF70B5036804465868E8
:10611000E56A94F83E1094F83D2010298CB0D2B274
:106120005FFA81FC21D0BCF1400F1ED0216C002908
:1061300000F093805969002511F0020FC1F3400669
:1061400056D0860556D5226C02B19D6994F83D2043
:1061500002F02802282A00F029826FF002010022B2
:10616000596184F83C200CB070BD99695A69D60712
:106170001AD4B5F52A0FF6D0B5F12A4FF3D0160789
:106180006ED5850540F18480626C616BD2B21A6174
:10619000002900F0FA81CA6B002A00F0FB815A68DE
:1061A00042F400625A60DEE785056FD5E26AB2F517
:1061B0002A0F00F0F881E26AB2F12A4F04BF0822E8
:1061C000E26294F83E20402A00F0E6812269B2F5AE
:1061D000804F00F0C081226D002A40F0FB81626C8C
:1061E000C2F3C81202F0060242F0F0021A61BAE7E6
:1061F000CD067CD402F0F702212A00F0D4804E06AE
:1062000040F11181450540F10E81490700F10E81F1
:1062100094F83D10628D92B2C9B2002AA3D0626A8E
:106220001B691370638D626A013B9BB26385638D4A
:1062300001329BB26262002B95D12A2993D1226848
:1062400053682225282123F4806353602046256368
:1062500084F83D10FFF7C0FD85E79D6959696BE73C
:10626000960715D5850513D594F83E20E06A256B71
:1062700094F83D102229D2B200F0BF810022099289
:106280005A6909929B690993099B6CE71507E7D541
:1062900011F0040F596800F0D28009053FF563AF93
:1062A000160640F1F280450540F1EF80510700F1FC
:1062B000EF8094F83D20208D94F83E10E56AD2B22C
:1062C000C9B2002840F04882212A00F03A834029D0
:1062D0007FF449AF222A7FF446AF628D92B2002A42
:1062E00040F098835A6822F480625A603BE7850543
:1062F00080D594F83D505A6822F4E0625A600B96BB
:106300005A690B921A6842F001021A600B9A1A68D5
:1063100022F480621A605A681105EDB200F1EA8039
:10632000638D9BB213B323685A6952070AD5626A18
:106330001B691370628D636A013A591C92B223681B
:10634000616262855A69560609D5626A1B691370D3
:10635000638D626A013B01329BB262626385638D29
:106360009BB21BB1236C43F004032364236C002B0A
:1063700040F0EB802A2D00F08B8194F83D30282BE3
:1063800000F07981236B222B02D0222D7FF4EBAE1B
:10639000002320222363204684F83D2084F83E30E9
:1063A000FFF71AFDDFE60D0628D5460526D54D0771
:1063B00027D494F83D00618D89B2C0B200293FF422
:1063C000D2AE616A11F8015B1D616162618D0139B4
:1063D00089B26185618D89B200297FF4C4AE292814
:1063E0007FF4C1AE5968282521F4806159602046A8
:1063F000226384F83D50FFF7EDFCB4E649077FF5D2
:10640000B2AE82057FF5AFAE628D92B2002A3FF444
:10641000AAAE626A12F8011B1961638D6262013BC8
:106420009BB263859FE64A077FF59DAE86057FF5A3
:106430009AAE628D92B2002A3FF495AE1AE00D0535
:106440003FF591AE510630D451077FF58CAE8205F1
:106450007FF589AEE16A628D92B2042A00F06D8107
:10646000628D92B2032A00F08981628D92B2022A73
:1064700000F0B981626A1B691370638D626A013B27
:1064800001329BB2626263856DE652077FF56BAEA7
:1064900086057FF568AEBCF1100F00F02A8120461A
:1064A0000CB0BDE87040FFF79FBC4605CCD5550742
:1064B000C2F38001CBD494F83D20222A7FF453AE5E
:1064C000628D92B2032A40F20482626A1B691370E1
:1064D000638D626A013B9BB26385638D9BB201321F
:1064E000032B62627FF43FAE2268536823F480631B
:1064F000536038E605F0F702222A00F09B80606BBB
:106500000268526892B26285628D92B21AB1226CB0
:1065100042F0040222645A6822F400625A60FEF7D4
:10652000EFFD012808D0606B9C4B0365FEF700FD72
:1065300010B1606B036D9847638D9BB2002B7FF4A5
:10654000F2AE236C002B3FF418AF20460CB0BDE830
:106550007040FFF723BD94F83D20212A626C16BFDE
:1065600042F0010202F0FE02D2B21A61626B1AB16D
:10657000D26B002A7FF413AEA26B002A3FF4F3AD76
:10658000D26B002A7FF40BAEEDE5A26B002A7FF4FC
:1065900002AEE8E5A26BF3E7226D42BB626C02F04B
:1065A000FE021A61DFE50122E2620AE65A6822F47D
:1065B00080625A602E066FEA95014FF0000354BFC7
:1065C000A289228B84F83C3001F001012046FFF7BC
:1065D00005FCC8E5226D012A7FF4C5AD626CC2F3EB
:1065E000C81202F0060242F0F1021A61BBE5626CC9
:1065F00042F00102D2B21A61B5E5216D11B9402A0B
:1066000000F0A380226D22B92169B1F5404F00F05E
:10661000A780628D92B2002A4AD102925A690292F0
:106620009A690292029A1A6842F400721A60002370
:10663000236598E5A06B0268526892B26285628D0C
:1066400092B21AB1226C42F0040222645A6822F417
:1066500000625A60FEF754FD01283FF461AEA06B62
:106660004E4B0365FEF764FC00283FF459AEA06B67
:10667000036D984754E600234949E16220222363D1
:10668000204684F83D2084F83E30FFF7A9FB6AE5F8
:1066900028222363204684F83D20FFF79DFB94F8D1
:1066A0003D30282BE7D0236B222B7FF45CAD6FE6C7
:1066B000628D92B2012A75D0628D92B2022A00F0E8
:1066C000E7801A6842F480621A605A68150508D596
:1066D000202800F2D880072800F2CA80012800F0A4
:1066E000CD80002208925A6908929B690893089B02
:1066F0009DE7E16A94F83D20212A7FF434AD628D54
:1067000092B2002A7FF485AE082900F05B8120292F
:1067100000F0588111F5803F00F05481596821F450
:10672000E061596011202023206384F83E20204638
:1067300084F83D30FFF74AFB15E55A68616A22F498
:1067400080625A601B690B7097E600915A6900924B
:106750009B690093009B06E5212A7FF4B8ADBCE558
:1067600001925A6901929A690192019A1A6842F457
:1067700080721A60236D01332365F4E45A6804299A
:1067800022F480625A603FF475AE02293FF472AE83
:106790001A6822F480621A606CE600BFA95E0008E5
:1067A0000000FFFF10F5803F00F02081082800F076
:1067B000E080202800F0DD80122D00F06681102896
:1067C00000F266819F4A0241D60700F161811A6892
:1067D00042F480621A60002205925A6905929B6910
:1067E0000593059B23E701390F2909D8DFE801F05C
:1067F0003B36083608080808080808080808083B57
:106800001A6842F400721A60626A1B691370638D21
:10681000626A2168013B9BB263850B69511C61620E
:106820005370638D2168626A013B9BB263854B683C
:10683000013223F44073202062624B6084F83D00F3
:1068400094F83E30402B00F00C810022122384F893
:106850003E2020462363FFF7BBFA84E41A6842F423
:1068600080621A60D0E71A6822F480621A60CBE76F
:10687000754A0838C240D0077FF533AF5A6842F4F2
:1068800080525A602DE710F5803F7FF42AAFF5E77C
:10689000102804D86D4AC240D50700F1C1801A689B
:1068A00022F480621A601A6842F400621A605A6820
:1068B000110506D5202840F2BB8010F5803F00F07E
:1068C000BC80002207925A6907929B690793079B35
:1068D000ADE6E06A02283FF446AC012A3FF643AC3D
:1068E0005B4A0A91126846F2A810B2FBF0F202EB82
:1068F00082020A9204E01A6812F4007200F0CD805D
:106900000A9A013A0A920A990029F4D1226C606A23
:1069100042F0200222645A6822F4E0625A601B6945
:106920000370638D626A013B01329BB22020638554
:10693000626284F83D00204684F83E10FFF7B0FA0A
:1069400011E4082D25D0202D23D015F5803F20D02F
:106950005A6822F4E0625A6011200021202320634B
:1069600084F83E10204684F83D30FFF72FFAFFF7F9
:10697000FABB1A68002122F480621A6006915A69F3
:1069800006929A690692069A1A6842F400721A6090
:106990004DE6596821F4E061596019680022202011
:1069A00041F400711960226384F83D0094F83E3090
:1069B00084F83E20402B20467FF4BCAEFFF712FA4D
:1069C000FFF7D1BB5A6822F4E0625A601A680021CE
:1069D000202542F400721A602046216384F83D505D
:1069E00084F83E10FFF7F2F9FFF7BDBB1A6822F4F6
:1069F00080621A605A6812F400623BD01A68002163
:106A000022F480621A6003915A6903929B6903938E
:106A1000039B0CE694F83E20402A7FF4FAAC3EE556
:106A20001A6842F480621A605A6812057FF549AF0D
:106A300007280FD801287FF444AF5A6842F48052E7
:106A40005A603EE7EBFFFEFF010100011400010068
:106A5000CC000020224A0838C240D6077FF531AF6B
:106A6000EBE7002384F83E3020462363FFF716FA55
:106A7000FFF779BB04925A6904929A690492049AC6
:106A80001A6842F400721A60D1E501287FF471AFF0
:106A90001A6822F480621A609DE61968606A21F41F
:106AA00080611960596821F4E06159601B690370C5
:106AB000638D013B20219BB2638584F83D10636A9E
:106AC00094F83E100133402963627FF4BFAE84F82E
:106AD0003E2020462263FFF7E1F9FFF744BB00BFE9
:106AE0000101000170B502685469536890F83E10C6
:106AF000E60582B0C9B223D5DD054FEA132CC3F3F6
:106B0000002E1DD56FF480735361A30539D56FF442
:106B10000073536163054FF0030543D4230507D584
:106B20001CF0010F04D06FF4006345F008055361B9
:106B3000036C2B43036402B0BDE87040FFF72EBA2C
:106B4000A60503D5DD054FEA132C24D46605C4F34E
:106B500080250ED54FEA132CC3F30025DB0543D463
:106B6000260504D51CF0010FDDD1002DE0D102B0C7
:106B700070BD2105FBD54FEA132C1CF0010FF4D09A
:106B8000D1E76305C4F380250CD4C4F3C0252405E4
:106B9000E8D47546CCE76FF40073536163054FF09A
:106BA0000205BBD5438D90F83DC0066B20299BB2F2
:106BB0005FFA8CFC0FD06FF48063102945F0040558
:106BC000536101D040290CD11368240543F40073AC
:106BD0001360A8D4ACE74BB16FF48063536145F008
:106BE000040521059FD4A3E70025DBE70CF0F7039C
:106BF000212B0CD0BCF1280FEED1212E07D06FF441
:106C000080632605536145F004058CD490E790F825
:106C10003D30C16A0829DBB20AD0202908D0212BD7
:106C200021D06FF48063536122059ED502687AE714
:106C3000282BF4D1184BC3625368019023F4E0630E
:106C400053606FF480635361136823F480631360AF
:106C500000232022036380F83D2080F83E30FFF7B8
:106C6000BFF80198E0E70C49C1620363202380F874
:106C70003D30002380F83E305368019023F4E063F8
:106C800053606FF480635361136823F4806313606F
:106C9000FFF7A0F80198C7E70000FFFF90F83D005C
:106CA000704700BF10B40D4C0D4A236823F0030356
:106CB000034323601369012943F0040313610AD0DD
:106CC00040BF20BF20BF064A5DF8044B136923F084
:106CD00004031361704730BFF5E700BF0070004048
:106CE00000ED00E0F0B44C6A34B1B2F1406F03D073
:106CF0008B6A0568013B2B618B691BB30D6A002D04
:106D000047D00068CE698F68C7612343002E50D0FA
:106D10001343CC6A2B43334323430C6B23434C6B09
:106D200023430C692343CC6823430C6823434C69F9
:106D3000B2F1406F43EA844343614BD04B688361B7
:106D4000F0BC70470B6A93B10068CD698E68C6616C
:106D50002343002D51D0CC6A13432B4323430C6BA8
:106D600023434C6B23430C692343CC68DEE7CB6998
:106D7000002B51D1002C2DD0CB6A006823430C6B23
:106D8000134323434C6B4A69234343EA82434361E1
:106D900020E0CD692343FDB1CC6A006813432B4347
:106DA00023430C6B23434C6B2343CC6823430C6875
:106DB000BCE7CC6A1A4342EA050323430C6B4A6BD7
:106DC0000D69234313430C684A692B43234343EA69
:106DD00082434361F0BC7047CC6A1A4342EA040321
:106DE0000C6B4A6B23430C684969134323430268C5
:106DF00043EA8143F0BC53617047CC6A1343234399
:106E00000C6B4A6B23430C6913434A69234343EADF
:106E10008243F0BC436170472343CC6A006813434C
:106E200023430C6B23434C6B9EE700BF704700BFAE
:106E300070B50446FDF7B6FE0646002C4CD094F81B
:106E4000413003F0FF02002B3DD0A56C2168A26801
:106E50000B68013A23F4F85343EA02230B608B6872
:106E600013F0200325D1E669E268256A08683243F9
:106E70002A436568A66920F07F4042EA056220F057
:106E8000D00002430A6062694D681848324326699F
:106E9000284042EA064202434A600A6801252A4322
:106EA0000A601846636484F84150002384F8403037
:106EB00070BD6B1CD3D0FDF775FE801BA8420DD8AA
:106EC00065B12168CBE784F84020204641F288353F
:106ED000FFF7ACFFA564B9E7012070BD042384F877
:106EE0004130636C012003436364DEE7FEF8E0FF9A
:106EF000704700BF10B5044670B10268136823F0F4
:106F000001031360FFF7F4FF00236364184684F85D
:106F1000413084F8403010BD012010BD2DE9F84308
:106F200004460E461546FDF73DFE94F84030012B11
:106F3000804643D0012384F8403094F84130012B3F
:106F40005FFA83F907D04FF00209002384F840303C
:106F50004846BDE8F88300236364022384F8413087
:106F60002768BA6812F0200216D131462046FFF792
:106F7000B9FE736A2BB1012384F8413009E06B1C20
:106F800021D1BB689A07FAD502220123FA6084F85E
:106F900041304FF00009D8E7691CE2D0FDF702FE4E
:106FA000A0EB0800854201D3002DD9D1042384F839
:106FB0004130636C43F001036364C6E74FF002099C
:106FC0004846BDE8F883FDF7EDFDA0EB08039D42C0
:106FD000ECD3002DEAD02768D3E700BF2DE9F047B6
:106FE00005461E4689469246FDF7DCFD95F8403081
:106FF000012B07465DD0012385F8403095F84130DC
:10700000012B5FFA83F807D04FF00208002385F8C0
:1070100040304046BDE8F08700236B64422385F88A
:1070200041302C68A368980627D4DAF80030A362B0
:10703000DAF804306362DAF80830E362236823F494
:10704000400CDAF810304CEA030C4CF48002DAF809
:107050000C30226049464FF00062C9F828302846BB
:10706000FFF740FEA3681A0718D508220123E26043
:107070004FF0000885F84130C8E7711CD2D0FDF709
:1070800091FDC01B864201D3002ECAD1042385F88E
:1070900041306B6C43F001036B64B7E7731CE1D0C4
:1070A000FDF780FDC01B8642F0D3002EEED02C6889
:1070B000D8E74FF002084046BDE8F08770B50446B7
:1070C000FDF770FD94F84130064698071BD5002265
:1070D000236884F840201A6851072AD41A68A56CDE
:1070E00042F002021A609A6892070ED50222A56C3D
:1070F000DA609A68910612D45A69012122F040623E
:107100005A6184F84110002070BD681CEBD0FDF777
:1071100049FD801B85421CD3DDB12368E3E76A1C6F
:10712000E7D0FDF73FFD801B854212D38DB1236868
:10713000DFE71A68E06B22F004021A60FDF7B0FE88
:1071400008B92368CAE7626C236842F004026264EB
:10715000C4E7042384F84130636C43F001036364A3
:10716000012070BD2DE9F843044689461746FDF716
:1071700019FD94F84030D4F80080012B054668D002
:10718000012384F8403094F84130012BDEB206D060
:107190000226002384F840303046BDE8F8830023FF
:1071A0006364B9F1000F58D0122384F84130D8F845
:1071B00010300133E362D8F81030C4F82490013362
:1071C000A362D8F8143023F04063C8F81430E36A9F
:1071D00041462BB38B685B070FD5636A1B7888F831
:1071E0002030E16A636A0139E162E26A0133636275
:1071F00062B321688B685B07EFD4781CEAD0FDF797
:10720000D1FC401B874201D3002FF2D1042384F824
:107210004130636C43F0010363640CE07B1C0ED1CE
:10722000D8F808309A07F9D50223C8F80C30204660
:10723000FFF744FF0646012384F84130A9E7FDF734
:10724000B1FC431B9F42E1D3002FDFD0D4F8008074
:10725000E6E702263046BDE8F883636C43F0080396
:10726000636496E72DE9F843044617468946FDF71F
:1072700099FCD4F80080D8F8182094F84030012BFD
:1072800005466ED0012384F8403094F84130012B3C
:10729000DEB206D00226002384F840303046BDE836
:1072A000F88300236364B9F1000F5ED0222384F8D1
:1072B0004130D8F810300133A363D8F81030C4F847
:1072C000309001336363D8F8143023F0406343F007
:1072D0008063C8F81430C8F81820A36B41463BB34C
:1072E0008B6813F0060F10D0236B98F820201A70CB
:1072F000A16B236B0139A163A26B013323636AB3D2
:1073000021688B6813F0060FEED1781CE8D0FDF7EA
:1073100049FC401B874201D3002FF1D1042384F89C
:107320004130636C43F0010363640CE07B1C0ED1BD
:10733000D8F808309A07F9D50223C8F80C3020464F
:10734000FFF7BCFE0646012384F84130A3E7FDF7B2
:1073500029FC431B9F42E1D3002FDFD0D4F80080EB
:10736000E6E702263046BDE8F883636C43F0080385
:10737000636490E770B5244E88B00D461446F8B9A2
:107380000090336B43F001033363336B069003F0DB
:10739000010300934FF480720223CDE902231B48BE
:1073A0000022032302A9CDE90423009BFDF7ACFED4
:1073B000B36823F0EC632B432343B36008B070BD84
:1073C00000220192336B124843F004033363336BA2
:1073D000069203F0040301934FF400720223CDE9F7
:1073E000022302A900220323CDE90423019BFDF718
:1073F0008BFEB36823F0784343EA050141EAC401F8
:10740000B16008B070BD00BF00380240000002400B
:1074100000080240014B0122DA6470470000474235
:10742000164908B58B6803F00C03042B1BD0082BFE
:1074300017D14A684B68496813F4800302F03F0291
:1074400013D10F48C1F38811A1FB000110F008F817
:107450000A4B5B68C3F3014301335B00B0FBF3F0FD
:1074600008BD074808BD074808BD0648C1F3881194
:107470000023A1FB00010FF0F3FFE9E70038024011
:107480000024F40000127A002DE9F0410D46044674
:1074900060B1454A136803F00F038B4209D2CBB2A7
:1074A0001370136803F00F038B4202D00120BDE874
:1074B000F0812368980714D5590704D53B498A6899
:1074C00042F4E0528A601A0704D538498A6842F4C7
:1074D00060428A603549A0688A6822F0F00202435F
:1074E0008A60DF0721D56268012A55D0931E012BDF
:1074F0002E4B1B684DD99907D8D52C4EB36823F075
:1075000003031343B360FDF74DFB41F28838074690
:1075100004E0FDF747FBC01B404542D8B3686268F2
:1075200003F00C03B3EB820FF3D11F4A136803F08F
:107530000F03AB4206D9EBB21370136803F00F03CD
:10754000AB42B3D123685A0706D51849E0688A6868
:1075500022F4E05202438A601B0707D5134A2169CF
:10756000936823F4604343EAC1039360FFF758FF35
:107570000E4A0F4C92680F49C2F303120346A25CF5
:107580000D48D34000680B60FDF7DCFA0020BDE831
:10759000F0819801B1D489E7044B1B689E03ACD4F9
:1075A00084E7032083E700BF003C0240003802402C
:1075B00000CA0108CC000020C8000020014B186858
:1075C000704700BFCC000020044B05499B68054A6A
:1075D0000868C3F38223D35CD84070470038024068
:1075E000CC000020F8C90108044B05499B68054AF6
:1075F0000868C3F34233D35CD84070470038024078
:10760000CC000020F8C901080E4B0F2202609A68D6
:1076100002F0030242609A6802F0F00282609A6807
:1076200002F4E052C2609B68DB0810B403F4E0533C
:10763000054C036123685DF8044B03F00F030B60F6
:10764000704700BF00380240003C02402DE9F04185
:10765000036813F0010582B004460BD09D494569CB
:10766000D1F88C2022F0C0622A43B5FA85F5C1F822
:107670008C206D0999070BD59649A069D1F88C200B
:1076800022F0C05202430028C1F88C2008BF012517
:107690001A0700F1A4805A0705D58F4B94F83820BB
:1076A000C3F8E0212368DF0608D58A49606AD1F86B
:1076B000942022F440020243C1F894209E060BD588
:1076C0008449A06AD1F8942022F000620243B0F10C
:1076D000006FC1F894202AD0590614D4012D30D05F
:1076E000802B2ED0DA0508D57A49E06AD1F88C20B3
:1076F00022F000420243C1F88C209B050DD40020EB
:1077000002B0BDE8F0817349206AD1F8942022F0DC
:1077100080520243C1F89420E0E76E4A216BD2F810
:107720008C3023F400430B43C2F88C30E7E7580653
:1077300007D5D1F89430226A23F080531343C1F85F
:107740009430664B634E00229A66FDF72BFA05468D
:1077500004E0FDF727FA431B022B3CD833681A01DB
:10776000F7D45D4B626BC3F8D8202268D3077ED56F
:107770006369002B7BD1E368A06861681B0643EA5C
:10778000801320690B43534943EA0073C1F88430E6
:1077900010060CD5E368A068626821691B0643EAFD
:1077A000801313434B4A43EA0173C2F884304B4BB6
:1077B000484E01229A66FDF7F5F9054604E0FDF70B
:1077C000F1F9401B022806D833681901F7D5236860
:1077D000DA0592D588E7032002B0BDE8F0813D4B81
:1077E0003F4E002201921A6C42F080521A641B6CC8
:1077F00003F080530193019B336843F4807333603B
:10780000FDF7D0F9074604E0FDF7CCF9C31B022BC6
:10781000E1D83368DB05F7D52E4EE369326F12F4F9
:10782000407212D003F44071914210D0336F2B4A52
:107830000121C2F8401E23F440730021C2F8401E0B
:107840003367336FD80736D4E36903F44072B2F577
:10785000407F25D01F498A6822F4F8128A601D4AA9
:10786000116FC3F30B030B431367236813E79707E9
:1078700003D5A369002B3FF47EAF960604D5A36A17
:10788000B3F1006F3FF477AF550681D5236A002B23
:107890007FF47EAFA36AB3F1006F7FF479AF6AE73C
:1078A0000C48826823F0704122F4F81221F44071F0
:1078B0000A438260D3E7FDF775F941F2883807463D
:1078C00004E0FDF76FF9C01B404584D8336F99077A
:1078D000F7D5B9E7003802400010474200004742A0
:1078E000007000402DE9F0410368DD0782B00446D6
:1078F0002FD59F498A6802F00C02042A00F0C2804A
:107900008A6802F00C02082A00F0B8806368B3F5B8
:10791000803F00F0F980B3F5A02F00F04C81944D2A
:107920002A6822F480322A602A6822F480222A609F
:10793000002B40F0EE80FDF735F9064605E0FDF737
:1079400031F9801B642800F202812B689B03F6D476
:1079500023689F0728D5864A916811F00C0F00F024
:107960009F80916801F00C01082900F09580E36880
:10797000002B00F00F817F4B7D4E01221A60FDF736
:1079800011F9054605E0FDF70DF9401B022800F24C
:10799000DE8033689807F6D53368226923F0F80350
:1079A00043EAC203336023681A0716D56369002BC4
:1079B00000F081806F4B6E4E0122C3F8802EFDF7E0
:1079C000F1F8054605E0FDF7EDF8401B022800F24E
:1079D000BE80736F9B07F6D5236858072FD5644A7E
:1079E000136C13F0805377D00025634E3368D905AC
:1079F00040F19D80A368012B00F0AD80052B00F0C5
:107A000019815B4E326F22F001023267326F22F031
:107A100004023267002B40F0A380FDF7C3F841F267
:107A20008838074605E0FDF7BDF8C01B404500F269
:107A30008E80336F9807F6D4002D40F0C680A3697E
:107A4000C3B14B4DAA6802F00C02082A2FD0022BBA
:107A5000484B4FF000021A6600F0BD80FDF7A2F817
:107A6000044604E0FDF79EF8001B02286FD82B683F
:107A70009B01F7D4002002B0BDE8F0814A685002B3
:107A80007FF544AF3A4A126891037FF562AF6268AE
:107A9000002A7FF45EAF0AE0526856023FF567AFF6
:107AA000334A1268950723D5E268012A20D00120C5
:107AB00002B0BDE8F0812F4A2D4EC2F8803EFDF79E
:107AC00071F8054604E0FDF76DF8401B02283ED82A
:107AD000736F9F07F7D47FE70193136C43F08053D4
:107AE0001364136C03F080530193019B01257CE721
:107AF0001F4920690A6822F0F80242EAC0020A60BF
:107B00001A077FF56AAF51E7194A136843F48033C7
:107B10001360FDF747F8164E054604E0FDF742F8FE
:107B2000401B642813D833689A03F7D510E73368ED
:107B300043F480733360FDF735F807463368DA05A0
:107B40003FF558AFFDF72EF8C01B0228F6D90320E9
:107B500002B0BDE8F081064A136F43F001031367DA
:107B6000FDF720F8024F064641F288380BE000BFCF
:107B7000003802400000474200700040FDF712F854
:107B8000801B4045E3D83B6F9B07F7D5002D3FF4A2
:107B900056AF1AE02C4A2D4E1360FDF703F8054648
:107BA00004E0FCF7FFFF401B0228D0D83368990798
:107BB000F7D42368F8E6254B1A6842F480221A604D
:107BC0001A6842F480321A60A3E7204A136C23F04B
:107BD0008053136433E7FCF7E5FF064604E0FCF747
:107BE000E1FF801B0228B2D82B689901F7D4216AE3
:107BF000E369626AE06A0B4343EA8213A26A216B7B
:107C000043EA0063520843EA0173013A0E4943EA2A
:107C1000024301226B600A66FCF7C4FF0B4D044669
:107C200004E0FCF7BFFF001B022890D82B689A01E4
:107C3000F7D51FE7054B1A6F42F004021A671A6F57
:107C400042F001021A678BE7000047420038024009
:107C5000704700BF10B50446A0B1437903F0FF029E
:107C600063B12168022363710B68002243F00403AF
:107C700001200B6060711046A26010BD0271FFF719
:107C8000E7FFEEE7012010BD704700BF38B504469E
:107C9000002860D0437F03F0FF02002B5DD02368F3
:107CA00053220220CA21607759625A62DA68550667
:107CB0003CD599686268256921F4E00121F0400112
:107CC0009960616998682A430A430243E1689A60AF
:107CD00019611A69A16842EA01421A61DA6822F060
:107CE0008002DA609A6891060DD51A6CA06922F4B8
:107CF00080221A641A6C02431A64FF21012259621D
:107D00000020627738BDDA6822F0A002DA60FCF762
:107D100049FF054605E0FCF745FF401BB0F57A7FBB
:107D200014D82368DA689206F5D5DEE74FF0FF3203
:107D3000DA60FCF737FF05462368DA685006B8D4E6
:107D4000FCF730FF401BB0F57A7FF5D92268FF21A0
:107D5000042351626377012038BD0277FFF794FF57
:107D60009DE700BF0368503343F82120704700BFF0
:107D70000368503353F82100704700BF2DE9F041EC
:107D800080460E4615461F46D8F8003001E07A1CA2
:107D90000AD19C6836EA04040CBF01240024AC42DA
:107DA000F5D10020BDE8F081FCF7FCFE069BC01A6F
:107DB000B842E9D3D8F80030D8F804105A68B1F5C1
:107DC000827F22F0E0025A6014D0D8F82820B2F561
:107DD000005F07D11A6822F400521A601A6842F450
:107DE00000521A600122002388F8512088F8503090
:107DF0000320D7E7D8F80820B2F5004F02D0B2F53B
:107E0000806FE2D11A6822F040021A60DDE700BFFD
:107E100030B5174B174D1B68A5FB035C85B04FEAC7
:107E20005C5C4FF47A7303FB0CF303934368B3F584
:107E3000827F044607D10CE0039B2268013B039339
:107E400093681B0602D5039B002BF5D1002005B0DB
:107E500030BD00920B4600228021FFF78FFF0028E3
:107E6000F4D0636D43F0200303206365EFE700BFA8
:107E7000CC000020819F5E1630B50B46114642684B
:107E8000B2F5827F83B0044608D000910022012120
:107E9000FFF774FF88B9002003B030BD8268B2F5E7
:107EA000004F1ED0B2F5806F0ED0009100228021CD
:107EB0002046FFF763FF0028EDD0636D032043F0F9
:107EC0002003636503B030BD05682A6822F04002D4
:107ED0002A60009100220121FFF750FF0028DAD02C
:107EE000EBE70068026822F040020260DDE700BFB5
:107EF000704700BF70B5044600283BD090F8513061
:107F000003F0FF02002B30D004F1080007C86368BB
:107F1000666A03430B436169E06913430B432268BC
:107F2000216A022584F8515003430B431168A0696C
:107F3000A56A21F0400111602B43010C00F4007090
:107F40000343136001F004033343B5F5005F53604E
:107F500004BFE36A1361D369002023F400630121A5
:107F6000D361606584F8511070BD80F85020FFF730
:107F7000BFFFC9E7012070BD90F85030012B10B54C
:107F8000044660D090F851300120834284F85000BC
:107F900042D100294CD0002A4AD00023A068A286F2
:107FA0004FF0030C84F851C06365E2862268E387D2
:107FB000B0F5004FA36363642364A38708BF13680D
:107FC000216304BF43F480431360A36AB3F5005FE9
:107FD00030D0A06C1D4B03641D4BC3631D4BC364A9
:107FE00000230365E38E0C329BB2FCF71DFFC0B982
:107FF00023681A68520603D41A6842F040021A60D5
:108000005A6842F020025A605A6842F002025A60EE
:10801000002384F8503010BD0220002384F8503033
:1080200010BD636D012243F01003636584F8512095
:108030000120F2E7136823F400531360136843F43C
:1080400000531360C5E7022010BD00BF8581000802
:10805000D9810008B581000838B5044690F8500071
:10806000012871D0012084F8500094F8510065680F
:1080700001285FFA80FC0DD0B5F5827F04D0022084
:10808000002384F8503038BDA0680028F7D1BCF137
:10809000040FF4D1002960D0002A5ED0002B5CD000
:1080A00094F8510021630428A16AA3861CBF05200F
:1080B00084F851000020B1F5005F60652168E38617
:1080C000A263A387E3872064606407D10B6823F46D
:1080D00000530B600B6843F400530B6094F851306D
:1080E000E06C042B3BD0204B0364204BC363204B3C
:1080F000C36400230365E38F0C319BB2FCF794FE4D
:10810000014618BB2268A06C536843F0010353601A
:10811000E38E0164C163C16401659BB2216B0C32C3
:10812000FCF782FE90B923681A68520603D41A68D5
:1081300042F040021A605A6842F020025A605A68BF
:1081400042F002025A609BE7022038BD636D0122B3
:1081500043F01003636584F85120012090E7054B3C
:108160000364054BC363C2E7A5810008FD820008D4
:10817000B58100089581000849820008704700BF5A
:10818000704700BF08B5806BFFF7FAFF08BD00BF5E
:10819000704700BF08B5806BFFF7FAFF08BD00BF4E
:1081A000704700BF08B5806BFFF7FAFF08BD00BF3E
:1081B000704700BF806B026808B5536823F0030363
:1081C0005360436D012143F01003436580F8511063
:1081D000FFF7EEFF08BD00BF30B5054683B0846BE6
:1081E000FCF7E0FC2B681B68DB05024621D4236802
:1081F000586820F020005860586820F0020058604D
:1082000064212046FFF704FE18B1636D43F020039C
:108210006365A36833B922680193D36801939368B7
:108220000193019B01230022E28684F85130636DA3
:1082300023B92046F9F724FD03B030BD2046FFF7EF
:10824000B7FF03B030BD00BF30B5054683B0846BC7
:10825000FCF7A8FC2B681B68D905054621D42368C8
:10826000A16A5A68B1F5005F22F020025A6035D049
:10827000A26852B35A6822F001025A602A46642169
:108280002046FFF7F9FD08B120236365012223682A
:108290000021E18784F851209A68D20606D4636DE4
:1082A00073B92046FFF76AFF03B030BD626D4FF629
:1082B000EF7142F0020262659960636D002BF0D0AD
:1082C0002046FFF775FF03B030BD6268B2F5827FCC
:1082D000D0D15A6822F003025A60CFE70122009001
:1082E000642311462046FFF749FD18B1636D43F042
:1082F000020363652368DA68BAE700BF30B5054654
:1083000083B0846BFCF74EFC2B681B68D9050546CF
:1083100022D42168A26A4B68B2F5005F23F02003E3
:108320004B602DD02A4664212046FFF771FD18B11D
:10833000636D43F02003636523685A68002122F0CF
:10834000030201205A60E186E18784F851009A68AF
:10835000D20606D4636D73B92046F9F7ABFC03B0BF
:1083600030BD626D4FF6EF7142F0020262659960B6
:10837000636D002BF0D02046FFF71AFF03B030BD2D
:1083800001220090642311462046FFF7F7FC18B144
:10839000636D43F0020363652368DB68C2E700BFD7
:1083A00030B502685168936813F0400F85B00446F9
:1083B000C3F3801505D113F0010F02D011F0400F67
:1083C00068D1980701D508065ED413F0200FC3F3D7
:1083D000401039D0880635D5002D5DD1606D40F054
:1083E000010060650020029090680290106820F003
:1083F000400010600298D8053CD4636D13B35368F5
:1084000023F0E003536001208B0784F851005BD018
:108410005368E06C23F00303536040B12C4B0365B9
:10842000FCF786FD18B1636D43F040036365A06CF3
:1084300040B1274B0365FCF77BFD18B1636D43F03A
:108440004003636505B030BD85B18D06FAD594F85B
:108450005150032D24D0656D45F0040565650090ED
:10846000D0680090906800900098C4E7DB05E9D5DB
:108470008D06E7D5636D002043F008036365039024
:1084800093680393039BB8E7636C204605B0BDE88F
:1084900030401847036CF9E794F85100032807D1DE
:1084A00000230193D368019393680193019BC9E76B
:1084B000606D40F00400606500200090D06800907E
:1084C00090680090009889E72046FFF771FEB9E7B1
:1084D000D584000808B5806B0023C387C386FFF7E7
:1084E00067FE08BD704700BF70B50E4615460446CE
:1084F00018B390F8493003F0FF02CBB1214651F890
:10850000080B00F053FBA2682068314600F08CFB9A
:10851000236BA2686068294600F0B2FB2268A1685C
:1085200052F8213043F0010342F82130002070BDA1
:1085300080F84820FFF7D6FFE0E7012070BD00BFBC
:10854000704700BF0368DA6842F00102DA609A6897
:1085500002F00702062A03D01A6842F001021A60EC
:10856000002070470368DA6822F00102DA601A6AB4
:1085700041F211110A4208D1196A40F244421142F3
:1085800003D11A6822F001021A600020704700BF70
:10859000704700BF704700BF704700BF704700BF03
:1085A000704700BF03681A69910710B5044602D5E9
:1085B000DA6892075FD41A69500702D5DA68510762
:1085C00046D41A69120702D5DA6810072ED41A6940
:1085D000D20602D5DA68D00618D41A69D10702D5B6
:1085E000DA68D2075DD41A69100602D5DA68110676
:1085F0005FD41A69520602D5DA68500661D41A6946
:10860000910602D5DA68920643D410BD6FF01002CD
:108610001A61DB69082213F4407F2277204664D078
:10862000FFF7BAFF002223682277D6E76FF008022F
:108630001A61DB69042299072277204652D1FFF79D
:10864000A9FF2046FFF7AAFF002223682277BEE792
:108650006FF004021A619B69022213F4407F2277B3
:1086600020463CD1FFF796FF2046FFF797FF0022F8
:1086700023682277A5E76FF002021A619B69012245
:108680009B07027725D0FFF787FF00222368227718
:1086900091E76FF0200220461A61BDE8104000F01B
:1086A000B3B86FF001021A612046FFF771FF23682B
:1086B00099E76FF080021A61204600F0A7F823685E
:1086C00097E76FF040021A612046FFF769FF2368C1
:1086D00095E7FFF75FFF2046FFF760FFD5E7FFF75D
:1086E0005BFFC4E7FFF758FFAEE7FFF753FF2046F5
:1086F000FFF754FF96E700BF334A0368904230B457
:108700004BD0B0F1804F33D0A2F57C4290422FD0B5
:1087100002F5806290422BD002F58062904227D011
:1087200002F57842904238D002F57052904223D040
:10873000264A904220D002F5806290421CD0A2F5D9
:108740009832904218D002F58062904214D002F51F
:108750008062904210D04D698C680A6823F08003D3
:108760002B4303600123C462826230BC43617047C3
:108770004A6823F070031343CC684A6923F44073BA
:10878000234323F0800313438C680A6803600123AA
:10879000C462826230BC436170474C68CA6823F08F
:1087A0007003234323F4407313434A6923F0800387
:1087B000134303608B68C3620B6883620B690363B6
:1087C000012330BC43617047000001400044014078
:1087D00010B50446B0B190F83D3003F0FF0263B12C
:1087E0002146022351F8040B84F83D30FFF784FF43
:1087F000012384F83D30002010BD80F83C20FFF7B5
:108800009FFEEDE7012010BD704700BF704700BF1D
:108810000268116938B50446C068A368256921F467
:10882000405101431161D168E0692B43656921F42E
:1088300016412B4321F00C0103430B43D3605369D2
:10884000A16923F440730B43B0F5004F5361284BEB
:1088500023D09A421ED003F580639A421AD0FEF7C5
:10886000B3FE636819219A00A0FB01019B0F0EF073
:10887000F7FD204AA2FB00135B092168642404FB76
:10888000130000013230A2FB00201B0103EB501348
:108890008B6038BDFEF7A8FEE3E79A4225D003F5CA
:1088A00080639A4221D0FEF78FFE626819219218E8
:1088B0004FF000035B41A0FB01010EF0D1FD0D4A1A
:1088C0002468A2FB00314909642303FB1103DB0088
:1088D0003233A2FB0323C3F342121B0902EB011242
:1088E00003F4F8731344A36038BDFEF77DFEDCE7A4
:1088F000001001401F85EB51704700BF38B504469A
:1089000050B390F8393003F0FF0203B322682423F8
:1089100084F83930D36823F400532046D360FFF73E
:1089200077FF23681A6922F490421A615A6922F08B
:108930002A025A61DA680025202142F40052DA60E6
:108940002846E56384F8391084F83A1038BD80F879
:108950003820FFF7D1FFD9E7012038BD704700BFAD
:10896000704700BF08B590F83A30222B22D18368B7
:10897000B3F5805F1FD0036943BB836A0268591C4B
:10898000526881621A70C38D013B9BB2C3858BB95B
:108990000368DA6822F02002DA60DA6822F4807272
:1089A000DA605A69202122F001025A6180F83A10F7
:1089B000FFF7D6FF08BD0269836A82B90268526870
:1089C000C2F3080223F8022B8362DCE70368826AA1
:1089D0005B68511C03F07F0381621370D3E7026868
:1089E0005268D2B223F8012B8362CCE7704700BFF4
:1089F00003681A6870B51607DD68596904460CD11A
:108A0000910601D5AE065DD4160601D5280632D4EE
:108A1000510601D56A064AD470BD11F0010168D132
:108A200015F4907FF0D0D6070AD5E80540F19E8076
:108A3000E06B40F00100E06350074BD500295CD1AA
:108A4000960760D5100700F18E80E16B0029E3D016
:108A5000900602D5A90600F18D805A69E16B02F0FB
:108A6000400201F0080152EA010553D12046FFF708
:108A7000BDFFE56370BD94F83920212ACCD1A268EE
:108A8000B2F5805F226A7AD0511C216212785A6056
:108A9000E28C013A92B2E284002ABDD1DA6822F077
:108AA0008002DA60DA6842F04002DA6070BDDA68AB
:108AB000202122F04002DA60204684F83910FFF7C6
:108AC0004DFF70BDBDE87040FFF74CBFE805AFD467
:108AD000560712D4960716D50029B3D0E16B41F0A2
:108AE0000401E1631107B0D5E16B41F00801E163D6
:108AF000ABE7D007EAD4560730D5E06B40F0020070
:108B0000E0639007EAD416079FD505F020000843DC
:108B10009BD0E9E7DA6822F49072DA605A69202182
:108B200022F001025A6184F83A105A69520611D5AE
:108B30005A69606B22F040025A6158B1164B0365C6
:108B4000FCF7F6F900283FF467AF606BBDE87040B2
:108B5000036D18472046FFF749FF70BD9007BDD44D
:108B60001107C1D471E7A906BED46EE756073FF5D9
:108B700067AFAFE72046FFF7F5FE23686DE7118882
:108B80002069C1F30801596010B9023222627FE7FF
:108B9000013222627CE700BF9D8B000808B5806B24
:108BA0000023C385C384FFF721FF08BD0A68F0B422
:108BB00050F822301B4D8C68CE68CF6B1D404B683F
:108BC000234333430E6933434E693343CE69334302
:108BD0000E6A33434E6A33438E6A3343CE6A33435D
:108BE0000E6B33434E6B896B33433B430B432B4339
:108BF000082C08BF43F04003B6F5801F40F8223030
:108C000003D042B90020F0BC7047002AFAD00368B4
:108C100043F480130360036819430160F0BC002033
:108C2000704700BF8004C0FF0B6900EB820203F1B4
:108C3000FF3C536810B58C6903F0404E0B6823432A
:108C40004C6843EA04138C6843EA0423CC684969FE
:108C500043EA044343EA0C53023943EA016343EA1B
:108C60000E0353600368DB024FEA0C5C05D54368D2
:108C700023F470034CEA03034360002010BD00BFDF
:108C8000B3F5804F30B406D06FF0704340F8223017
:108C900030BC0020704750F822300A4C8D691C40CF
:108CA0000B682B434D6843EA05138D68C96843EA96
:108CB000052343EA0143234340F8223030BC00201F
:108CC000704700BF0000F0CF054BD3F888204FF06D
:108CD000006142F47002C3F888209960704700BFB9
:108CE00000ED00E0DFF834D0002103E00C4B5B58CE
:108CF000435004310B480C4B42189A42F6D30B4AAE
:108D000002E0002342F8043B094B9A42F9D3FFF7F3
:108D1000DBFF0FF099FDF7F7B5FA7047000004206C
:108D2000A01A02080000002008020020080200200B
:108D300098180220FEE737B50D4600F108010246FB
:108D4000C36A03C91C688DE803001046694601F038
:108D50008AF8B5F90020BDF9003022449A4217DCA8
:108D6000B5F90420BDF90430121B9A4210DBB5F9A5
:108D70000220BDF9023022449A4209DCB5F906000E
:108D8000BDF90630041B9C42ACBF0020012000E06E
:108D9000012003B030BDB0F9003070B5B0F9046007
:108DA0001588D088948852884D80F31A9BB2181A7F
:108DB0009B1A08808B80CC8070BD438E1B0713B537
:108DC0000C460FD5684601F061FBBDF802302380E8
:108DD000BDF80630A380BDF800306380BDF80430D4
:108DE000E38002E0084601F051FB02B010BD38B547
:108DF00004460D4601F0F9FFE36A284629461A6841
:108E0000BDE8384005F0D0BA37B50C46054607F046
:108E100033FB428E0190944203D04486284602F0F0
:108E20002CF801A807F036FB03B030BD37B50C466F
:108E3000054678B107F020FB428E019004EA02015A
:108E40008C4204D014434486284602F016F801A848
:108E500007F020FB03B030BD37B50D46044670B1B6
:108E600007F00AFB428E019022EA05018A4203D0F4
:108E70004186204602F001F801A807F00BFB03B081
:108E800030BD0000024B42861B68C36201867047FA
:108E9000D0000020F0B50D4685B00646002800F051
:108EA000938007F0E9FA2B680290162B52D00CDC65
:108EB000112B33D002DC0D2B3ED07EE0142B77D06B
:108EC000152B7AD1B0F9303070E01F2B6BD002DC5B
:108ED0001E2B42D071E0312B1ED0B3F5407F6CD1F8
:108EE000C36A1968EB68C3621B6802A8CD1A07F051
:108EF000D1FA304607F0C0FA04AC694244F8040DD8
:108F00000A462B46009500F034FF204607F0C2FACF
:108F1000304601F0B2FF4EE000243FE0438ED90618
:108F20004BD5EB681B7A002B47D002A807F0B2FAAA
:108F3000304601F017F840E0EB68DB68002B3CD0CE
:108F40001B7A002B39D002A807F0A4FA304601F0B2
:108F5000BDFA30E0EB6803862DE0EB68418E012B13
:108F600008D1CA060DD5304641F00101FFF74CFF8C
:108F7000082708E021F001013046FFF745FF0927E7
:108F800001E04FF0FF3702A807F084FA7B1C4FF096
:108F9000000405D03046394601F0B7F8EC600DE02A
:108FA0000123EB600AE0438EC3F30013EB6002E0A1
:108FB000E968FFF71CFF002400E00124029B23B1B5
:108FC00002A807F067FA00E00124204605B0F0BDD2
:108FD00070B50D46FE211646044601F035FA2946C5
:108FE00000F0B3FF2046FF2101F02EFA3146BDE824
:108FF000704000F0AABFF8B51C46438E069F1B07C1
:109000000D4616460AD5002C07DB2846311BA2194F
:1090100006F00CFB013C3D44F5E7F8BD002C07DBF6
:109020002846311BA21906F089F8013C3D44F5E7BA
:10903000F8BD37B505460C4619B9684601F026FA61
:109040006C466B8E1B0705D5224628466946FFF7FE
:10905000A2FE6C4628462146FFF76DFE18B1EB6A6A
:1090600020461B69984703B030BD2DE9F04F2DED28
:10907000028B85B00D4607F0FFF90090006905F0FE
:109080000FFF009BD86805F039FF022005F0ECFEC9
:10909000009CA68CE36916F001061AD0002B77D04D
:1090A000A06807F0E9F90190C26A636917681F4474
:1090B00001F01EF9A369384433B1012B70D1B5F921
:1090C000003083426CDD1CE0B5F90430834218DBCC
:1090D00066E0002B5CD0A06807F0CEF90190C36A6F
:1090E000D3F8008006F004F863690746C8EB03096B
:1090F00001F006F9B5F90210EA88484407448F42A6
:1091000003DA01A807F0C6F942E012B29042F8DC97
:10911000A06802A901F0FCF8019BBDF90CB0DA6D62
:10912000D3F854A0BDF90870256AC2EB0B0BB3F855
:109130007820D207574458BFD3F88C603D4435445B
:10914000BD4222DDE369ED1AFAE7BD421BDDA069ED
:1091500005F094FE236AD4ED0A7AEB1ACAEB0303F6
:10916000C8EB03039B1B08EE103AB8EEC88A2846EA
:1091700028EE278A494605F09FFFB0EE480A94F88A
:109180002C0005F099FCE3691D445D45DDDDB8E781
:10919000684607F07FF905B0BDEC028BBDE8F08FA3
:1091A000A06802A901F0B4F8019B1D6ED3F85880A5
:1091B00005F09EFFBDF90E60019BBDF80AA0D3F833
:1091C0008030761B256A751B1D44B54201DAE369C0
:1091D000FAE74FF0020990FBF9F908FA8AF39D4289
:1091E0008FDBB5421CDCA06905F048FE236AD4ED94
:1091F0000A7A711BC91A019BD3F880208A1808EEDD
:10920000102AB8EEC88A384628EE278AC9EB05012D
:1092100005F052FFB0EE480A94F82C0005F04CFC23
:10922000E369ED1AD9E700002DE9F34781463020C4
:10923000884617461E4607F0F1FB8246D0B107F07C
:109240001BF902AD0D4A45F8040D4FF07E538362C1
:10925000C0F81490C0F818808784C66100F10C0330
:10926000044692E8030083E80300054B2360284688
:1092700007F010F9504602B0BDE8F087D400002096
:109280006B90000800B52DED028BF0EE408A83B0A4
:1092900090B107F0F1F890ED0A8A0190B4EE688A77
:1092A000F1EE10FA04D0C0ED0A8A806801F0E5FD05
:1092B00001A807F0EFF801E09FED048AB0EE480A3C
:1092C00003B0BDEC028B5DF804FB00BF00000000A2
:1092D00013B5044607F0D0F80190406A20B107F0BA
:1092E00005F9019B00225A6201A807F0D3F8204635
:1092F00007F0FCF802B010BD2DE9F0438BB007F089
:10930000BBF80790406A002860D007F0B5F8079BCB
:1093100005900646986807F0AFF8079BD0F8548090
:10932000056E876DC46D069008A9986800F0F0FF7F
:10933000BDF82230079A0698BDF82010D2F8209088
:109340001F44ADF82270BDF82430BDF826701C1BF8
:109350007F1B1369D0F88C505D1B92F82830414474
:1093600089B2A4B2BFB2012BADF82010ADF82440F1
:10937000ADF82670D0F8808009B208D024B2641B02
:109380000134A14204DD0C1B06EB44062D1B0C46E8
:10939000002D15DD906905F0B1FD4FF0FF3201237E
:1093A0008DE80C00079A3FB292F829300293C9EB7E
:1093B000070930462946224609EB080306F05AF908
:1093C00006A807F067F805A807F064F807A807F0F3
:1093D00061F80BB0BDE8F0831FB590F82830012B81
:1093E0000446806827D102A900F092FFA06807F028
:1093F00043F8BDF80A20836D01901344ADF80A309C
:10940000BDF80E20036ED31AADF80E30426DBDF8D4
:1094100008301344226913449BB29A1E01A8013BF1
:10942000ADF80820ADF80C3007F034F8A06802A9B8
:1094300001F0E7FC01E000F05FFB04B010BD0000AC
:109440002DE9F74380462C200E4617461D4607F0AF
:10945000E5FA044618B3700007F0E0FA814658B107
:1094600057B14DB107F008F839466A0001900FF086
:1094700067FA01A807F00EF8204606F0FDFF0A4B38
:109480000190C360094B0360094BC0F82490C0F8F9
:10949000188046610561436001A806F0FBFF204685
:1094A00003B0BDE8F08300BFD9930008F99200082B
:1094B000D19200081FB5ADF8061006F0DDFF02904E
:1094C00068B1406A06F0D8FF0DF10602014603902C
:1094D0000223029800F03FFB03A806F0DBFF02A87E
:1094E00006F0D8FF05B05DF804FB13B50C4660B17B
:1094F00006F0C2FF036A0190A34203D004628068B1
:1095000001F0BBFC01A806F0C5FF02B010BDF0B52C
:109510008BB002A9044600F0FBFE204606F0ACFF2B
:10952000BDF90A20BDF90E600190B61A826D456D35
:10953000C76DB61A026EB61AB0F87820510707D474
:10954000416FB1422046D4BF0021012100F0FBFC55
:10955000019BBDF90C105A6FDA67BDF90820C3F8FA
:1095600084608A1A551BB3F878209207C7EB05056B
:1095700007D4196FA9422046D4BF0021012100F071
:10958000E0FC0198036FC0F88830C0F890507C3040
:1095900000F08AFF0198883000F086FF019B03F1FC
:1095A0007C0207CA883307AE86E8070093E8070005
:1095B00004AD85E8070001A806F06CFF204631469F
:1095C0002A46FFF705FD0BB0F0BD73B50C46064605
:1095D00006F052FF0190204607F05AFB0546204650
:1095E00000F0F6FE019BFE280CBFC3F88050C3F8C4
:1095F0008C50304601F041FC01A806F04BFF02B050
:1096000070BD2DE9F04F44680668054697B02046C6
:109610002946FFF73FFCB6F5407F074602D12046BA
:10962000FFF775FF002F00F064822B680B2B00F012
:10963000008206DC052B40F059822046FFF767FFC9
:1096400054E20F2B03D0262B00F03D824EE2ED6852
:109650000295204606F010FFC36AC16D1B68D0F862
:109660005490D0F858B0D0F860A00D900EAD2846B8
:109670000393019100F00AFF0D982946FFF7D9FCEA
:1096800095E8030012AB83E803000398BDF84A1085
:1096900082B25944BDF84E001144ADF84A1002EBB5
:1096A0000A01411AADF84E10BDF848101144494462
:1096B000ADF8481001990A44BDF84C108A1AADF86B
:1096C0004C2093E8030010AA82E80300104600F043
:1096D000FBFB0D9B586B05F00FFC06F09DFA0D9BF4
:1096E000D3F8943013B12046002198470D9D95F88A
:1096F0006C30002B00F08D80204614A900F008FE8D
:10970000EB6ABDF856001B68BDF85420BDF8521036
:1097100004930790BDF85030286C05920693089189
:109720006E6CAF6C05F0EAFB05F0DCFC099016B935
:10973000002F4BD146E0EB6C06EB030CB5F878300C
:10974000DB0754BFD5F88C3000230CEB0308B04581
:1097500002DBC6EB0808FAE795F87A0005F098FBFB
:109760000598019A03B206984A4401B2C2F1010277
:109770005B1A13449845DBDA0498BDF95210BDF921
:10978000563095F87A20484440445944CAEB0303C4
:109790001AB1024605F02CFF02E01A4605F0CEFC95
:1097A000B044DDE795F87B0005F072FB0799089857
:1097B0000BB20BEB0A0201B2C2F101025B1A1344B5
:1097C0009E420CDB099805F063FB22E02E6DD5F874
:1097D00080303E44F61ABE42E4DBF61BFBE70198FC
:1097E000BDF95420BDF95610BDF95030121A95F844
:1097F0007B00CAEB0101891B4B4420B118460B4684
:1098000005F0F6FE03E00846194605F00FFF3E445A
:10981000CCE7039A12A80EA904F0C6FD12A800F026
:1098200053FB0D9B93F83B20FF2A00F0A380B9F176
:10983000000F08D1BBF1000F05D1019919B9BAF198
:10984000000F00F09780DA6A14A92046156800938B
:1098500000F05EFD00F04CFD049000F051FDBDF9FC
:109860005220009BBDF9546005905A440392019A1E
:10987000986BBDF95070BDF95680B61A05F03CFBE7
:10988000009BD86B4F44CAEB080805F037FBB9F1D1
:10989000000F1BD002980499B0F9003009F1FF3293
:1098A0002A445B1A934211DCBDF95630BDF95000D1
:1098B000CAEB030305EB0B01013306F07BF9039AB6
:1098C000781E511E08F1010205F038FCBBF1000FB3
:1098D00017D002980599B0F902200BF1FF332B4401
:1098E000521A9A420DDCBDF95000BDF95210BDF973
:1098F000542006F05FF9039A791E501E721C05F081
:1099000095FE019BD3B10299BDF95420D01AB1F94B
:109910000430049901305B1A83420FDBBDF95630E5
:10992000CAEB030305EB0B01013306F043F9039A7D
:10993000701C511E08F1010205F000FCBAF1000F85
:1099400018D00298BDF95630B0F906200598CAEB38
:1099500003010131C0EB020A8A450BDBBDF950005F
:10996000BDF9542006F026F908F10100791E721C99
:1099700005F05CFE0D9BD3F8943013B12046012115
:10998000984710A800F0A0FA0D9B586E07F08CFCC9
:1099900000250746BD421AD00D9B2946586E07F098
:1099A00005FD06F069FD149078B10668304606F0B2
:1099B00063FD0C9030B103680299304698470CA8BB
:1099C00006F068FD14A806F065FD0135E2E712A86F
:1099D00000F07AFA0D9B986E07F066FC00250746AA
:1099E000BD421AD00D9B2946986E07F0DFFC06F0A9
:1099F00043FD149078B10668304606F03DFD0B90AB
:109A000030B103680299304698470BA806F042FD32
:109A100014A806F03FFD0135E2E7002000F054FAFB
:109A20000D9BD3F8943013B12046022198470DA81E
:109A300046E0204606F020FD1290406E07F034FC10
:109A400000240646B442129B18DA586E214607F0ED
:109A5000ADFC06F011FD149070B10568284606F0C3
:109A60000BFD109028B1476810A806F013FD28469A
:109A7000B84714A806F00EFD0134E3E7986E07F02E
:109A800013FC00240546AC42129B0FDA986E214667
:109A900007F08CFC06F0F0FC149028B1006806F08A
:109AA00025FD14A806F0F6FC0134ECE716AC586E60
:109AB00007F053FC54F8103D986E07F04EFC20461A
:109AC00006F0E8FC15E0EB68052B0FD12046AE68E8
:109AD00000F0F0FB864205D02046AE6800F0E5FBC2
:109AE000864203D16868A968FFF76FFD284601F038
:109AF000EFFD17B0BDE8F08F2DE9FF41044606F0F9
:109B0000BBFC034604A8D3F8548040F80C3D9F6D7D
:109B1000DE6D1D6E06F0BEFC204602A900F0F8FBCB
:109B2000BDF808309844BDF80A30ADF808801F44ED
:109B3000BDF80C30ADF80A709E1BBDF80E30ADF8C4
:109B40000C605D1B204602A9ADF80E5001F059F9DA
:109B500004B0BDE8F081F8B51D46836804460E46A2
:109B6000174623B30069636998420ED1421E6A43C7
:109B7000084629440EF036FE2069013800FB0560D6
:109B800039462A460EF02EFE0CE0431C236100FBF2
:109B9000051011462A460EF025FEE36813B1204653
:109BA0009847F8BDA068BDE8F840FFF7A5BFF8BD2D
:109BB000F0B587B00C9C00940D9C0194174C029456
:109BC000109C6C34039401F099F9064618B307F021
:109BD00000FC054607F0FDFB0446304606F04CFC51
:109BE00045660F4D84660F9905900022FFF74AF9EC
:109BF00006AF0FCD57F804ED0EF134040FC40FCDAE
:109C00000FC495E80F0084E80F000E9BAEF8783083
:109C1000384606F03FFC304607B0F0BD039600081A
:109C2000DC00002010B586B0089C0094099C0194CB
:109C30000A9C02940B9C039400240494FFF7B8FF41
:109C400006B010BD30B585B004460191D0B106F024
:109C500013FC04AB456E43F8040D184606F01AFCDD
:109C6000019806F009FC024604A8946040F8082D0B
:109C700006F010FC284601A9042207F024FB204628
:109C800001F0FBF805B030BD30B585B00446019158
:109C9000D0B106F0F1FB04AB856E43F8040D184615
:109CA00006F0F8FB019806F0E7FB024604A8946072
:109CB00040F8082D06F0EEFB284601A9042207F023
:109CC00002FB204601F0D9F805B030BD73B50D4652
:109CD0001446064698B106F0CFFB032C019009D834
:109CE00000EB8400446BAC4205D04563304601F084
:109CF000C4F800E0002401A806F0CCFB00E0044614
:109D0000204602B070BD73B50E46054678B106F028
:109D1000B3FB90F86C400190B44204D080F86C60C2
:109D2000284601F0AAF801A806F0B4FB00E00446BA
:109D3000204602B070BD2DE9F3410F4690461D4606
:109D4000064698B106F098FB044602A8089B2366D5
:109D500040F8044D6765C4F85880E56506F09AFB45
:109D60003046FFF7D4FB304601F087F802B0BDE87B
:109D7000F0812DE9F04F87B0C46903938A4693467A
:109D8000002C6DD0204606F077FB816A059001F427
:109D90002073802BB0F8008042888688C58808D060
:109DA000B3F5207F08D108EB0A091FFA89F9039B54
:109DB00008E0039883B201E01FFA8AF303EB080975
:109DC0001FFA89F901F4A0613344B1F5807F9BB299
:109DD00008D0B1F5A06F08D102EB0B0C1FFA8CFC78
:109DE000109F08E010998FB201E01FFA8BF707EB84
:109DF000020C1FFA8CFC0FFA89F90FFA88F812B2DC
:109E00002F440FFA8CFCB9EB08010292BFB2C2EBEF
:109E10000C0200D142B120460193CDF800C000F001
:109E200008FADDF800C0019B1BB2C9EB030936B28A
:109E3000029BC6EB08083FB22DB2CCEB070C5D1BB2
:109E400019EB08010CEB050200D112B1204600F01D
:109E5000E1F806A850F8043D1C6A06F01BFB8FE7EA
:109E600007B0BDE8F08FB0F90030B0F90220084625
:109E70005242594205F0D4B810B5044670B100F012
:109E8000FCFF204600F0BBFA04463CB12046FFF739
:109E9000F3FF204606F0E6FA046AF6E710BD13B5B4
:109EA000044670B106F0E8FA826A0190930705D47F
:109EB00042F0020282622046FFF7DEFF01A806F0B0
:109EC000E9FA02B010BD0000044B10B51B685C6CD1
:109ED000586400F02BFE204610BD00BF2401002076
:109EE000F7B50D46114606461F4600F0ADFA04468A
:109EF000A5B120B93046394606F0D9FE14E006F087
:109F0000BBFA02AB826A43F8040D22F4004242F02D
:109F100002028262184606F0BDFA05E020B100F0A8
:109F20008CF9204601F006FB201C18BF012003B06D
:109F3000F0BDFE220823FFF7D3BFFF220023FFF767
:109F4000CFBFFFF7FABFFFF7F4BF1FB530B129B19C
:109F5000242303916946009300F038FF05B05DF8B3
:109F600004FB0000F0B587B00446002102A81022CF
:109F70000EF052FC002C3AD01F4B204A196852F8C0
:109F80002100844216461F4631D01E238DE8110061
:109F9000029310B102A907F033FA0123204602A967
:109FA000059307F02DFA059D15BB3B6846F8234045
:109FB000204600F084F9044638B12023029302A918
:109FC00000AB059307F01CFAF2E7009C204600F076
:109FD00032F968B1204600F072F9044640B12023FE
:109FE000029302A900AB059307F00AFAF2E70125F4
:109FF000284607B0F0BD00BF341702202417022006
:10A00000024B1A6818601046704700BF3C170220C8
:10A0100007F0E2B92DE9F04151EA02038AB0804627
:10A020000E4617466ED000286CD006F025FA03467F
:10A03000039003C804AD06AC85E8030084E8030080
:10A040007EB19A6A02F42072802A05D1BDF81820E8
:10A05000961BADF8186004E0BDF81C201644ADF85E
:10A060001C6087B19A6A02F4A062B2F5807F05D1C4
:10A07000BDF81A20D71BADF81A7004E0BDF81E20F9
:10A080001744ADF81E709B6ADA0302D5404600F013
:10A0900081FD94E80300039B83E803009B6A9B0710
:10A0A0000AD508A82946224604F0CAFF039B08A83F
:10A0B00099691A6A00F072FEBDF91C40BDF91430AE
:10A0C000BDF91E70BDF91600BDF91860BDF910107C
:10A0D000BDF91A50BDF91220E31A381A0AACAA1AAF
:10A0E0000090711A0398FFF744FE54F81C1D01F10B
:10A0F000080004F015FA4046052100F06BFE2046EA
:10A1000006F0C8F90AB0BDE8F0811FB52623039117
:10A110006946009307F09AFA05B05DF804FB2DE953
:10A12000F04188B006460C46154604A800211022CE
:10A130000EF072FB36B3304606F09EF921462A46F1
:10A14000019004F06DFF0198214608302A4604F082
:10A1500067FF08A850F81C2DD2F81C80176A06F07B
:10A1600099F9404621462A46FFF7D9FF0323049375
:10A17000304602AB04A90793029403953E4607F0CC
:10A180003FF9D7E708B0BDE8F0812DE9F0438BB087
:10A1900006460D46144606A8002110220EF03CFB90
:10A1A000002E43D00DB9002C40D0304606F064F9A3
:10A1B0000346019003C80DF1080888E80300224611
:10A1C0001846294604F02CFF01980AAF294622467A
:10A1D000083004F025FF57F8243DD3F81C9038468A
:10A1E00006F058F9224648462946FFF798FF3046C0
:10A1F00006F042F9826A019092070AD5816941B15D
:10A20000026A00F0B6FD019B404699691A6A00F0A7
:10A21000B0FD384606F03EF903230693304604AB02
:10A2200006A909930495059407F0EAF80BB0BDE878
:10A23000F083FFF7AABF00F09DBC13B588B106F00C
:10A240001BF9826A02AC910744F8040D06D522F08E
:10A25000020282628169026A00F0A0FD204606F0D7
:10A2600019F902B010BD70B506460D4606F0FAF8B1
:10A27000C4694CB1204600F0ABF8A842204613D088
:10A2800006F0F0F8046AF4E7304606F0EBF8C4692B
:10A29000204644B12946FFF7E6FF28B9204606F0DC
:10A2A000E1F8046AF4E770BD70BD10B1FF21FFF75B
:10A2B000DABF704710B1FE21FFF7D5BF704708B570
:10A2C000034610B106F0CEF88369184608BD08B5FC
:10A2D00020B106F0C7F8B0F9000008BD08BD08B508
:10A2E00020B106F0BFF8B0F9020008BD08BD0000BB
:10A2F000024B1B68986CFFF7EABF00BF24010020E7
:10A30000024B1B68986CFFF7EABF00BF24010020D6
:10A31000F0B50C4687B0064600284BD0002949D03E
:10A32000FF2100F091F8FE210546304600F08CF840
:10A3300069460746304607F0B1F9304602A900F0F9
:10A340003BF8C7B1384604A907F0A8F9BDF90010D9
:10A35000BDF9022004A84942524204F061FE384689
:10A3600000F046F800F08200822804D1BDF81030D9
:10A37000013BADF80C30CDB1284604A907F08EF9A9
:10A38000BDF90010BDF9022004A84942524204F070
:10A3900047FE284600F02CF800F48170B0F5817F6C
:10A3A00004D1BDF81230013BADF80E3002AB03CB47
:10A3B0002060616007B0F0BD1FB5039104A91423AC
:10A3C00041F8103D694600F001FD05B05DF804FB61
:10A3D0001FB504461022684600210EF01DFA152311
:10A3E00020466946009300F0F1FC039804B010BDCC
:10A3F00008B518B106F036F8008D08BD08BD08B5DF
:10A40000034610B106F02EF8C369184608BD37B5EB
:10A410000D4606F031F802ABC46943F8040D184646
:10A4200006F038F820466CB1FFF7D2FFA84220466C
:10A4300008D02946FFF7EBFF20B9204606F012F8B6
:10A44000046AEFE703B030BD08B1FFF7E0BF704723
:10A45000034B1B685A7C034B53F82200704700BF24
:10A46000240100201417022037B50D4658B151B110
:10A4700006F002F802AC294644F8040D00F0B5FCE1
:10A48000204606F007F803B030BD0000044B01463B
:10A49000186810B9034B1B68986CFFF7E5BF00BF45
:10A4A000101702202401002002688368D31A426832
:10A4B000002ABCBF00224260426823EAE3739A424A
:10A4C000C8BF4360704700F0D8BC000073B50546B4
:10A4D000002832D005F0D0FF02AC034644F8080D46
:10A4E000006A08B968460EE09B6A1A0711D405F0A5
:10A4F000C3FF836A02AE1B0746F8040D06D5684603
:10A5000005F0C8FF304605F0C5FF16E0304605F0FF
:10A51000C1FF009B68469E6905F0BCFF284600F01D
:10A52000B7FA3146284600F061FA284600F0A5FC4B
:10A5300028460349002207F0D0F802B070BD00BFE2
:10A54000C7A400080A4A0B49002313700A4A0B608B
:10A5500013600A4A4B601360094A13605360094A4A
:10A560001360094A1360094A1360094A136070476F
:10A57000E4D7012024170220BCD70120481702206D
:10A58000501702205C170220101702203C170220EF
:10A590004C17022010B5044605F064FF836A044A94
:10A5A00013F4803F034B204608BF1346984710BD65
:10A5B000F9B30008E5B90008F0B5054685B00C46CA
:10A5C0001646002D4CD0284605F056FF876A0190AC
:10A5D000BB0701463DD502AD26B12846324603F001
:10A5E0006DFF02E003C885E803002046294604F019
:10A5F000CDFC70B317F0010F019B1ED13EB1B3F932
:10A600000220B6F902309A42A8BF134601E0B3F91E
:10A610000230B4F902209342B4F9062006DDBDF8F9
:10A620000A3019B28A4214DB013B04E0BDF80E3057
:10A6300019B28A420DDDE3800BE0DF694FB1384685
:10A6400021462A46FFF7B8FF384605F00BFF076A98
:10A65000F4E704A850F80C3D1D6A05F01BFFB0E7B5
:10A6600005B0F0BD2DE9FF4104460F469046002598
:10A67000002C37D0204605F0FFFE866A0190B20715
:10A68000014628D502ACB8F1000F04D0204642465E
:10A6900003F014FF02E003C884E8030038462146B3
:10A6A00004F074FCB8B1F30705D4BDF80C300133E5
:10A6B0003B8001250FE0019BDE6966B130463946DB
:10A6C0002246FFF7CFFF0028304618BF012505F0CE
:10A6D000C9FE066AF1E704A850F80C3D1C6A05F0B3
:10A6E000D9FEC5E7284604B0BDE8F081F0B50446C0
:10A6F00085B00E461746002C31D0204605F0BCFE32
:10A70000856A0190AA07014622D502AC27B12046EE
:10A710003A4603F0D3FE02E003C884E80300304663
:10A72000214604F033FC98B1EB0704D4BDF808309F
:10A73000013BB3800CE0019BDD694DB128463146F9
:10A740002246FFF7D3FF284605F08CFE056AF4E7A2
:10A7500004A850F80C3D1C6A05F09CFECBE705B040
:10A76000F0BD00002DE9F341214D2B680646986CA1
:10A7700005F082FE0090304605F07EFE02AC0146F8
:10A78000019054F8080D083004F000FC074628B387
:10A790000199009A2B68174C1F6DD3F84C8001F17A
:10A7A0000800083203F08AFE684605F073FE019A3D
:10A7B0002B68B2F90010B2F90220D9641A6501A819
:10A7C000266005F067FE3046FFF7E4FE00232360B5
:10A7D0002B681F65C3F84C80012705E0684605F02B
:10A7E00059FE01A805F056FE384602B0BDE8F081DA
:10A7F00024010020101702202DE9F347064605F03A
:10A800003BFE836A01909B0705D401A805F042FE38
:10A8100002B0BDE8F087C469002CF6D0204605F0F0
:10A820002BFE836A02AD03F00303032B45F8080DEA
:10A8300037D10199083104F0A9FB002831D002A8D2
:10A8400050F8043DB3F80890B3F80A809F89B3F834
:10A850000EA005F01FFE684605F01CFE2046FFF71F
:10A8600081FF70B1204605F0FDFD00902046FFF706
:10A87000C3FF204605F0F6FD0090304605F0F2FDDE
:10A880000190304605F0F8FD0190204605F0F4FDFA
:10A89000019B0090A3F80890A3F80A809F81A3F879
:10A8A0000EA0009B68461C6A05F0F4FDB4E70000AA
:10A8B00037B5044605F0E0FD826A019040F60103D9
:10A8C0001340012B05D001A805F0E4FD2046FFF759
:10A8D00061FE144B1B6813B32046FFF78DFF204623
:10A8E00005F0C0FD8569046ACDB194B1204605F03C
:10A8F000B9FD836A03F00303032B02D12046FFF75F
:10A9000031FF2046FFF778FF204605F0ABFD046AD3
:10A91000EBE7284605F0A6FD046A8569E4E703B085
:10A9200030BD00BF5C1702202DE9F347174D2B689F
:10A930000646986C05F0A0FD2A68B0F808A0B0F8AB
:10A940000A90B0F80C80C78902AC083244F8040DB4
:10A9500000F1080392E8030083E80300204605F0B5
:10A9600099FD3068FFF7A4FF2B68986C05F084FD13
:10A970000190A0F808A0A0F80A90A0F80C80C78168
:10A98000204605F087FD02B0BDE8F08724010020D5
:10A99000F7B507460D46284605F06EFD836A02AC02
:10A9A00013F00206014644F8040D04D1204605F0D8
:10A9B00071FD304616E0384603F0B2FD019B9E69FA
:10A9C000204656B905F066FD074B1A68954208D037
:10A9D00058682B1A5842584104E005F05BFD354693
:10A9E000D9E7012003B0F0BD14170220F0B50446EA
:10A9F00085B00D46002949D005F03EFD00230362D5
:10AA000085610190284605F037FD019BC5690290DC
:10AA10009F6A2DB9C46101A805F03CFD02A833E08E
:10AA2000284605F029FD04AE07F0080746F8040D96
:10AA300077B9836A1A070BD5019B1D62029B01A897
:10AA4000DC6105F027FD02A805F024FD30461BE07F
:10AA500002A805F01FFD304605F01CFD284605F054
:10AA600001FD0390039B1D6A0DB91C620BE0284693
:10AA700005F0F8FC002FF4D1836A1B07F1D5039B86
:10AA80001C62019B1D6201A805F004FD05B0F0BD2C
:10AA900070B5044605F0E6FC05468069A8B105F0EE
:10AAA000E1FCC369A342064605D1184605F0DAFC6D
:10AAB000036AF36170BD43B1184605F0D3FC036A25
:10AAC000A342F8D12B6A036270BD70BD03460846ED
:10AAD000B3F90220B3F9001004F0A2BA114B30B55B
:10AAE0001C68626C85B00546BAB11068516802AB4B
:10AAF00003C30D4B186800B9A06C05F0BDFC04AC95
:10AB000002A944F80C0DFFF7E1FF204605F0C2FC56
:10AB100002A8294603F004FD02A802F033FF05B0A5
:10AB200030BD00BF24010020101702201FB50E4BBE
:10AB30001B6893F854200AB10C4811E0986C05F09A
:10AB40009BFC019003C802AC84E8030001A805F057
:10AB5000A1FC074B196811B12046FFF719FF2046E9
:10AB6000FFF7BCFF04B010BD24010020C8D70120AE
:10AB700010170220064B10B50446186828B1A042F1
:10AB800004D005F06FFC4069F8E710BD012010BD4E
:10AB90003017022013B5044600B305F06DFC826A3D
:10ABA0000190930717D5406A40B10D4B1B68A34233
:10ABB00004D001F0DFFD019B00225A622046FFF71E
:10ABC0001EFC04463CB12046FFF7E4FF204605F09A
:10ABD00049FC046AF6E701A805F05CFC02B010BD70
:10ABE00058170220B0F90020B0F904309A4208DC6E
:10ABF000B0F90220B0F906309A42CCBF0020012003
:10AC00007047002070470000F0B585B006460D463D
:10AC1000174605F027FC846A0190A30734D528461F
:10AC2000FFF7E0FF00282FD040F601032340012B5F
:10AC30002AD0304605F020FC02AC0246019029469D
:10AC4000204603F03BFC2046FFF7CCFFC8B1019B38
:10AC50009E6A44F22001314003F1080529B12846DB
:10AC60002946224604F0ECF90BE094E803003E4349
:10AC700085E803009E62054B1A8801321A8003F0B2
:10AC800015FE01A805F006FC05B0F0BD2C1702204A
:10AC90002022FFF7B9BFF0B50F4685B0154606462E
:10ACA00048B305F0E9FB836A04AC9B07024644F80D
:10ACB0000C0D03D4204605F0EDFB1CE002A839463C
:10ACC00003F0FCFB0028F5D0204605F0E3FB3046FE
:10ACD00002A92A46FFF798FF3046FFF790FB04468B
:10ACE0004CB1204602A92A46FFF7D5FF204605F0C1
:10ACF000B9FB046AF4E705B0F0BD2DE9FF418046D9
:10AD000017461D460C46002930D0084605F0B4FB16
:10AD1000866A0190B307024625D502A8414603F092
:10AD2000CDFB00B340F601033340012B07D1019B5B
:10AD300002A899691A6A2B46FFF7DFFF04E0204654
:10AD400002A92A46FFF760FF019BDC695CB1BC42A7
:10AD500009D0204602A92A46FFF79DFF204605F0AC
:10AD600081FB046AF2E701A805F094FB04B0BDE89A
:10AD7000F08170B5054608460C46164605F072FB94
:10AD8000836A13F4803F2846214632460CBF2023B5
:10AD90004FF48043BDE87040FFF7AFBF2023FFF7BB
:10ADA000ACBF13B5044605F067FB8169019041B162
:10ADB000026AFFF7F3FF2046FFF76AFE019B0022BD
:10ADC0009A6101A805F066FB02B010BD08B106F05B
:10ADD00017BB70471FB504AB019043F8101D6946BF
:10ADE00006F00EFB05B05DF804FB00230B808288A3
:10ADF0004B800388D31A8B80C2884388D31ACB80B8
:10AE00007047F0B50F4687B00546002833D005F0EF
:10AE100033FB866A0190B2072AD503C804ACF3035A
:10AE200084E8030002D52846FFF7B4FE5FB1386816
:10AE3000796802AB03C3019802A9FFF747FE2046D9
:10AE400002A903F06DFB20462946FFF7A1FD78B16A
:10AE500040F601033340012B06D1019B204699693E
:10AE60001A6AFFF79BFF03E028462146FFF710FF11
:10AE700001A805F00FFB07B0F0BD0021FFF7C1BF2F
:10AE800010B5044605F0EEFA80690028F9D1054BAB
:10AE90001A68944205D05868844214BF4FF0FF30BE
:10AEA000012010BD1417022008B5FFF7E9FF0028A4
:10AEB00003DBBDE8084004F035B808BD0D4A13684F
:10AEC00070B59D6C0446164608B90B4A14689C641C
:10AED0002046FFF7E9FF03F04DF9204605F0C2FADE
:10AEE0003368B0F90010B0F90220D9641A65284619
:10AEF00070BD00BF24010020301702202DE9F74F5C
:10AF00000C9D9B464B4B0746884692461E6865BB88
:10AF1000494B1B8863B3494B1B685A7C484B53F819
:10AF200022305A1C24D01BB31D46284605F0A4FA33
:10AF3000B0F90020B0F90230019017449844BAF1FA
:10AF4000000F05D1B0F904A0C2EB0A0A0AF1010A08
:10AF5000BBF1000F05D1B0F906B0C3EB0B0B0BF141
:10AF6000010B01A805F096FA02E06B1CDDD100256B
:10AF70000F982C3005F052FD0446002856D00D9B4A
:10AF80001E432D4B1A8801321A8005F075FA0E9B6C
:10AF900003610DF108092B4B826A49F8080D334013
:10AFA0000780A0F802805744D8441343013F08F1BA
:10AFB000FF3883628780A0F80680684605F06AFA49
:10AFC000214B186848B105F04DFA0746204605F0B8
:10AFD00049FA7B6943617C6100E01C602946204698
:10AFE000FFF704FDB50602D52046FFF767FFF0071F
:10AFF00003D5164B1A6801321A60710602D5204635
:10B0000006F076FBB2070DD5204605F035FA836AC7
:10B01000009043F002038362684605F03BFA204645
:10B02000FFF72BFF20460121FFF7D4FE204603B097
:10B03000BDE8F08F3C1702200C17022024010020ED
:10B04000141702209F3F3F00301702205C17022098
:10B0500073B5044600286ED0FFF78CFD00286AD037
:10B060002046FFF70DFF0B2105462046FFF7B2FEF5
:10B07000204606F028FA204605F0FEF90190406AC5
:10B0800008B101F077FB2D4B2D4A002119602D4BA3
:10B090001B6852F82300A04208BF42F823102A4A36
:10B0A00052F82310A14204BF002142F82310274B7D
:10B0B0001B682BB15A68A24204BF00225A60F7E70E
:10B0C00020460721FFF721F8019EF069FFF7C0FF36
:10B0D000F369002BF9D12046FFF763FE1C4B18687B
:10B0E00050B105F0BFF906464069A042F8D12046AC
:10B0F00005F0B8F943697361019B9B6ADA0703D5D0
:10B10000144A1168013911609B0603D5124B1A8845
:10B11000013A1A8001A805F0BDF9104B1A882046A3
:10B12000013A1A8005F0E2F9002D04DB0C4B53F8CC
:10B130002500FFF7C3FE02B070BD00BFD8D70120C5
:10B14000241702203417022050170220481702202B
:10B15000301702205C1702202C1702200C17022047
:10B16000141702202DE9FF415D4F3B6893F854000E
:10B17000002800F0B2805B4B5A69012A1C4603DDAF
:10B18000013A5A610020A8E004F108061B6996E81C
:10B190000300013302AD236185E8030023B923884E
:10B1A000ADF80830638811E0A3896289ADF80A2000
:10B1B00001339BB2B4F90420ADF808301BB29A42B7
:10B1C00006DA2388ADF80830E3890133ADF80A3098
:10B1D000BDF90A20B4F90630DFF808819A4204DD8F
:10B1E0006369013B0020636177E03B68986C05F080
:10B1F00043F9BDF90820B8F9003001909A421CD1FA
:10B20000B8F80630ADF80E30B8F80430ADF80C30B0
:10B21000334B1B689A6C5AB1104605F023F98046EF
:10B220000022006A2946FFF7C7F9D8F81820F2E78C
:10B23000019B2946D869FFF7BFF9BDF80830ADF882
:10B240000C303B689A6C6AB1104605F00BF9294640
:10B2500080460022006AFFF705FA0028EDD1D8F8F1
:10B260001820F0E7019B2946D869FFF7FBF9002871
:10B27000E3D1A388BDF90820ADF80C301BB29A4287
:10B2800007DD95E8030086E8030001A805F002F950
:10B2900097E73B689A6C52B1104605F0E3F8074611
:10B2A0000022006A2946FFF721FABA69F3E704AFE2
:10B2B000294657F80C3DD869FFF718FA384605F0CB
:10B2C000E9F8236944F62062934289DC95E803009B
:10B2D00086E80300FFF72AFC012004B0BDE8F081F6
:10B2E00024010020C0D701202DE9F041394F3B68EF
:10B2F00093F8542086B0064612B9FFF717FC64E0B5
:10B30000354D6A690132012A6A612C465DDC986C10
:10B3100005F0B2F84FF0FF322A61304A00901278FF
:10B320002AB100F1080302AA93E8030005E0826A4B
:10B3300012F002080AD003C802AA82E8030002AD94
:10B3400066B12846314603F0EBF807E06B696846C2
:10B35000013B6B6105F09EF8404637E03B68204EAC
:10B360005A6CC2B1009B10685168019304AB03C3CF
:10B37000336833B101A805F08DF8306805F07CF82A
:10B380000190019804A9FFF7A1FB284604A903F046
:10B39000C7F801A800E0684605F07CF8316819B1EB
:10B3A0002846FFF7F5FA28B13B682846996CFFF765
:10B3B000EFFA18B96369013B636107E095E80300A0
:10B3C00084E80300FFF7CEFE00E0012006B0BDE8F0
:10B3D000F08100BF24010020C0D7012039170220CE
:10B3E0001017022008B503F067FD024B1B6800220E
:10B3F0005A6408BD24010020F0B589B0044605F068
:10B400003BF80769866A0190083003C802AD85E8F9
:10B41000030001A805F03EF8002F31D0B3072FD567
:10B4200020462E21FEF7F4FD164B1A7816F4805FA5
:10B4300002F101021A701E460AD00F2305940493EC
:10B440000795FFF7CFFF204604A905F0D9FF10E0CC
:10B450002846FFF749FF60B10F2304930594079531
:10B46000FFF7C0FF204604A905F0CAFFFFF77AFEE8
:10B47000F1E733782046013B2F213370FEF7C8FDFA
:10B4800009B0F0BD39170220F0B589B006AC0390C1
:10B4900004F0F2FF00F108020346059092E8030071
:10B4A0009D6A9E691F6984E8030005A804F0F2FF05
:10B4B00044F220032B40002B34D0BFB12046039927
:10B4C000FFF766FA90B10398FFF7F8FC69070FD50C
:10B4D00026B105F0010585F0010500E00125009584
:10B4E0002046124903AA002300F0DAFA002403E000
:10B4F0000398FFF7DDF90124039804F0BDFF826A89
:10B50000059022F4804323F02003920448BF43F0C7
:10B510000403836205A804F0BDFF054B1A88013AB5
:10B520001A8000E01C46204609B0F0BD29A9000899
:10B530002C17022008B504F095FF836A43F40043FA
:10B540008362024B01221A6008BD00BFBCD70120F4
:10B550002DE9F04F4C4B1B689FB003B19847002674
:10B560004A4D2B68DBB14A4B1C68BCB1204604F045
:10B5700083FF826A47691EAB12F4004F43F8700DD7
:10B5800007D0184604F086FF2046FFF761FD3C46D1
:10B59000EBE718463C4604F07DFFE6E72C603D4BA8
:10B5A0001B6803B198473C4B1B682BB93B4F3B686A
:10B5B00093F8543043B103E098470028F6D058E0A0
:10B5C00003F012FD002854D13B6893F854504DB15C
:10B5D000334B1D8835B1334B1B68002B4BD01B6898
:10B5E000984701253B6893F8543013B9002D37D1A3
:10B5F00045E0DFF8AC80B8F80030002BF6D0DFF87B
:10B60000A890D9F800400CB9214B1C6802A803F09F
:10B61000A9FC3B68D3F830B0D3F834A014B90024A7
:10B620000DE063B92046FFF72FFF03462046019344
:10B6300004F018FF4469019B002CF2D1EFE7584653
:10B64000C9F8004003F05AFC504603F055FC02A82C
:10B6500003F092FCB8F80030002BC7D00126C1E7F8
:10B66000104B186810B14368984708E002F01EFFBD
:10B6700005E0012674E7012002F018FFB1E730462B
:10B680001FB0BDE8F08F00BF20170220BCD70120FB
:10B69000301702201C1702209C17022024010020D2
:10B6A0002C1702204C170220D8D70120024B1B6810
:10B6B000012283F85420704724010020034B1B68AB
:10B6C000002283F8542002F055BD00BF2401002061
:10B6D00010B5044640682368E168172B0FD006DCDC
:10B6E0000E2B0ED0142B14D1FEF7BEFE11E0222B30
:10B6F0000CD0282B0DD1BDE81040FFF7BEBBE06099
:10B7000010BD2146BDE8104005F0A0BF6FF07043AA
:10B7100000E00023E36010BD03680E2B10B5044663
:10B7200002D00F2B09D020E0C3685A68012A21D12A
:10B730001868BDE8104003F04FBC0F4A4368116819
:10B740008B4206D05268934214BF4FF0FF3301235F
:10B7500000E00023094A52F823006FF0704398423A
:10B7600003D003F0C9FB04F057FA2046BDE81040AF
:10B77000FFF7AEBF10BD00BF141702204017022014
:10B7800030B52B4B187885B01D4600284DD1294B7C
:10B790001860294B1860294B1B685864284B188087
:10B7A000284B04461880204604F012F9C0B14FF02F
:10B7B000FF3202238DE80C00002043F6FF72224B7B
:10B7C0000293039013460146FFF798FB1F4B43F883
:10B7D00024001F4B6FF0704243F82420FFF74DFB0D
:10B7E0000134022CDFD11B4805F07AFF1A4805F01E
:10B7F00077FF1A4805F074FF194805F071FF1948E2
:10B8000005F06EFF184805F06BFF104B1868FFF746
:10B8100055FBFFF74BFF01232B701448144B0360BB
:10B8200005B0BDE8304004F007BA05B030BD00BF38
:10B83000E4D7012030170220D8D7012024010020AE
:10B840002C1702200C17022019B700081417022029
:10B850004017022080180220701802206018022071
:10B86000881802207818022068180220DCD70120EE
:10B8700045A500082DE9F04F87B0044604F0FCFD13
:10B8800006AFB0F800808688B0F80290B0F806B035
:10B8900047F8040D0FFA88F836B2C8EB0606D0F860
:10B8A00024A0013638460FFA89F90FFA8BF504F017
:10B8B000F1FDC9EB0505002E05F101054DDD002D5B
:10B8C0004BDDBAF1000F4AD0504604F0D5FD06AB6F
:10B8D000868843F8080DC58836B2184604F0DAFDAC
:10B8E000464502D12DB24D4532D0504641464A46DA
:10B8F00000F086F82CE0836A43F480338362384694
:10B9000004F0C8FD404600F093FF0746504603F0A0
:10B91000F7FA404600F0B4F82D4B05FB06F2197813
:10B920002C4D2D4E920002F015FD2046D5F80080DA
:10B930003460FEF7CCFC28602046FFF75DFD002058
:10B94000C5F80080306003F0DBFA384600F070FF85
:10B95000204604F087FD406A37E0002035E0FEF71E
:10B9600077FD844212D102F09FF8824602F0A4F8DB
:10B97000564502DC854209DD00E056468542A8BFF7
:10B980000546314620462A4605F008FE134B019332
:10B990004FF0010A124B02934046494632462B466D
:10B9A000CDF800A000F04EFE8046204604F064FD75
:10B9B0000590C0F82480B8F1000F9CD1384604F0FF
:10B9C00069FD2046FFF718FD404607B0BDE8F08F3F
:10B9D0000C010020681702205817022050CA0108E5
:10B9E00028F5010838B5054605242846FFF742FF2B
:10B9F00010B9013CF9D138BDBDE8384006F086BB2E
:10BA000037B50D46144618B9114B1B68186EE8B1CE
:10BA100004F032FDA4B2ADB2C4808580009002F083
:10BA2000A9FB009B586970B104F026FD009B0190B2
:10BA30001A895B898280C38012B10BB10580448072
:10BA400001A804F027FD684604F024FD03B030BDD2
:10BA50002401002013B520B9084B1B68186E04465A
:10BA600048B104F009FD02ABB0F90A4043F8040DF7
:10BA7000184604F00FFD204602B010BD240100203E
:10BA800013B550B104F0F8FC044602A840F8044D88
:10BA900004F000FD04F11800FFE702B010BD000043
:10BAA0002DE9F04F1E4689B04E4B04921A6803915F
:10BAB000547C4D4A1257012A05469B46204606DD16
:10BAC00001F0E0FF0746204601F0DFFF05E001F04E
:10BAD000DFFF0746204601F0DEFF044625B306A837
:10BAE00007A903F0F1FA069BB5F900A0B5F9042007
:10BAF000B5F902801F44079B2AEAEA7A013F974280
:10BB0000D4BFCAEB0707CAEB02071C44B5F90620ED
:10BB100028EAE878013C9442D4BFC8EB0404C8EB9F
:10BB200002040137013401E0A846AA4606B966427C
:10BB3000002F52DD002C50DD129B009350464146F1
:10BB40003A46334600F038FE054620B90498039B78
:10BB50009847012042E0FFF77DFFA042064606D04D
:10BB6000DBF80030986C10B1322105F035FC284626
:10BB700000F05EFE73420593A1460027B14503DA4B
:10BB80002846494606F0C2FB47B12846514607EB16
:10BB90000802FFF735FF284606F0CEFB039B04980A
:10BBA0009847124B1B680BB100209847284600F0BD
:10BBB000B7FE3744059BA7429944DFDB284600F0D7
:10BBC000D9FD002000F034FEA64206D0DBF800309C
:10BBD000986C10B1332105F0FFFB002009B0BDE8DF
:10BBE000F08F00BF2401002060170220E8D7012059
:10BBF0000248012918BF0020704700BF50CA010841
:10BC00000248162918BF0020704700BF1D1F0108F9
:10BC100008290CBF20200020704708B50068C368C1
:10BC20001B6A984708BD37B580680C4604F024FCB1
:10BC3000034602A89988DA881D8940F8043D5B898B
:10BC40002180628029441A440139013AA180E280AE
:10BC500004F020FC03B030BD0E4B1B6873B50546E5
:10BC6000186E0E4604F008FC034602A8B3F906401D
:10BC700040F8043D03F11801361BDC68B3F90430C9
:10BC800004FB0614ED1A04F005FC04EB85042046C1
:10BC900002B070BD2401002008B508461146FFF728
:10BCA000DBFF006808BD0000154B1B6873B5186EFC
:10BCB00015460E4604F0E0FB294600903046FFF79B
:10BCC000CBFF009B1B681B6904469B689847236851
:10BCD0005840009B2060586960B104F0CDFB02AC75
:10BCE000836844F8040D1B6831462A46984720466D
:10BCF00004F0D0FB684604F0CDFB02B070BD00BF7D
:10BD00002401002073B51C46104B1B68186E0E46AC
:10BD1000154604F0B1FB294600903046FFF79CFF22
:10BD2000009B0460586960B104F0A6FB02AC836814
:10BD300044F8040D1B6831462A469847204604F013
:10BD4000A9FB684604F0A6FB02B070BD24010020E8
:10BD50002DE9F7432C4D1E462B68186E0F461446EE
:10BD600004F08AFB00904069A94608B104F084FB06
:10BD7000019021463846FFF76FFFD9F80020009B5D
:10BD8000D16B127CD3F80C80D1F80090D207054615
:10BD90001FD51B681B699B6898478046019828B18E
:10BDA00082683946D2F800C02246E0472B6883EA11
:10BDB00008032B60009B0134DB68B4421D44EDDDB9
:10BDC000684604F067FB019BD3B101A804F062FB55
:10BDD00016E0019B63B10198836822461B683946CF
:10BDE00001349847B442C5F800904544F3DDE7E7D5
:10BDF000341B0134013CC5F800904544FAD1DFE71B
:10BE000003B0BDE8F08300BF240100202DE9F04F0E
:10BE1000DFF8ACB01446DBF8002085B0106E0F469A
:10BE20001D4604F029FB214602903846FFF714FF17
:10BE3000029ADBF80030D2F80C90DB6B06465069B2
:10BE4000D3F800A0ED1B013538B304F015FB0E9AB2
:10BE50000DF11008131B48F8040D01330093394607
:10BE600022462B4606F03CFA404604F013FB14E051
:10BE7000DBF800301B7CDB0713D5029B1B681B69BA
:10BE80009B68984732462B461168013B81EA0001C6
:10BE900042F8041BF8D14E4401340E9B9C42E7DD6E
:10BEA00008E0002DF7DD2B463246013B42F804AB9B
:10BEB000FBD1F0E702A804F0EDFA05B0BDE8F08F81
:10BEC0002401002007B50092FFF7A0FF03B05DF842
:10BED00004FB00002DE9F04F9D4C9A46236891B079
:10BEE0008046186E07920E46DDF874B01F9D00283C
:10BEF00000F0878304F0C0FA0E90406908B104F0A6
:10BF0000BBFA0F9010A850F8083DDB680A9304F0C4
:10BF1000C1FA1E9F0F983744049750B123681B7CC9
:10BF20009C0706D41A9F00970499079A534606F077
:10BF3000D7F904980799FFF78FFE1B9F172F064626
:10BF400064DD4FEA8A0706974FF000091A9F0F98A1
:10BF5000B94557DA30B18368079A5C6804994A4456
:10BF60005346A047D8F81030D86828B13046594613
:10BF7000069A0CF0E5FC3EE05B689847000E0590E1
:10BF8000354657465C463B4622464FF0000C52F879
:10BF9000041B0598090E8142059808BF0CF1010C9D
:10BFA000814203F1FF3314D0BCF1000F14D04FEAEB
:10BFB0008C03284621461A460393CDF808C00CF09E
:10BFC000BFFC039BDDF808C01D441C44CCEB0707F5
:10BFD0000FE0002BDBD1E7E72068020EFF2A05D037
:10BFE000D2432968D2B202F0B9FA28600435043489
:10BFF000013F002FC7D11C9FBB440A9F09F10109D3
:10C000003E44A3E7002840F0F982FAE21B9F102F7C
:10C0100037D1061F00251A9F0F9CBD4280F2A080D9
:10C02000079F2F443CB1A3680499D3F804C020466D
:10C030003A465346E047ABF1020306930596D146D4
:10C040000499D8F81030069A5B6832F8020F06920D
:10C050005144C9EB010103919847059B039943F8AB
:10C06000040F059324B1A36820461B683A469847FD
:10C07000B9F10109E4D11C9FBB440A9F01353E443C
:10C08000C9E71B9F082F00F104066DD1079F079990
:10C090001A9A0F9C7B1A9342A6F1040060DA2C4B8B
:10C0A0001B681B7C6DB313F0030305D0022B51D129
:10C0B000B146DDF810801CE01BF8032055F8222063
:10C0C00040F8232001335345F6D143E055F823309F
:10C0D00049F8043C2CB1A36820461B6841463A4607
:10C0E0009847049B08F101085344434509F10409AA
:10C0F00030D00498C0EB0B0313F80830002BF0D0BD
:10C10000E4E713F0030305D0022B23D1B146DDF899
:10C11000108015E0594652460CF012FC1AE049F81E
:10C12000043C2CB1A36820461B6841463A46984718
:10C13000049B08F101085344434509F1040909D05F
:10C140000499C1EB0B0313F80830002BF0D0E6E79D
:10C15000240100201C9A0A9B934401371E4496E751
:10C16000002C40F04B824CE21E9FB24B09967F00A0
:10C170000C971E9FBF000D97079F0597002D08BFC6
:10C180001D46099F07983C1F059F3B1A1A9FBB42FB
:10C1900080F232821B9F022F00F0AD80042F00F04E
:10C1A0004F81012F40F01E82DFF89092D9F80030C5
:10C1B000186E04F061F99BF800309F4A1E99D65C16
:10C1C000D9F800300E901B7CDDF83CC003F003036F
:10C1D000022B5746C1F1080846FA01F620D0032B7E
:10C1E00061D0012B5FD05A46474538BFB846C8EBEF
:10C1F00007074346214606F00100013B55F82000A1
:10C2000041F8040B4FEA5606F5D104EB8804002FE1
:10C210006DD012F8013F88494FF00808CE5CE3E783
:10C220006B68DDF810900B93CDF820B0474538BF10
:10C23000B846C8EB0707BCF1000F26D01EB904EBC7
:10C240008804C14425E0F0070CD5DCF80830059AD5
:10C250001B68CDF808C06046494698470B9BDDF83F
:10C2600008C02360B8F1010809F1010904F10404D0
:10C270000FD07608E2E7F10744BF0B9B2360B8F1CB
:10C28000010804F1040404D07608002EF3D104EB75
:10C29000880467B30898684A10F8013F0890D65C94
:10C2A0004FF00808C2E703681B699B689847594626
:10C2B000474538BFB846C8EB0707231DC646F207F7
:10C2C00004D553F8042C424043F8042CBEF1010E6F
:10C2D0004FEA560603F10403F1D104EB880437B1A9
:10C2E00011F8013F544A4FF00808D65CE0E70EA869
:10C2F00004F0D0F876E11E9F0C9BDDF83CC0C7F13E
:10C3000004069BF800709F404C4B1B681B7C03F09D
:10C310000303012BF6B2FFB266D008D3022B40F024
:10C3200061810498CDF820B0D04606903EE05A4690
:10C3300053469E42C8BFDEB29B1B314620464FEAA1
:10C34000971C013955F82CC040F804CBBF0011F000
:10C35000FF01FFB2F3D1013EF6B2013604EB8604D1
:10C36000002B00F03F8112F8017F0426E1E70699D7
:10C3700017F0C00F494422D109F101095FFA89F28F
:10C38000BF009642FFB2F2D1069F013EF6B27B1C7F
:10C39000721C9E1904EB82040696B8F1000F00F09F
:10C3A0002181089B13F8017F089304264645C8BFE6
:10C3B0005FFA88F6C6EB08084FF00009D7E7BA091C
:10C3C00055F8222044F82920BCF1000FD4D0DCF825
:10C3D000082012680B926046CDF808C0059A0B9BA6
:10C3E0009847DDF808C0C7E7584653469E42C8BF85
:10C3F000DEB29B1B221DB44617F0C00F05D052F8C9
:10C40000041C81F0FF0142F8041C0CF1FF3CBF004A
:10C410001CF0FF0CFFB202F10402EDD1013EF6B2B6
:10C42000013604EB8604002B00F0DC8010F8017F5D
:10C430000426DBE710CA010890F30108240100205C
:10C44000714A9BF8003012680D98127C0F9F02F021
:10C4500003028340012ADEB200F09C8002D3022A4C
:10C4600035D0BFE01E9F5FB136090BF1010255F8D0
:10C47000263023609BF80160099C0AF1FF3301E03C
:10C4800053465A46012B1ADD581004F1080103F0F7
:10C49000010302EB00084FEA161C06F00F0655F8E0
:10C4A0002C7041F8087C55F8266041F8046C12F8AD
:10C4B000016F424501F10801EDD104EBC004002BEE
:10C4C00000F09080360955F8263023608AE01E98E7
:10C4D000C0B113F0F00F0AD0360955F826302360AA
:10C4E0002FB1BB6804991B68059A38469847049990
:10C4F000099C9BF8016001F101080AF1FF3C0BF176
:10C50000010911E0D446D946DDF810800CE016F0A0
:10C51000F00F0DD116F00F061BD119F8016F08347A
:10C5200008F10208ACF1020CBCF1010FEFDC21E0D4
:10C53000330955F823302360002FEBD0BB68059AF0
:10C540001B68CDF808C0384641469847DDF808C05A
:10C55000E0E755F826306360002FDED0BB68059A0F
:10C560001B68CDF808C0384608F101019847DDF88E
:10C5700008C0D2E7BCF1000F34D0360932D055F8EC
:10C580002630236077B3BB68059A1B68384641465E
:10C59000984727E01E9FC7F10203DBB25F46524671
:10C5A0009342C8BFD3B2D21A201D9C4616F0C00FCA
:10C5B00005D050F8041C81F0FF0140F8041C0CF178
:10C5C000FF3C36011CF0FF0CF6B200F10400EDD187
:10C5D000013BDBB2013304EB83041AB117F8016F9E
:10C5E0000223DDE7059B1C9F0133BB4405930A9F93
:10C5F000099B3B440993C4E50F9B13B10FA803F0BB
:10C6000049FF11B0BDE8F08F240100202DE9F3416E
:10C610000E469046074603F02FFF036802ACDB6826
:10C6200044F8040D5B6A0020162198470546204611
:10C6300003F030FF1DB1384631464246A84702B0EC
:10C64000BDE8F0812DE9F04F3E4E87B01D463368BE
:10C65000109F5B7C83468A4690461198129900226F
:10C6600003F0C8F90446002833D003699B68984753
:10C6700001F0BFFA08FB00F60390073604F0C4F897
:10C6800017F001094FEAD60604D1042390FBF3F01A
:10C6900000EB4000002D09DC1EB11838B0FBF6F0AD
:10C6A00000E030466D42A842B8BF0546B9F1000F20
:10C6B00009D1CDF800905846514642462B4605F028
:10C6C000CFFD074600E00027002D04DC204603F0E4
:10C6D0008FF9002032E006FB05F01830B9F1000FA9
:10C6E00002D004F01DF901E004F098F9814640B948
:10C6F000204603F07DF9002FEBD0384603F0F6FE1C
:10C700001BE003F0B9FE034606A8039A40F8043D77
:10C710001A611C60A3F804B0A3F806A0A3F808806F
:10C720005D81DE605F6103F0B5FE064A129B236106
:10C730001368C4F808905B7CA361484607B0BDE865
:10C74000F08F00BF2401002037B5054670B103F01B
:10C7500093FE036802AC1B6944F8040D9B6898477C
:10C7600001F047FA0546204603F094FE284603B040
:10C7700030BD000037B50446D0B10E4B1B681B6EB0
:10C78000834201D102F0E4FB204603F075FE0190E4
:10C79000406908B105F090FD02AD55F8043D1868F8
:10C7A00003F026F9284603F075FE204603F09EFEAE
:10C7B00003B030BD240100202DE9FF479A46194BF4
:10C7C0000C9D1B680746587C174B53F82040884641
:10C7D0009146E3681B68042B06D02468002CF8D12E
:10C7E00003F0F6F8044630B1E3682046DB6A012125
:10C7F0009847064608B9002010E02469A3689847C6
:10C80000013004BF45F00105084C02948DE860003A
:10C81000384641464A465346FFF714FF04B0BDE888
:10C82000F08700BF240100209017022028F501089E
:10C83000114BF7B51A680446166E1F4610B902F080
:10C8400087FB16E00EB102F083FBFEF737FF2046B0
:10C8500003F012FE02AD3B6845F8040D1C6600684B
:10C8600003F004F9284603F015FE01F079F801F011
:10C8700081FC304603B0F0BD240100202DE9F043D7
:10C880000C4685B015460646002841D0002002F02F
:10C8900011FB214B1B6807463046D3F8608003F03C
:10C8A000EBFD03680190986902F03CFB1B4B9C4236
:10C8B000019B04BFB3F90440B3F906501A895B89A0
:10C8C000ADF80840013A013B22442B448146ADF8C3
:10C8D0000C20ADF80E30ADF80A50FEF7E7FE01A8C7
:10C8E00003F0D8FD02A8FEF7FFFC48B9484602F065
:10C8F00019FB4046FFF79CFF384602F0DBFA07E0E1
:10C90000304621462A4604F077FFFEF72BFCECE781
:10C9100005B0BDE8F08300BF2401002001F0FFFF57
:10C9200001490A46FFF7AABF01F0FFFFF8B5044628
:10C930000E46D0F88C302A2115469847E16AD4F883
:10C94000903031442046C1F30F219847E16AD4F872
:10C950009030B7B239442046C9B29847E16AD4F85A
:10C96000903031442046C1F30F219847E16AD4F852
:10C97000903039442046C9B29847D4F88C302046CC
:10C980002B219847216BD4F8903029442046C1F3DD
:10C990000F219847216BD4F89030AEB23144204635
:10C9A000C9B29847216BD4F8903029442046C1F38E
:10C9B0000F219847216BD4F8903031442046C9B2FA
:10C9C0009847D4F88C3020462C219847F8BD2DE9A3
:10C9D000F041044688461F462A21D0F88C30069D37
:10C9E00016469847E16AD4F8903041442046C1F396
:10C9F0000F219847E16AD4F8903041442046C9B2EB
:10CA00009847E16AD4F8903039442046C1F30F21A9
:10CA10009847E16AD4F8903039442046C9B2984723
:10CA2000D4F88C3020462B219847216BD4F89030D5
:10CA300031442046C1F30F219847216BD4F8903040
:10CA400031442046C9B29847216BD4F8903029442C
:10CA50002046C1F30F219847216BD4F89030294428
:10CA60002046C9B29847D4F88C3020462C219847EC
:10CA7000BDE8F08113B50D4A0446516810686B4655
:10CA800003C3D4F88C30204636219847636BA18CC1
:10CA900002AA134421F0E00113F8083C1943204690
:10CAA000D4F8903089B2984702B010BD14F3010851
:10CAB00013B50446D0F80C312E209847216AD4F8DB
:10CAC0002831684603319847226A00AB13441DF8A9
:10CAD000022059789878D2088908D20242EA411295
:10CAE00042EAD00002B010BD1FB50446D0F82C3188
:10CAF0002E209847216AD4F8483168460231984779
:10CB0000236A00A901EB43023DF81300528802F4A6
:10CB10007C41C2F3C40242EA511200F0F80042EA3A
:10CB2000002004B010BD38B504460D46D0F80C31D5
:10CB3000080A9847D4F80C31E8B2984738BD08B5D0
:10CB4000D0F82C310846984708BD08B5D0F8103108
:10CB5000C8B2984708BD08B5D0F8303108469847A4
:10CB600008BD0000082902D0102905D07047064BE7
:10CB7000C0F88C30054B03E0054BC0F88C30054BFA
:10CB8000C0F89030704700BF27CB00084BCB00089F
:10CB90003FCB000857CB0008F0B585B084680A9FEA
:10CBA0000097BD1A581A013500FB0555D4F8A87036
:10CBB0000B9E2046B847D4F80C312E209847D4F865
:10CBC0002831216A02A89847D4F8283102A8032105
:10CBD00098479DF808309DF80920DB089208DB0291
:10CBE00043EA42139DF80A20013D43EAD20326F8A6
:10CBF000023BE9D105B0F0BDF0B587B084680C9F69
:10CC00000097BD1A581A013500FB0555D4F8A870D5
:10CC10000D9E2046B847D4F82C312E209847D4F8E2
:10CC20004831216A02A89847D4F8483102A8022165
:10CC30009847BDF80A3003F47C42C3F3C40343EAC7
:10CC40005213BDF8082002F0F80243EA0223013D26
:10CC500026F8023BE8D107B0F0BD000010B504464D
:10CC600000F0A6FDA368124AC3F8AC20114AC3F82D
:10CC7000A820114AC3F8B020104AC3F8B8200022F7
:10CC8000C3F8BC20C3F8CC200D4A0E491268C3F883
:10CC9000C420DA8C0968C3F8B41022F003020A49F0
:10CCA000DA840A4AC3F8C810C3F8942010BD00BF44
:10CCB0002DC90008CFC9000875CA0008B1CA00080C
:10CCC000140100201001002099CB000865CB00085A
:10CCD00008B5D0F8B430984708BD08B5D0F8303161
:10CCE00088B2984708BD00002DE9F04F3D4F846899
:10CCF00082463868007C10F0010F85B00E4615465C
:10CD00009846C1EB030945D04FEA490B0E9885427E
:10CD100065DCD4F8C4C0E76EBCF1000F01D1B446A5
:10CD200007E08DE8A000504631462A464346E047DA
:10CD300011E0C4450EDCD4F8EC30CDF80CC06146EF
:10CD400050462A469847DDF80CC027F8020B0CF134
:10CD5000010CEEE7E76EBB1E09F1010C5F44BB421C
:10CD600005D0A26A59884A4023F8022FF7E70095B8
:10CD70002A46D4F8A870CDF80CC020463146434668
:10CD8000B847DDF80CC0D4F83831E06E61469847FA
:10CD90000135BBE70E980090851AD4F8A8602046AC
:10CDA000B0473B68A76EDB6B09F10109D3F800803F
:10CDB00005FB0995012395B1FA2D34BF2E46FA26BD
:10CDC0002BB138461FFA88F1324601F095FAD4F8B3
:10CDD0003831384631469847AD1B0023EBE705B0A4
:10CDE000BDE8F08F240100202DE9F04F8DB085685B
:10CDF000179F05937B1E012B099008910A920B95B2
:10CE000003D9042F01D0082F06D18F4B1B681B7C40
:10CE100003F00303022B10D00A9A169F1A9D08995B
:10CE2000059B3A442944013A0B9D00920B44D5F8E6
:10CE3000A8400A9A2846013BA047DDF828B00A9F7F
:10CE4000169DC7EB0B03AB4280F25182179F7B1EEE
:10CE50000F2B00F24582DFE813F01000B700430209
:10CE60004001430243024302D7014302430243020B
:10CE700043024302430243023D02734B099D1B6878
:10CE8000AC681B9D1B7C2F686D680795DDF820A0A2
:10CE90001A9D03F00303022BAA441BD0032B6ED070
:10CEA000012B6CD0059EDDF8648098F80010D4F852
:10CEB000303180222A41114216BF0799B8B288B298
:10CEC00001359847082D04BF08F101080025013EEF
:10CED000EBD105E2199D0695D4F86C90DDF86880D9
:10CEE000CDF80CA0002556462B46069F4FF0800C2F
:10CEF0003A784CFA08FC12EA0C0C0BD013B9D4F8AF
:10CF00006C900396079FA9F80070013509F102099A
:10CF1000012317E0012B14D1CDF800B0CDF810C0DB
:10CF200020460399D4F8A8705A46731EB847D4F81F
:10CF30003831E06E29469847DDF810C065466346F3
:10CF400000E0634608F10108B8F1080F06F1010698
:10CF500004D1069F013706974FF00008059A524406
:10CF6000B242C2D1059F7B1E5344002D00F0B88110
:10CF7000CDF800B0D4F8A860039920463DE1DDF873
:10CF800014801A9E199DDDF814902A78802333416D
:10CF9000D1441A42C8EB09090DD0D4F8EC300998F5
:10CFA00049465A469847A36AD4F8F0704340494628
:10CFB00009985A46B8470136082E04BF01350026A5
:10CFC000B8F10108DFD18BE1099D1B9FAC68002FF0
:10CFD00000F086811C4B199D1B6895F800A01B7CF6
:10CFE00013F0030311D0022B40F07A811A9DDDF873
:10CFF0002090E76E0397A944A846199D0795002540
:10D00000CDF818904E462B4640E01A9D059E199F7C
:10D01000C5F103035B00C3F10602C02141FA02F22D
:10D0200002EA0A02DA401B99D4F8303131F82200C2
:10D0300001359847042D03D197F801A00025013749
:10D04000013EE5D14CE100BF2401002013B9E76E99
:10D05000039706961B9F57F82C30039F3B8002379F
:10D0600001350397012308F10108B8F1040F06F117
:10D07000010606D1079F97F801A0013707974FF0E7
:10D080000008059A4A44B24200F0AC80C8F103029D
:10D090005200C2F106014FF0C00C4CFA01FC0CEA40
:10D0A0000A0C3CFA02FCD1D1012B14D1CDF800B00E
:10D0B000CDF810C020460699D4F8A8705A46731EC1
:10D0C000B847D4F83831E06E29469847DDF810C0EB
:10D0D00065466346C7E76346C5E7099D1B9FAC6885
:10D0E000002F00F0FD80834B199D1B6895F800A070
:10D0F0001B7C13F0030311D0022B40F0F1801A9D2A
:10D10000DDF82090E76E0397A944A846199D07957E
:10D110000025CDF818904E462B463CE01A9D059E02
:10D12000199FC5F101039B00C3F10402F02141FAEC
:10D1300002F202EA0A02DA401B99D4F8303131F8DF
:10D14000220001359847022D03D197F801A0002550
:10D150000137013EE5D1C3E013B9E76E03970696A8
:10D160001B9F57F82C30039F3B80023701350397F4
:10D17000012308F10108B8F1020F06F1010606D1FA
:10D18000079F97F801A0013707974FF00008059A0D
:10D190004A44B24226D0C8F101029200C2F1040111
:10D1A0004FF0F00C4CFA01FC0CEA0A0C3CFA02FCC1
:10D1B000D2D1012B14D1CDF800B0CDF810C020464B
:10D1C0000699D4F8A8705A46731EB847D4F8383177
:10D1D000E06E29469847DDF810C065466346C8E70B
:10D1E0006346C6E7059F7B1E4B44002D78D0CDF8E3
:10D1F00000B0D4F8A860069920465A46B047D4F843
:10D200003831E06E29466AE0099D1B9FAC68002F0B
:10D2100066D0384B1B681B7C13F0030309D0022B2C
:10D220005ED1DDF82090D4F86C8000264F4633465E
:10D2300022E0199D199B059F3B445B1B002B4FDD92
:10D2400015F8012B1B9FD4F8303137F8220098478E
:10D25000F0E713B9D4F86C80B9461B9D55F82A3015
:10D26000A8F80030013608F102080123089A059D4C
:10D2700001372A44BA421CD0199D08982A1A12F87C
:10D2800007A0BAF1000FE4D1012B10D1CDF800B006
:10D29000204649465A467B1ED4F8A850A847D4F8E1
:10D2A0003831E06E3146984756465346DEE75346DE
:10D2B000DCE7089F6B1E3B4496B1CDF800B02046DA
:10D2C0004946D4F8A8505A46A847D4F83831E06EF9
:10D2D000314604E00B9D1998D5F8383105999847E7
:10D2E000199F189D2F4419970BF1010BA7E50DB05D
:10D2F000BDE8F08F2401002010B5044600F058FA74
:10D30000A468104BC4F8E4300F4BC4F8E8300F4B5E
:10D31000C4F8EC300E4BC4F8F0300E4BC4F8A0301B
:10D320000D4BC4F8A430D4F8C430C4F8FC30204607
:10D33000D4F89430102198471023A363074B6364FB
:10D3400010BD00BFE9CD0008E9CC0008FFD60008F9
:10D350006FD60008D1CC0008DBCC0008B4F501087A
:10D36000084670470068401A013870470846704701
:10D370000068401A01387047104670474068801AAC
:10D3800001387047104670474068801A013870476E
:10D3900010467047104670474068801A0138704741
:10D3A0004068801A01387047084670470846704741
:10D3B0000068401A013870470068401A0138704709
:10D3C00010B58468D4F8F040A04710BD08B5836854
:10D3D000D3F8EC30984708BDF7B504460F4616461B
:10D3E0008568FFF7F3FF0190DDF804E0AB6A2046A3
:10D3F000394632468EEA0303FFF7E2FF03B0F0BD81
:10D4000013B584680092D4F8E840A04702B010BD7C
:10D4100013B584680093D4F8E8400B46A04702B0E7
:10D4200010BD37B5069C85680094D5F8E840A04744
:10D4300003B030BD30B587B085680A9C00940B9C62
:10D4400001940C9C02940D9C03940E9C04940F9CDC
:10D450000594D5F8E440A04707B030BD7047000000
:10D4600073B5079E84680C4D76B1286888B9069814
:10D470000090D4F8A8602046B047D4F8A8302B60BC
:10D48000064BC4F8A83004E02B6813B1C4F8A830E8
:10D490002E6002B070BD00BFECD701205DD4000843
:10D4A00008B5026CD0F8D4309069984708BD08B52B
:10D4B000026CD0F8D8309069984708BD2DE9F74341
:10D4C0000A9D8468009517462046D4F8A8609946BE
:10D4D0008846ED1BB047216CD4F8DC3088690B9985
:10D4E000C8EB09086A1C08FB0222984703B0BDE894
:10D4F000F0832DE9F7430A9D84680095174620467E
:10D50000D4F8A86099468846ED1BB047216CD4F842
:10D51000E03088690B99C8EB09086A1C08FB0222F5
:10D52000984703B0BDE8F0830139172924D8DFE814
:10D5300001F01023232323232323230C250E15235B
:10D54000232323232323231F1A210D4870470D482B
:10D55000704703689B68D3F8FC00704703689B68BA
:10D56000D3F8F400704703689B68D3F8F80070475D
:10D5700005487047054870470020704704487047C9
:10D58000DFD8000881D80008E5D7000861D400087A
:10D59000CBD80008013980680D2923D8DFE801F0D5
:10D5A000090B0D0F2222221107252513181D00201B
:10D5B0007047006870474068704780687047C0686F
:10D5C0007047806B704788B1406B00F00100704776
:10D5D00060B1406BC0F34000704738B1406BC0F39E
:10D5E000800070474FF0FF3070470120704783681C
:10D5F00001290CBF586C00207047836800220A8004
:10D600004A801A685B68013A013B8A80CB80704788
:10D61000F0B5104D2E4607460FCE91B06C460FC4A4
:10D6200096E80F00203584E80F000FCD08AC0FC43A
:10D6300095E80F0084E80F007B6B10AA02EB8303D0
:10D6400053F8402CC7F8002153F8203CC7F80431A8
:10D6500011B0F0BD1CF3010807B580698DE8060024
:10D6600003216A46F3F718F903B05DF804FB2DE9CE
:10D67000F74384689846E38C9B078946174632D562
:10D68000D4F8003120469847D4F8045106463A466B
:10D6900020464946A8472369A2699E42ACBF0023A1
:10D6A00001239642D4BF1A4643F0010263699842AF
:10D6B000ACBF134642F00103054613B9E369984233
:10D6C0000ADD62682368013A00920021D4F8A8704C
:10D6D00020460A46013BB847D4F8AC702046314694
:10D6E0002A46B84703E0D4F8AC502046A847D4F8FF
:10D6F000A43020464146984703B0BDE8F083F7B513
:10D700008468E38C9B070F46164645D5D4F8003154
:10D7100020469847D4F8043132460546394620461B
:10D720009847D4F8983006461BB1204601210022C4
:10D7300098472369A2699D42ACBF0023012395420B
:10D74000D4BF1A4643F0010263699E42ACBF134640
:10D7500042F0010313B9E3699E420ADD626823685F
:10D76000013A00920021D4F8A87020460A46013BF5
:10D77000B8472946D4F8AC30204632469847D4F80A
:10D78000A03020469847D4F8983005466BB1204623
:10D7900000210122984708E0D4F8AC302046984791
:10D7A000D4F8A030204698470546284603B0F0BD7F
:10D7B00038B58568044695B94FF4BA7002F0B4FFE5
:10D7C0004FF4BA72A060294600F0C4FDA36802229B
:10D7D000DA8401221A62024A1C64C3F8082138BDA7
:10D7E00011D6000870B506460D461446FFF7E0FF57
:10D7F000B368002B3BD0262D02D0272D16D070BD4C
:10D800009A6B102A02D0122A08D070BD184AC3F8A9
:10D81000D440C3F8B820C3F8B42070BD154AC3F88B
:10D82000D840C3F8BC20C3F8C02070BD9A6B102A42
:10D8300002D0122A0ED070BD3CB10F4AC3F8DC40B2
:10D84000C3F8C820C3F8C42070BDC3F8C840C3F8EB
:10D85000C44070BD3CB1094AC3F8E040C3F8CC20D5
:10D86000C3F8D02070BDC3F8CC40C3F8D04070BD21
:10D87000A1D40008AFD40008BDD40008F3D4000838
:10D8800038B50546FFF794FFAC684FF4FA7002F024
:10D890004BFFA36BA0660733D8102368584302F0F0
:10D8A00043FF01210022E066A869F2F7F5FFD4F8F2
:10D8B00008310546204698472046D4F8B0309847AE
:10D8C000002DD4BF0020012038BD70B504460D46A0
:10D8D0001646FFF76DFFA36883E8600070BD70B562
:10D8E00004460D461646FFF763FFA3689D60DE60A1
:10D8F00070BD38B505460C46FFF75AFFAB68226885
:10D90000DA6262681A63A2685A63520707D593E81D
:10D9100006001A605960DA689968D9609A60A2892D
:10D920009A84226912B122EAE2721A6238BD2DE9A4
:10D93000F04104461F4616468846FFF739FFA568A2
:10D940004146682205F586700AF0FAFF2046B04786
:10D950002046B84723699B689847A862BDE8F081D4
:10D9600010B5074C2368186B00F05EFC00F07CFCDF
:10D970002368586B00F058FCBDE8104000F090BCE4
:10D980002401002037B5094C23685A7C084B054612
:10D9900053F82200C2686946126B904720682946F6
:10D9A0006A46083000F08AFD03B030BD2401002033
:10D9B0009017022037B50D46144602F009F8019081
:10D9C00008B901200CE0C3680A215B6A01A89847E6
:10D9D00003460028F5D001982946224698470020A2
:10D9E00003B030BD37B50D46144601F0F1FF01908C
:10D9F00008B901200CE0C3680B215B6A01A89847B5
:10DA000003460028F5D00198294622469847002071
:10DA100003B030BD37B50D46144601F0D9FF019073
:10DA200008B901200CE0C36810215B6A01A898477F
:10DA300003460028F5D00198294622469847002041
:10DA400003B030BD012810B50C4608DC01F0C0FF62
:10DA500020B1C36821469B6A984710BD10BD0020C5
:10DA600010BD38B5044621460120FFF7EBFF2146E3
:10DA700005460020FFF7E6FFA842B8BF284620EA87
:10DA8000E07038BD0121FFF7DDBF0221FFF7DABFEB
:10DA90000321FFF7D7BF0421FFF7D4BF0821FFF709
:10DAA000D1BF0921FFF7CEBF024B1B68587CFFF79F
:10DAB000E9BF00BF24010020024B1B68587CFFF720
:10DAC000E4BF00BF24010020024B1B68587CFFF715
:10DAD000E8BF00BF2401002008B5044B53F8200024
:10DAE000C36808219B6A984708BD00BF90170220B1
:10DAF00008B501F06DFF20B1C3680221DB6A9847C9
:10DB000008BD08BD024B1B68587CFFF7F1BF00BF82
:10DB100024010020024B53F820301B6958687047DD
:10DB200090170220024B53F820301B691868704789
:10DB3000901702200120FFF794BF0220FFF791BF4A
:10DB40000320FFF78EBF0000024B1860024B1960E4
:10DB5000704700BFF4D70120F0D70120014B1868AF
:10DB6000704700BFF4D70120014B1868704700BF11
:10DB7000F0D7012000283BD030F0010329D030F04D
:10DB8000030328D030F0070327D030F00F0326D04E
:10DB900030F01F0325D030F0FF0324D020F4FF73B2
:10DBA00023F001030BB320F47F6323F00F03E3B1F1
:10DBB00020F4FF4323F07F03BBB1030C1B04A3B18C
:10DBC000830C9B049BB110F07F4F0CBF18202020CA
:10DBD00070470120704702207047032070470420DF
:10DBE00070470520704708207047102070471220AA
:10DBF000704708B5FFF7BEFF01280FD0831E062B24
:10DC000009D9A0F10903072B07D91138102834BF0F
:10DC10002020002008BD082008BD102008BD0000FD
:10DC200070B5084B1B681A7C80EA0201490705D5CC
:10DC30009C6BD96B26680D6825600E6018741046C1
:10DC400070BD00BF2401002008B5024B1B689B6813
:10DC5000984708BD1801002038B5144B1B680A46C8
:10DC6000B3F90A108A4204461EDBB3F90E108A4249
:10DC70001ADCB3F90810884216DBB3F90C1088429D
:10DC800012DC197C587C11F0010F094951F8200071
:10DC900004D0C3682146DB69984738BDC168DB6B97
:10DCA0008D691B682146A84738BD00BF24010020AC
:10DCB0009017022038B5104B1C68B4F90A3099420D
:10DCC0000D4617DBB4F90E30994213DCB4F9081095
:10DCD000B4F90C308842A8BF01469A42B8BF134637
:10DCE0008B4207DB607C054A52F82000C2689468CA
:10DCF0002A46A04738BD00BF24010020901702200B
:10DD000038B5104B1C68B4F9083005469D421046E2
:10DD100017DBB4F90C309D4213DCB4F90A20B4F9D6
:10DD20000E309142A8BF0A469842B8BF03469342BC
:10DD300007DB607C044951F82000C168CC682946A3
:10DD4000A04738BD240100209017022073B50E466D
:10DD500012490C68B4F90810B4F90C508842A8BFF5
:10DD60000146AA42B8BF15468D4214DBB4F90A2019
:10DD7000B4F90E009642A8BF32468342A8BF0346BC
:10DD8000934208DB647C064850F82400C468009382
:10DD900024692B46A04702B070BD00BF24010020BB
:10DDA000901702202DE9F04FDFF8ACC18FB0DCF8FE
:10DDB00000C009900E4615469B461C9CDDF87880F5
:10DDC000BCF1000F0DD0189D199E009501961A9F69
:10DDD0001B9D1D9E0297039504940596DCF8004058
:10DDE00053E0189F199847EA0003012B4FD1584B75
:10DDF0001868B0F90A20511A002908DDC1EB0B039D
:10DE0000002B40F3A2801B9F07FB014401E05B460F
:10DE100032465E44B0F90E10013E761A002E03DD44
:10DE20009B1B002B40F391800999B0F90C602944A9
:10DE30000139891B099E0029C8BFC1EB0505C8EB44
:10DE40000601B0F90860B1420CDAC1EB060C08EB30
:10DE50000C078E1B2CF0070C354404EBE7046144DF
:10DE600007F00708002D70DD467C3A481A9F50F8ED
:10DE70002600C668019703941B9F1D9C0093029780
:10DE8000CDF81080059474682B46A0475DE01A9F7A
:10DE9000C7F108070C976746DC4556DA2C4B1998F2
:10DEA0001B683044B3F90A200A90411E91420B913D
:10DEB00045DBB3F90E309E4241DC4FF00008DDF83F
:10DEC00024900894C246AA4539DAB8F1000F05D16A
:10DED000089A1778013208924FF008080C981A999E
:10DEE0001B4A47FA00F3C1EB08088F4013F0FF010B
:10DEF000FFB203D11068007C80071BD41268D26B7C
:10DF000010680D901D9810B150F8213000E0DBB280
:10DF1000189913604A1E4A440B9BCDF81CC0484612
:10DF20003146FFF713FF0A4B0D9A1B68DDF81CC042
:10DF3000DB6B1A60189B0AF1010A9944C3E71B9E28
:10DF40000CF1010C34440A9EA6E70FB0BDE8F08F37
:10DF50002401002090170220641702202DE9F04FC1
:10DF6000DFF80CC291B0DCF80090079205468846B5
:10DF70009B461C9E1E9CB9F1000F0CD01A9D1B9F46
:10DF8000009501971D9D1F9F029603950494059788
:10DF9000D9F8004081E01A9F1B9847EA0003012B43
:10DFA0007DD1714B1868B0F90A20531A002B08DD97
:10DFB000C3EB0B01002940F3D4801D9F07FB0344F2
:10DFC00001E059464246D844B0F90E3008F1FF3816
:10DFD000C3EB0808B8F1000F04DDC8EB010100290C
:10DFE00040F3BF80079BB0F90CC02B44013BCCEB46
:10DFF0000303002B02DD079FFF1A0797B0F908C043
:10E00000654533DA079FC5EB0C03FF1A082E079707
:10E0100027D00DDC022E14D0042E1AD0012E26D1CA
:10E0200023F0070C04EBE304654403F007031EE050
:10E03000182E18D0202E16D0102E18D104EB430421
:10E0400013E023F0030C04EBA304654403F0030383
:10E050000DE023F0010C04EB6304654403F00103BD
:10E0600005E01C4401E004EB830465460023079FA0
:10E07000002F76DD90F811E03C481D9F50F82E00EF
:10E08000D0F80CE003948DE842001F9C04930297A3
:10E090000594DEF80440079B2946A04761E0C6F1DD
:10E0A00008070E97CDF828900A9F5F4559DA2E4B46
:10E0B0001B9F1B684744B3F90A200C97013F974206
:10E0C0000D9746DBB3F90E30984542DC4FF0000A5D
:10E0D0000B94AC465746079887423ADABAF1000FDC
:10E0E00006D10B9890F8009001300B904FF0080A81
:10E0F0000E991D4A49FA01F313F0FF0109FA06F9D6
:10E100005FFA89F9C6EB0A0A03D11068007C800720
:10E110001BD41268D26B10680F901F9810B150F882
:10E12000213000E0DBB21A9913604A1E6244604657
:10E130000D9BCDF820C04146FFF708FE0A4B0F9A11
:10E140001B68DDF820C0DB6B1A601A9B01379C440A
:10E15000C1E70A9FDDF8308001370A971D9F3C44D4
:10E16000A2E711B0BDE8F08F240100209017022033
:10E170006417022008B5054B1968054B4A7C53F813
:10E180002200C36808311B6B984708BD240100209A
:10E190009017022037B5FFF7EDFF04F02DFF04467E
:10E1A00000283DD10546284601F012FC019048B1F7
:10E1B000C3680C215B6A01A89847034670B30198B5
:10E1C000984704430135022DEDD14CBB04F030FFDC
:10E1D0000124204601F0FCFB0190D0B1204600F064
:10E1E000A1FE0420FFF730FD43F6FF720020014638
:10E1F0001346FFF7ABFD0020FFF726FD02A80E2116
:10E2000050F8043DDB685B6A9847034608B1019803
:10E21000984714F1FF34DCD2002002E0012000E036
:10E22000204603B030BD000008B5054B1B685A7C82
:10E23000044B53F822301B691B68984708BD00BF88
:10E24000240100209017022008B5054B1B685A7C5A
:10E25000044B53F822301B695B68984708BD00BF28
:10E260002401002090170220044B1B681A7C5207DF
:10E270004CBF9B6BDB6B1860704700BF2401002014
:10E2800008B5064B1B68196B814206D01863FFF76F
:10E29000CBFFBDE80840FFF7E7BF08BD2401002021
:10E2A000044B1B681A7C52074CBFDB6B9B6B1860DE
:10E2B000704700BF2401002008B5064B1B68596B4E
:10E2C000814206D05863FFF7AFFFBDE80840FFF773
:10E2D000E7BF08BD2401002008B5024B1B685B683E
:10E2E000984708BD1801002008B5024B1B681B6841
:10E2F000984708BD1801002070B5840702D5018039
:10E30000013A023055082B4605B3032D01EB0144B9
:10E3100002DC06461D4612E003462E46043E032E4E
:10E320001C605C609C60DC6003F11003F6DC043D63
:10E33000AB085E1C00EB0610A5EB8303E9E71DB1FB
:10E3400046F8044B013DFAE700EB8300D30748BFD2
:10E35000018070BD70B52AB1830703D000F8011B9E
:10E36000013AF8E7930801D1024417E04FF0013475
:10E3700002F003024C43032B054606DD04604460B3
:10E380008460C460043B1030F5E71E461BB145F8BD
:10E39000044B013BFAE700EB8600E5E7904202D030
:10E3A00000F8011BFAE770BD0B8892B2134403809A
:10E3B0008B889B1A83804B8813444380CB889A1A9E
:10E3C000C28070470128F7B504460D4665DC344B22
:10E3D0001B6803B19847012D04D0022D21D0002DD8
:10E3E0005BD135E02F4E56F82470B7B9204601F0C6
:10E3F000EFFA0190002850D0C3680D215B6A01A894
:10E4000098470346002848D001982946984756F86F
:10E410002430013346F8243018E0013746F82470E0
:10E420003BE0204601F0D4FA0190002835D0C368C3
:10E430000D215B6A01A89847044600282DD01A4B8D
:10E440001B6803B1984701980221A047002025E0EE
:10E45000144D55F82430012B01D0012015E0204641
:10E4600001F0B6FA01900028F7D0C3680D215B6A6D
:10E4700001A8984706460028EFD00B4B1B6803B154
:10E48000984701980021B047002055F82430002B10
:10E4900018BF013B45F8243000E0012003B0F0BD77
:10E4A00004D80120FCD70120F8D70120024B1B68BB
:10E4B0000146587CFFF786BF2401002070B5B2F9F1
:10E4C0000030B1F90040B1F90250B1F90460B1F97E
:10E4D00006109C42B8BF1C46B2F902309D42A8BF4C
:10E4E0002B46B2F90450B2F90620AE42B8BF354609
:10E4F000A4B2ADB29142B8BF0A460480858024B26E
:10E500002DB29BB292B2A5424380C28006DB10B20C
:10E510001BB29842B4BF0020012070BD002070BD26
:10E520000B8810B5B0F900401AB29442B8BF03800E
:10E530004B88B0F902401AB29442B8BF43808B882E
:10E54000B0F904401AB29442C8BF8380CB88B0F9B6
:10E5500006101AB29142C8BFC38010BD01F07F43BC
:10E56000B3F17F4FF0B527D0D343DBB2CDB2C6B203
:10E570005D4302FB065501F47F4600F47F445E4391
:10E5800002FB046601F47F0400F47F075C43090E7C
:10E59000000E02FB07444B43360A02FB0032240AFA
:10E5A000C5F3072306F47F401843120404F47F03E5
:10E5B000184302F07F421043F0BD000070B50A4CD2
:10E5C0000A4D20680A4E01F043FF286801F040FF21
:10E5D000306801F03DFF074A00231360064A3360AC
:10E5E0002B602360136070BD0CD8012008D8012077
:10E5F00010D8012014D8012024D801202DE9F84397
:10E600001C46284B17461A680646884632B901222E
:10E6100025481A60254B036001F00EFB244D2B6842
:10E6200033B9244B1B682B6013B9FFF789FA2860B4
:10E630000CB12B68236096B11F4B1A6899460024D1
:10E640004AB92868800002F06FF8D0F10104C9F8D7
:10E65000000038BF0024D9F80030336000E03446B1
:10E66000B8F1000F0DD0154E33683BB92868800013
:10E6700002F05AF80028306008BF01243368C8F857
:10E68000003067B10E4E33683BB92868800002F055
:10E690004BF80028306008BF012433683B602046F7
:10E6A000BDE8F88324D801201CD80120BDE500086E
:10E6B00014D80120981702200CD8012008D8012076
:10E6C00010D801202DE9F04F93B000241D9E0B902F
:10E6D0000C9190461F4634600FA810A9224611AB3A
:10E6E000FFF78CFF0546002840F0C380634C119A69
:10E6F0002368587C624B53F8203007939742A8BF99
:10E7000017461A690D920A97FFF7E6F923680890F1
:10E71000587CFFF7FFF95B4B0490984205D05A4BA9
:10E72000C31A18BF0123069300E0069500250A9C32
:10E73000AB4643461C9A53F8040B05939047030ECF
:10E740008146099300F08580BBF1000F3FD14B4B10
:10E750000B9F1B680A9AB3F90830DDF82CC00C999E
:10E760002F44BB42C8BFC7EB030B0BEB050AC8BF66
:10E770001F460F9B4FEA8A0A534494440093079B19
:10E7800001930CF1FF3238460B46CDF80CC004F073
:10E79000F9FB089A0F98DDF80CC0172A06DC5044E4
:10E7A000CBEB04010D9B04F093FC01E0069B13B935
:10E7B0004FF0010B0BE0C7EB0C078244DAF80000C6
:10E7C000049A9047013F4AF8040BF7D1F0E72F4B2A
:10E7D0000F99D3F800C0109F4FEA850ABCF1000FD3
:10E7E00024D007EB0A025144109223460F91404671
:10E7F000E0470F9D109A002358F8031001F07F4066
:10E80000B0F17F4FE85801D1D05005E000F07F40D3
:10E81000B0F17F4F08BFD150013C03F10403EBD1AD
:10E820003368109743F00103336020E0099BFF2B0E
:10E8300004D151F80A3047F80A3011E0099B51F829
:10E840000A10DA434846D2B2FFF788FE47F80A00BA
:10E8500002E0109B43F82500336843F00103336066
:10E86000013C05F1010502D0DDF8148061E7109844
:10E8700000E0204613B0BDE8F08F00BF2401002067
:10E8800090170220CF0B0108CD0B010818D80120EA
:10E890001FB508B103AA00E0024601A802A900239F
:10E8A000FFF7ACFE05B05DF804FB000008B5024BB5
:10E8B0001B6803B1984708BD28D80120B5EEC00AEF
:10E8C000F1EE10FADFED0D7A48BFB1EE400A30EEFE
:10E8D000270A0020B5EE400AF1EE10FA0CD0F2EE55
:10E8E000047A20EE270A0130FCEEC07AC0B217EE9F
:10E8F000903A002BF3D07047704700BF5F708930AB
:10E90000B5EEC00AF1EE10FA08B5F6EE007A0AD5B7
:10E9100070EE677A17EE900A08F022FC41EC100BBB
:10E9200007F0BAFB09E070EE277A17EE900A08F0BC
:10E9300017FC41EC100B07F02FFC51EC100B08F00A
:10E94000EFFC00EE100A08BD0E4B53F8213007EE25
:10E95000903AF8EE677A70B520EE270A05460C4625
:10E960001646FFF7CDFFBDEEC00A294610EE100A8D
:10E9700022461EB1BDE8704000F0AEB8BDE8704060
:10E9800000F09DB8E8F4010838B5B5EE400AF1EEA4
:10E9900010FA2DED028B0446B0EE408A0D4652D09F
:10E9A000B5EEC00AF1EE10FA24DBF7EE008AB4EE01
:10E9B000E80AF1EE10FA1DD5FFF780FFA04202DC55
:10E9C00078EE287A46E0F6EE007AB4EEE78AF1EEC9
:10E9D00010FA09DBDFED367A002C18BFF0EE687A0A
:10E9E00008BFB0EE688A35E044B3F0EE687A9FED78
:10E9F000308A2FE0B5EEC08AF1EE10FA28D5FFEE8E
:10EA0000008AB4EEE88AF1EE10FA21DDB0EE480A91
:10EA1000FFF754FFA04204DCF7EE007A78EE677A45
:10EA200018E0FEEE007AB4EEE78AF1EE10FA03D8B1
:10EA30004CB9B0EE688A0BE044B104E0DFED1C7A1B
:10EA4000B0EE678A06E0F7EE007A03E09FED188AE1
:10EA5000F0EE487A174B53F8243000EE103AB8EE37
:10EA6000400A27EE800AFFF74BFFBDEEC00A10EE0A
:10EA7000100A01F061FF012DC4EB000020EAE070F4
:10EA800005D1B5EEC08AF1EE10FAC8BF0130B0EE84
:10EA9000480ABDEC028B002C0CBF2346631C1844B3
:10EAA00021462A46C0B2BDE83840FFF74DBF00BF3F
:10EAB00000000000E8F401080021FFF765BF1FB562
:10EAC00004AB01AC43F8104D6B4601F059FF2046F2
:10EAD00000F0FAFE04B010BDF0B585B004AC0D46F0
:10EAE00001AE6946174644F8106D01F03DFF00285D
:10EAF000C4BF05F1FF35EDB229463A466B4601F039
:10EB00003FFF304600F0E0FE05B0F0BD034A0023B1
:10EB10001360034A1360034A136070472CD8012026
:10EB200030D801203CD801202DE9F043194B1F6853
:10EB300085B000259846D8F80030164C33B300F065
:10EB400091F90646206801F097FC034604A859692C
:10EB500040F8103D891B002913DC216803910196C0
:10EB600019695E68029168462660D3F8009001F04A
:10EB700091FC01A8C8474EB12368BB4205D00125CE
:10EB8000D9E7684601F086FC00E00025284605B07C
:10EB9000BDE8F08330D80120F0B5254C85B005469E
:10EBA00001F06AFC2368019013B92560436039E0E5
:10EBB000184601F061FC04AB466943F8100D684645
:10EBC00001F068FC019B5A69921B002A03DC226851
:10EBD0005A60256026E02668304601F04DFC04AC02
:10EBE000466844F8080DBEB1304601F045FC04AB60
:10EBF000476943F8040D184601F04CFC019A53692B
:10EC0000DB1B002B029B02DC56605D6007E02046A8
:10EC10005E6801F03FFCDFE7019B5E6045602046D7
:10EC200001F038FC01A801F035FC05B0F0BD00BFD3
:10EC300030D8012037B50546F0B101F01DFC0F4B6F
:10EC400000901C68AC4204D142681A6011E001F0E7
:10EC500021FC74B1204601F00FFC034602A85C6859
:10EC600040F8043DAC42F2D1009A52685A6001F07B
:10EC700011FC684601F00EFC03B030BD30D8012015
:10EC8000002337B50360094B1C68054654B1204684
:10EC900001F0F2FB02AB026943F8040D2A6018464A
:10ECA00001F0F8FB204603B030BD00BF2CD8012096
:10ECB000002373B50B600E46044690B101F0DCFBF7
:10ECC00002AD846845F8040D44B1284601F0E2FB2A
:10ECD000204601F0D1FB036901903360284601F022
:10ECE000D9FB204602B070BD2DE9F74381461C20B8
:10ECF0000E4690461F4601F091FE0446002831D092
:10ED00001A4B1B4A1A6001F0B7FB009016B900F0CD
:10ED1000A9F8064602A850F8085D68466E61C5F875
:10ED20000090C5F81080AF8101F0B4FB2046FFF7DA
:10ED300033FF104B1A6832B901220F481A600F4B8B
:10ED4000036000F079FF204601F096FB0C4A019029
:10ED5000136813B91460836001E08360146001A834
:10ED600001F098FB204603B0BDE8F0837417022041
:10ED700029EB00083CD8012034D801200DEB000815
:10ED80002CD8012073B5044658B3174D2E6886421F
:10ED90000BD101F071FB02AB826843F8040D2A60CD
:10EDA000184616E0684601F075FB304601F064FB3A
:10EDB000866802ADA64245F8080DF3D1204601F061
:10EDC0005BFB009B826801909A6001A801F062FBE6
:10EDD000684601F05FFB2046FFF72CFF204601F05C
:10EDE00085FB02B070BD00BF2CD8012013B50C46C6
:10EDF00040B101F041FB02AB846143F8040D1846B9
:10EE000001F048FB02B010BD13B5044698B101F003
:10EE100033FB019000F026F802AB53F8042D916902
:10EE200008445061184601F035FB2046FFF702FF09
:10EE30002046FFF7B1FE02B010BD13B50C4668B115
:10EE400001F01AFB02AB828943F8040D1442184604
:10EE50000CBF0024012401F01DFB00E0012420462A
:10EE600002B010BD05F016BB034B1B68B3F92A2096
:10EE700058851046704700BF24010020034B1B68D3
:10EE8000B3F92C2098851046704700BF240100205C
:10EE9000024B1B689A7E987610467047240100202A
:10EEA000034B1B68D96900B1D8610846704700BFA1
:10EEB00024010020FEF7C8BE08B5002000F01CF8B1
:10EEC0006FF07F4000F01AF8012000F07DF800207C
:10EED000FFF7D4FF0020FFF7C7FF0020FFF7EAFF8E
:10EEE000044B1868FFF7DCFF0020BDE80840FFF77F
:10EEF000CFBF00BF28010020FFF7EEB9FFF7F4B93C
:10EF000010B5074B1C7820B101221A704FF0FF306A
:10EF100002E018706FF07F4004F0C8F8204610BD82
:10EF20008117022070B5084D2B68012804465E7CCD
:10EF300008D800F04DFD28B12B685C7400F008F88B
:10EF4000024B1C60304670BD2401002034170220A3
:10EF500008B503F003FFFEF703FDBDE80840FCF72A
:10EF6000A5BB000008B5034B7022196809F0E8FC46
:10EF700008BD00BF2401002008B5034B01467022E4
:10EF8000186809F0DDFC08BD24010020B0F902205A
:10EF9000B1F906309A4214DCB1F90220B0F906301A
:10EFA0009A420EDCB0F90020B1F904309A4208DC34
:10EFB000B0F90430B1F900209A42CCBF0020012002
:10EFC0007047002070470000024B1B681A7E1876BD
:10EFD0001046704724010020024B1A6802B91860DD
:10EFE000FFF764BC40D801200A4A0B49136809683E
:10EFF0008B4210B50BD0094CA34293E8030014BF19
:10F000000833503B136002F02FFB012010BD00209D
:10F0100010BD00BF200100201C01002094D8012059
:10F0200068B1038889B20B440380838819444388FC
:10F03000818092B213444380C3881A44C2807047CF
:10F0400010B538B309B30AB3B1F90040B2F90030D2
:10F050009C42B8BF23460380B1F90240B2F90230A6
:10F060009C42B8BF23464380B1F90440B2F9043052
:10F07000B1F906109C42A8BF23468380B2F906303E
:10F080009942A8BF0B46C38010BD11460B680360B0
:10F090004B68436010BD0000054B1B68002B18BF78
:10F0A0000020044B0129B8BF01211954704700BF4B
:10F0B0009CD8012060170220024B1B685884998459
:10F0C0000020704724010020044BB3F90030036096
:10F0D000034BB3F900300B60704700BF7817022074
:10F0E0006C170220014B1B68987E7047240100209A
:10F0F00003F0E4BF0A4B10B51C681CB1A047041C08
:10F1000018BF0124FCF724FA064B1B68002818BF1F
:10F1100001241BB19847002818BF0124204610BDC8
:10F12000741702208C17022010B50024FFF7E2FFAD
:10F1300008B10124FAE7204610BD00000F4B73B55B
:10F140001B68DE6C1C6D06440D19B3B2144468468E
:10F15000ADF80030ADF80430ADF80250ADF806401F
:10F16000FCF7C2F838B1304629462246FEF7C8FD02
:10F17000FBF7F8FFF6E702B070BD00BF24010020E6
:10F180001E4B1B689B7E013B032B32D8DFE803F04C
:10F19000020D1A221A4B06300340002B03DA013B02
:10F1A00063F00F0301330B2B08E0164B0340002BD9
:10F1B00003DA013B63F003030133012BCCBF0020D2
:10F1C00001207047142390FBF3F203FB12000B287D
:10F1D00009DC10E0182390FBF3F203FB12000B286C
:10F1E00009DD20F00400103801288CBF0020012028
:10F1F0007047002070470120704700BF24010020A5
:10F200000F00008003000080C0F30B00B0F5006F1A
:10F21000C6BFA0F5006001210021B0F5806FC8BF16
:10F22000C0F5006000F03F0310B582110B4CC3F134
:10F2300040039BB234F81200402B00FB03F008D0CF
:10F24000102A06D00132C3F1400334F8122003FB28
:10F2500002002030800901B1404210BD9CF4010839
:10F2600000F58060FFF7D0BF2DE9F74FDDF8308063
:10F27000171A5C1A54EA070C05460E46D8F800B077
:10F2800004D103B0BDE8F04F04F000BB87EAE7709B
:10F29000A0EBE77084EAE471A1EBE471884204DB3F
:10F2A00021463C460F46002106E011461A460B4611
:10F2B000294635460E460121009184EAE471A1EB0E
:10F2C000E4718C4208D01E462B46644215467F42AC
:10F2D0001A464FF0FF3A01E04FF0010A002FDFF825
:10F2E00048913ED1009BD3B1D9F800309B7E8BB9B9
:10F2F0003046294603B0BDE8F04FFEF701BDFFF7E9
:10F300003FFF30B9D9F800305B6E30465B68791941
:10F3100098470137A74207EB0B00F0DD1DE0D9F855
:10F320000030997E11B1DDF800A012E05B6E284636
:10F330001B683146984774E0FFF722FF38B9D9F8C7
:10F3400000305B6E0AEB05005B68314698470AF1B6
:10F35000010AA2450AEB0B00EEDD0138C8F80000F7
:10F360005FE0D9F800104FF00202897E94FBF2F2C0
:10F37000B8BF5242D9B99346A846C5EB0803A34289
:10F380004FDC009B9BFBF4F131442BB9D9F80030E2
:10F390005B6E40465B6805E0D9F800305B6E5B68E9
:10F3A00008464146984708F10108BB44E5E7BAF131
:10F3B000FF3F04BF04EB0B01C8F800100192AB46FD
:10F3C000C5EB0B01A142D8F800001EDC5044C8F880
:10F3D0000000FFF7D5FE80B9DDF804C0D9F80000C1
:10F3E000009B406E9CFBF4F1314413B943685846CE
:10F3F00002E04368084659469847DDF804C0BC441B
:10F400000BF1010BCDF804C0DAE7BAF1FF3F04BFFE
:10F410002418C8F80040D8F80020CAEB0203C8F846
:10F42000003003B0BDE8F08F240100202DE9F04F3B
:10F43000674D2C6894F818B0BBF1010F87B0814676
:10F44000884617461E46AA4604D1109C0094FFF732
:10F450000BFFBAE0841ACD1A54EA050300F0B58018
:10F46000002CBABF644201230023002DBCBF6D42B3
:10F4700043F00203A5420BF1FF3B04DD224643F0BB
:10F4800004032C461546022294FBF2F202EB85257A
:10F4900095FBF4F4A1114F4AC4F38304C4F11005A1
:10F4A00032F91100102D05FB00F004D0013132F9C2
:10F4B000112004FB02001022083090FBF2F05907E3
:10F4C00048BFC0F58060DA0748BFC0F500609B0701
:10F4D00048BFC0F5805000F580652846FFF7C0FEA4
:10F4E00000FB0BF42846FFF78FFE002C00FB0BF00F
:10F4F00004DAC4F500739B125B4202E004F500736A
:10F500009B12002806DAC0F5007B4FEAAB2BCBF14B
:10F51000000B03E000F5007B4FEAAB2B002B03DD73
:10F52000581C40105B1005E0022293FBF2F0013BF7
:10F5300093FBF2F3BBF1000F05DD0BF1010252105A
:10F540004FEA6B0B06E002219BFBF1F20BF1FF3B54
:10F550009BFBF1FB80B21FFA89F4011992B2ADF85E
:10F5600008101FFA8BFB1FFA88F15518CBEB01012D
:10F570009BB2ADF80E10B9B2E41ACB1AADF8103048
:10F58000B3B20144CBEB030B13440022ADF81410CB
:10F59000ADF8163002A813460421ADF80A50ADF8B4
:10F5A0000C40ADF812B004F08FF8DAF800305B7E52
:10F5B0001BB94846414604F069F9DAF800305B7E31
:10F5C0001BB93846314604F061F907B0BDE8F08F49
:10F5D00024010020BEF4010830B585B004AC00253C
:10F5E00044F8045D0094FFF721FF05B030BD000032
:10F5F0002DE9F8431E460C4B1C6881460020E56C43
:10F60000246D88461746FBF76FFE50B109EB0500E5
:10F6100008EB04017A193319FFF7DEFFFBF7A2FDAF
:10F62000F3E7BDE8F88300BF24010020F7B5104FD1
:10F630003B681D6DDC6C05440E19ABB21444684682
:10F64000ADF80060ADF80440ADF80230ADF806301A
:10F65000FBF74AFE48B13B685B6E30461B682946A3
:10F6600022469847FBF77EFDF4E703B0F0BD00BFEC
:10F67000240100202DE9F04F9846814B8BB08A463B
:10F680001968069000209146149F159ECD6C0C6D54
:10F69000FBF72AFE002800F0EF800AF100430698ED
:10F6A000013B00EB43030793169B002B14BF6FF045
:10F6B00001030223A9444444099327B9FBF752FDEF
:10F6C0000028FAD1D8E0002EF8D0BAF1000FF5DD0D
:10F6D0007B1C04D1012E14BF022301230AE0012F59
:10F6E00004D1012E14BF0323002303E0012E14BF15
:10F6F000052304230593624B1B685B69EBB1B3F9E7
:10F700000080B3F90200B3F90420B3F906B0049005
:10F7100008F1FF38C14509EB0A03B8BFC9EB080877
:10F7200003F1FF33B4BF28EAE8784FF000089342B2
:10F730000ADDC9EB0202013207E04FF0FF3B5246FF
:10F74000CDF810B0984600E05246169B1BB9069BB8
:10F7500003EB480300E0079B90450393AEDA4A446D
:10F7600008920022C844012302920398099905884F
:10F7700008442DB247F6FF718D4203900DD10298D7
:10F7800000286FD1002B6FD1114608F1FF30019294
:10F79000FEF762FA0123019A67E00598411EDBB18A
:10F7A000042917D8DFE801F00305070B0F00621BDF
:10F7B0000EE0651B00E02544B5FBF6F208E02544A9
:10F7C00007FB05F204E0254407FB05F2B2FBF6F265
:10F7D00000234AE02A19FBE7042912D8DFE801F0E8
:10F7E0000305070B0E00651B0CE0651B00E02544BC
:10F7F000B5FBF6F506E025447D4303E025447D4353
:10F80000F6E7254404998A4201DA8D4225DB5A4500
:10F8100001DD5D4521DC05EB020C0221AA429CFBC7
:10F82000F1FC08F1FF300BDC114662468DE8081050
:10F83000FEF766FADDF804C0404661462A4609E054
:10F8400061468DE80810FEF75BFADDF804C040461B
:10F8500029466246FEF754FA009B029A0132029250
:10F860002A4602E0002302930123089808F10108C8
:10F8700080457FF47AAF21E70BB0BDE8F08F00BF81
:10F8800024010020F8B50B4B1B680546B3F92C008A
:10F8900040F002000F461646FFF7F0FA39460446DC
:10F8A0003246284600F008F82046BDE8F840FFF749
:10F8B000E5BA00BF24010020024B1B6859849A84DA
:10F8C00000F002B8240100202DE9F74F044600287B
:10F8D00079D03E4D00F0B4FC2B688046B3F82290FE
:10F8E00000F096FC2B689A8C87B2D21B9A842378FE
:10F8F000002B5DD047F6FF71204600F0D7FB06468F
:10F900003146204600F000FC2B689A8D02F003027D
:10F91000012A05D0022A14BF002290FBF2F200E077
:10F920000246598C8A1A92B291B259841FFA80FA0F
:10F930009B8CADF800100AF1FF310A44ADF802309B
:10F940001FFA88FB013B5B44ADF80420204631469A
:10F950006A46ADF8063000F007FC2B68BDF80220BF
:10F960009A842046314603F029FE235C0A2B04EBDF
:10F97000000201D00D2B12D12B68998D01F00301EB
:10F98000013901298ABF198CA3F822905984117872
:10F990000A290BD1998C8B44A3F824B006E00B4BB9
:10F9A000BDF800001B688244A3F822A0137843B975
:10F9B0002B689A8C17449A8D9F8422F003029A85B3
:10F9C00001E0541C93E703B0BDE8F08F2401002050
:10F9D000012809DC054B53F8200020B1C3681B68DF
:10F9E0001BB10068F9E770470020704790170220AC
:10F9F00000F02EBD012BF8B506460D4617461C46F5
:10FA000001DD0020F8BD1C2000F08EFE0028F8D09B
:10FA10000DB1056109E0094B53F8241029B10B68B9
:10FA20000BB11946FBE70B69036100238360846116
:10FA30008782C66003604360F8BD00BF9017022054
:10FA4000094B826953F82210814204BF016843F8D0
:10FA5000221043680BB102681A60026802B1536059
:10FA600000230360436070479017022070B538B3DD
:10FA70008269012A24DC194951F822300D4613B954
:10FA800041F822001AE0596809B10B46FBE7C1684A
:10FA90000E68D9680C68B44203DD1B68002BF8D1EE
:10FAA0000EE002D1818A012911D0596899B108600C
:10FAB00041605860984208BF00230360002070BD79
:10FAC000012070BDCB681B68A3420B46EDDB1968B3
:10FAD0000029F7D1E9E745F82200EAE7901702206C
:10FAE00038B51D46FFF786FF044648B1FFF7BEFF55
:10FAF000E3681B6823B9034B16351B6843F82540A0
:10FB0000204638BD2401002010B5074B07480024CB
:10FB1000214670221C60FEF71DFC21460448082285
:10FB2000BDE81040FEF716BC1CD90120A4D8012066
:10FB30009017022038B5194D2B681A1DDA6303F1AE
:10FB400008029B631B6442615A7C154B044653F8C0
:10FB50002200C36804F108011B6B9847114B6366D0
:10FB6000114B1B68E3612B68083363610123237623
:10FB7000FAF76EFC032384F868306FF07043236358
:10FB80006363A0640020FEF7A7FB6FF07F40FEF7E1
:10FB9000ABFB064B064A1A6038BD00BF24010020AB
:10FBA00090170220E0F401082801002088170220A5
:10FBB000CC1502082DE9F347074604209A460E4665
:10FBC0009146FEF741F8134B1C68E56C246D2F44F9
:10FBD000264480464D4454446846ADF80070ADF864
:10FBE0000450ADF80260ADF80640FBF77DFB28B984
:10FBF0004046FEF729F802B0BDE8F08738463146A6
:10FC00002A462346FEF7A2F8FBF7ACFA0028F5D106
:10FC1000EEE700BF2401002010B500200146FFF7E9
:10FC20004BFA044843F6FF7201461346BDE8104004
:10FC3000FFF7C0BF01C0FFFF80B483B000AF7860A2
:10FC4000054B1A687B685A60034B7A681A600C3758
:10FC5000BD465DF8047B7047A0D8012008B5084B6D
:10FC60001A6862B901221A60F0F714FDF0F73CFD42
:10FC70000448054B0360BDE80840FFF7DDBF08BD41
:10FC80001CD9012014D9012009FB000890B583B0CC
:10FC900000AF204B1F4A126822F001021A601E4B6F
:10FCA00001221A601D4B1E4A1A601C4B1A681D4B1C
:10FCB0009A4200D0FEE7FFF7D1FF1B4B2E221A70AD
:10FCC00004F0EAFB1948FFF735FFFEF763FA7860A6
:10FCD000FDF744FF0346002B04D0FDF745FF034624
:10FCE000002B09D1FDF726FF0446FDF726FF03464A
:10FCF00020461946FDF728FF0020002103F070FC84
:10FD0000FBF73EFD0A4B01221A707B6818460C3740
:10FD1000BD4690BD002000E00830024000300240A7
:10FD2000C2A507F4CDB5E8B562170220A4D801201A
:10FD30008017022038B103888B4202D843888B4257
:10FD400001D28068F6E770472DE9F04F384C236800
:10FD5000B3F92A90DB69054689B0D8692946FFF7CF
:10FD6000E9FF002861D0B0F800804768C8EB0508BB
:10FD700007EBC806484696F802B0FDF765FF256810
:10FD800017F83820D5F81CE0B5F924109EF81AC0F1
:10FD90009EF8183006938246B5F92200CDF800C0CF
:10FDA0009EF81BE0CDF804E04FF0010ECDF80CB04A
:10FDB000CDF808E073680493AD6B069B0595FEF7DC
:10FDC000CDF82368DA6992F819B0117E8B4520D9F5
:10FDD000B9F1020FD57E1CD0079103F04DFC81468E
:10FDE00003F043FCFFF78AF8246817F83870E269DB
:10FDF000B4F92430B4F92200D27E079907FB02023D
:10FE000001FB05310BFB0533FDF7A0FF4846FFF76B
:10FE100075F85046FDF718FF054B1B68DA69598CD9
:10FE2000907E727800FB02125A8409B0BDE8F08F10
:10FE3000240100200D4B70B51B68DD6906460C4699
:10FE4000E8693146FFF776FF70B103884268F61A19
:10FE500002EBC6035878AB7E10FB03F024B112F816
:10FE6000362012FB03F3236070BD00BF2401002085
:10FE700001230B80704708B5C069FFF75BFF0030B6
:10FE800018BF012008BD0000524B2DE9F04F1B6840
:10FE9000D9695F8CCC699D8CA28990428BB008D3C4
:10FEA000E689864205D3D4F80090821A4FF0FF3BD2
:10FEB00015E0A268D4F80490002A00F0818016882A
:10FEC000B0427DD3B2F802C0844579D35268801B1A
:10FED00080B202EB800632F92020B6F902B0501C45
:10FEE0006ED091F81880A17CB3F82AA0267C0692E7
:10FEF00018FB01F107910FFA8AF108460891FDF706
:10FF0000A3FE344909900B68069AD969887E00904F
:10FF1000C97E019101210291A17C0391079901FB06
:10FF2000029204929B6B05933FB22DB2384629464C
:10FF300032464346FEF712F8BBF1FF3F1BD04AF0B2
:10FF4000020000B2FDF780FE224A1368DA69917E52
:10FF50000091D27E0192012102910799A27C039225
:10FF600001FB0B9204929B6B05933846294632465F
:10FF70004346FDF7F3FFDFF85C80D8F80030DB691B
:10FF80005A7E1B7E9A4217D9089A022A14D08AF008
:10FF9000040000B2FDF758FED8F80030DB6993F892
:10FFA00018E0D97E9A7E5B7E38460EFB015106FB37
:10FFB00002722B44FDF7CAFE099BD8B2FDF744FE3E
:10FFC000044B617C1B685A8C0A445A840BB0BDE810
:10FFD000F08F00BF24010020044B1B68DB69DB6944
:10FFE00009B11A7C0A60587C704700BF24010020C8
:10FFF00002230B807047C3699A898A4202D8DA8942
:020000040801F1
:100000008A420FD2986880B1038899420CD3428803
:100010008A4209D3C91A426832F82100C043C0F3AA
:10002000C0307047012070470020704770470000C3
:1000300037B5154602AB1A4A43F8081D01901268FD
:10004000184C6946904723680190586958B90120B7
:10005000FEF72CFA2368DB695B69BBB19B680198EA
:100060000099984717E02946FEF790FF0028EED147
:1000700014E001A803F08EFA2368DB691B680546CB
:100080009847094B1B680BB128469847009B013BDA
:10009000002B0093EDDA0020FEF708FA03B030BD24
:1000A0002C010020240100207C17022037B50D46CA
:1000B0000190044698B10B4B1B68DB695B690BB17F
:1000C0005B680BB9002408E0984709E001A803F039
:1000D00061FA20B10A2802D00134AC42F6DB204696
:1000E00003B030BD2401002013B502A9002441F85B
:1000F000044D00F0B7F8019B8342CCBFC0EB030076
:10010000204602B010BD000037B5154A019002AB81
:10011000126843F8081D694690470190F0B1114BF1
:100120001B68DB695B690BB11B6813B900252C46A2
:1001300002E00099984711E0009B013B002B0093DF
:1001400007DB01A803F026FA054600F081F8044415
:10015000F2E72846FFF7C8FF2044FFE703B030BDB1
:100160002C01002024010020274B1B6873B5054695
:100170000C4663B10020FBF7B7F8002841D02846B1
:1001800021466A46FFF754FFFAF7ECFFF5E71068DF
:1001900051681E4E6B4603C33368BDF80010B3F8B8
:1001A0004C20B3F850301144ADF80010BDF80210E7
:1001B0001944ADF80210BDF804100A44ADF804204B
:1001C000BDF8062068461344ADF80630FBF78CF8FE
:1001D000336840B9598CDA6C8A1A5A84998C1A6D32
:1001E0008A1A9A840DE0BDF800205A84BDF80220D6
:1001F0009A84284621466A46FFF71AFFFAF7B2FFAB
:10020000E6E702B070BD00BF6417022024010020A1
:100210000A4B1B689A8D02F00C02082A07D00C2AA0
:1002200005D0042A07D1DB69187E01387047DB69E5
:10023000187E400870470020704700BF240100204E
:10024000024B1B68DB69587E704700BF2401002009
:1002500008B5034B1B68DB6900215B68984708BD44
:100260002401002008B5034B1B68DB695B689847D5
:1002700008BD00BF24010020074B5A68596A0132AB
:1002800010B55A605A6B02EBC0046160002102F89D
:100290003010586210BD00BFA017022038B50B4DBA
:1002A000002405F140002146802285F82840FEF711
:1002B00051F828462146C022FEF74CF82146044852
:1002C0000C22BDE83840FEF745B800BFA017022059
:1002D00020D9012010B542680F230D4901EBC3045A
:1002E000246CA24203D213F1FF33F6D210BD0F2BC0
:1002F0000CD80C68A21A0A608268C06802B150600B
:1003000008B1026010BD01EBC3035A6410BD00BF09
:10031000A0170220F8B5264EF3685A1EB36B0546A7
:100320001344081898420C4605D84B591BB943682A
:100330001D44FFF7CFFFB36B9C420AD954F8047CED
:10034000E71B3B682BB97B6838461D44FFF7C2FFAB
:100350003C460F2306EBC302126C954203D213F105
:10036000FF33F7D222E00F2B20D8083306EBC3026D
:1003700061195268A260002084E82100246141F8DC
:10038000045C04F1080102B1516006EBC303E060B4
:100390005960336896F82910054A2B44336029B90F
:1003A000D168CB1A9168994238BF93602846F8BD4E
:1003B000A0170220254B2DE9F74FDA689C6B013A14
:1003C000824602EB04099B4694E82800002B33D1B7
:1003D00004EB0508C8452FD254F805C0D8F80460CE
:1003E000BCF1000F28D0DBF83430184F13F83C3044
:1003F000012B21D1FB6A20468DE80810FFF76AFF28
:10040000D8F800107A6B02EBC102204654604146D6
:10041000324608F0E7F99DE808109C4502D17B6B55
:100420005B1B7B632846A119FFF774FFBAF1000F2D
:1004300001D0824505D935462C444C45C4D3012012
:1004400000E0002003B0BDE8F08F00BFA01702203D
:1004500028B1034AD36B036003B15860D06370477F
:10046000A017022028B1034B5B6B03EBC000406870
:1004700008307047A0170220054BD9690131D961B6
:100480005B6B13F83010013103F83010FFF7EABF4F
:10049000A017022030B50268094B52F8081C5A6BAD
:1004A00012F83140012C03D9DD690DB1013DDD6148
:1004B000013C02F8314000230360184630BD00BF04
:1004C000A0170220024B21F0030118605960704709
:1004D00020D9012030B1044B5B6B03EBC0004368B3
:1004E00058680C38704700BFA017022010B50446AA
:1004F00080B1094B5B6B03EBC00213F83030012B6A
:1005000008D151684868FFF705FF2046BDE8104054
:10051000FFF7B2BE10BD00BFA01702202DE9F041C9
:10052000224CE36A3BB9224B9D685B680835B3FBFC
:10053000F5F5023503E023691D1D05EBD305E80041
:1005400000F078F9804660B3616B2269E76A01EBDD
:10055000C003D2005E680836304608F0F1F922691F
:10056000666306EBC201C4F82C8004311346681E92
:10057000834201F1080103D2013341F8083CF6E758
:1005800006EBC30300265E60636862629B1A2B441D
:100590006360256138463FB1FFF7A8FF3046BDE8EC
:1005A000F0810120BDE8F081BDE8F081A0170220B4
:1005B00020D90120F8B5584E96F82810002940F0AF
:1005C000AA80564D6A68012386F82830B2F5205F6C
:1005D00028BF4FF420522B6894080020A0420CD072
:1005E00047184FF0FF0EB7FBFEFECEEB0E2ECEEB04
:1005F000070743F820700130F0E70020A04216D032
:1006000047184FF0FF0EB7FBFEFECEEB0E2ECEEBE3
:10061000070E53F82070774507D0AA683F4B002A91
:1006200055D15A6892089A6051E00130E6E70131ED
:100630000229D2D1540800210020A0420CD0471832
:100640004FF0FF0EB7FBFEFECEEB0E2ECEEB0707F4
:1006500023F810700130F0E70020A0420FD04718B7
:100660004FF0FF0EB7FBFEFECEEB0E2ECEEB0707D4
:1006700033F810C0BFB2BC45CFD10130EDE7013136
:100680000229D9D100210020904207D04418FF2729
:10069000B4FBF7F73C441C540130F5E700209042CE
:1006A0000BD04418FF27B4FBF7F73C441F5C04F061
:1006B000FF04A742B1D10130F1E701310229E2D1B3
:1006C00000219142A9D0002058540131F9E7144883
:1006D000144B0360FFF7B0FA5A2333620023102152
:1006E00006EBC30299400133102B0B4C1164F6D179
:1006F00068682968A16302232361A0F114030B44F5
:1007000001256363E0605D6065626560FFF702FE7E
:10071000FFF704FF2563F8BDA017022020D90120B0
:100720002CD901209D0201082DE9F0410546264EF5
:100730000335FFF73FFF25F00305336CF26B0435FB
:100740009D4238BF1D4614462CB154F8043CAB42C0
:100750002CD02468F8E7F368B26B02EB030858F872
:10076000047CC7EB08073B6833B12046FFF722FE45
:1007700058F8047CC7EB08073B6813BB7B68AB42A7
:100780001FDB38461C1DFFF7A5FDF36878685B1B6F
:10079000F3607369641B2B44401B3C44736102D0BB
:1007A0003946FFF7B7FD44F8045C0AE023680BB153
:1007B00061685960616801B10B60A24201D1236890
:1007C000F3632046BDE8F081A017022008B5FFF7CB
:1007D000F1FE00220B4B1344D3F8BC3013B19B68DD
:1007E00000200BE0083A12F1800FF3D1F8E75A68C5
:1007F0009B68904238BF104613B19B68002BF6D11E
:100800000C3808BDA017022008B5FFF7DFFFB0F5D0
:10081000800F4FF06403064A04D990FBF3F0136A8B
:10082000584308BD126A5043B0FBF3F008BD00BF47
:10083000A01702202DE9F843384D0446FFF7BAFE11
:100840002F6C2B68BC4224BFE71C27F003070C3732
:100850009F42324C3ED8236B62689A420FD96B6834
:100860006E6A013B6B606B6B4FEAC60903EB0902D2
:1008700052686A62012203F8362056B92AE0013B29
:100880002363FFF74BFE236B013323630028E6D07D
:1008900020E00F2305EBC302126C97420CD213F138
:1008A000FF33F7D208E094682CB16268974214D9FC
:1008B000A268002AF7D101330F2B03D805EBC3023E
:1008C000526CF6E73846FFF775FD0028E1D0304658
:1008D000FFF7D2FC0020BDE8F883D4F804802B6C2D
:1008E000C7EB08020C3320469A4238BF4746FFF751
:1008F000F1FC6B6B4B44E1195C60B8454FF00003B1
:1009000084E8C000A360246141F8047C03DDC7EBE8
:100910000800FFF7FFFC3046BDE8F883A01702206F
:1009200008B1FFF787BF704710B504460068FFF7AE
:10093000DDFD0023236010BD10B580EAE071A1EB5E
:10094000E0710022531C0A2B06D0064C54F82340B9
:10095000A14201D31A46F5E70028B8BF931C1846F8
:1009600010BD00BFE8F40108002807DD0B685A1C21
:100970000A602B221A700B6800221A707047000060
:10098000B0F1004FF0B51C6809D1601C1860013946
:100990002D202070C9B26FF0004001260CE0002825
:1009A00006DA651C1D602D2525704042012400E0FB
:1009B0000024091BC9B200260AB30139C9B21EE0DE
:1009C0004D1E9142EDB205D11C68671C1F60114F8E
:1009D0003F782770104C54F8257090FBF7F4E4B280
:1009E0000A2C0ED807FB14007DB10A2C18BF29462B
:1009F0001D6808BF01246F1C30341F602C70002953
:100A0000DED11B6800221A70F0BD002EEDD001343B
:100A1000E4B2EAE762170220E8F4010873B505467C
:100A2000FFF77EFF064658B1FFF726FD02AC002116
:100A300044F8040D2A46FDF78DFC2046FFF72AFDF9
:100A4000304602B070BD00002DE9F7431E4CD4F8CB
:100A500000E0DEF84C40DEF85060051914449EF8C2
:100A60001820013A92B28F191E44AB1AADF800302B
:100A70001319ADF804306846BB1A3244ADF80230A1
:100A8000ADF80620FAF730FCD0B1284639462246A8
:100A9000FDF710F907F1010928463146224606F113
:100AA000FF38FDF707F9284649464246FDF728F981
:100AB000204649464246FDF723F9FAF753FBE3E7A0
:100AC00003B0BDE8F08300BF24010020C0F3C421BF
:100AD000064B00F01F02C0F345109A5C5B5C03EB11
:100AE0000243034A105C03EB00207047AC1302087A
:100AF0006C130208C0F30741064BC2B2C0F30720D3
:100B00009A5C5B5C03EBC223034A105C03EB40106E
:100B1000704700BFCC140208CC1302084FF6FF70D8
:100B200070470000F8B50F4F3F6806460D46144663
:100B30009C460FB1B847F8BD56F8042B0A49D3B20A
:100B4000013CC85CC2F30743C2F30722CB5C0749F0
:100B50008A5C03EBC02303EB42132B806544EBD18B
:100B6000F8BD00BF38D90120CC140208CC1302080C
:100B7000F8B5134E3668844614461D460EB1B0478C
:100B8000F8BD501E02F18042013A03FB00C001EBA8
:100B9000820102880B4B02F01F06D70A9E5DDB5DC7
:100BA000C2F3451203EB0643074EB25C013C03EB74
:100BB000022341F80439C5EB0000EAD1F8BD00BFBB
:100BC00034D90120AC1302086C1302087047704737
:100BD00070474FF0FF30704710B550F8044B0C6071
:100BE000013A1944F9D110BD10B5046841F8044B1D
:100BF000013A1844F9D110BD10B59CB004466846BE
:100C0000FEF7B0F9094B1868FDF76EFBB4F9000068
:100C1000B4F90210B4F90420B4F90630FFF714FF58
:100C20006846FEF7A9F91CB010BD00BF3CD90120F1
:100C300010B59CB004466846FEF794F9094B186855
:100C4000FDF752FBB4F90000B4F90210B4F9042026
:100C5000B4F90630FFF7F8FE6846FEF78DF91CB0D0
:100C600010BD00BF3CD9012007B56846F9F70EFC5E
:100C70006846FFF7C1FF03B05DF804FB07B568469F
:100C8000F9F704FC6846FFF7D3FF03B05DF804FBF7
:100C900013B5044640B1FFF7EFFB02AB046D43F818
:100CA000040D1846FFF7F6FB204602B010BD1FB535
:100CB00001F00803002B40F28A3440F28A5208BF48
:100CC00022460CBFFF23FE238DE805000020029181
:100CD000039302460346014600F0AEF8062104469F
:100CE000F9F713FA204604B010BD07B5FFF7C4FBAF
:100CF0000190406E00F0D4FB02A8002250F8043DA1
:100D00005A66DA65FFF7C6FB03B05DF804FB438E55
:100D10001B0710B512D5B0F90420B0F900300888CF
:100D20004C880C80D31A8A88CC888C8001339BB283
:100D3000C043D24318441344C8804B8010BD10B543
:100D4000044600F0B6FCFAF798F82046F9F7B7FA2F
:100D50002521BDE81040F9F75BB90000F0B589B076
:100D60000E9E109C119DFAB9F3B9304606A9F9F709
:100D700023FB14F0080F2C4BBDF91C70BDF91EE0CD
:100D800009D0BDF91A10B3F90020781CC1EB0E038D
:100D9000801A013308E0BDF91800B3F900300EF1F4
:100DA00001013A1AC91A013200960F9E01961F4E90
:100DB0000296129E3C360396FAF7A0F806460028E3
:100DC0002FD0FFF759FB04F00802E30648BF42F0BA
:100DD0001002A5F1FE0348BF92B2012B88BF42F07A
:100DE000100229460590F8F74DF8114B08AF0FCBCC
:100DF00057F80C4D04F1340585E80F006423E364D3
:100E00000C4D0A236365002323652B686364384611
:100E1000FFF740FB2B6830465B6898473046FFF78A
:100E20008EFF304609B0F0BD44010020DB0E010802
:100E3000300100204001002010B586B0089C0094CD
:100E4000099C01940A9C02940B9C03940024049432
:100E5000FFF784FF06B010BD37B50C46054600B35A
:100E6000FFF70AFB002C0190C16C426D05DB8A1A6A
:100E700022EAE272944202DC00E000242246016D84
:100E800091420BD002652846F9F7F7FF01A8FFF75A
:100E900001FB28460521F9F738F902E001A8FFF720
:100EA000F9FA03B030BD73B50D46064660B1FFF7E1
:100EB000E3FA024602A8146D40F8042DFFF7EAFA9F
:100EC00030466119FFF7C8FF02B070BD4FF0FF3127
:100ED000FFF7E9BF0121FFF7E6BF2DE9F04F4468B6
:100EE00080468FB020464146F7F7D4FF002800F037
:100EF000C081D8F80030232B00F082810BDC0E2B50
:100F000000F02A810F2B12D00B2B40F0AF8120462E
:100F1000FFF715FFAAE140F21312934200F07F8120
:100F2000B3F5107F12D0242B40F0A08143E120467E
:100F3000FFF7A2FA0590002800F09B81436C05A8FA
:100F40001D68FFF7A7FA2046A84792E1D8F80C7071
:100F5000002F00F08B813B7A2046002B00F0D680DA
:100F6000FFF78AFA05A9836C0390066D204698471F
:100F7000039BB3F832A05D6DDA6C1AF0080FC5EB75
:100F8000020903D097E806003A6079609A6D3F68DD
:100F9000032A14D12046FFF7A8FE0D9B0C990220CE
:100FA00093FBF0F3FF1A069BFB1A581E00FB09F097
:100FB00002F049F9039B0646186603A87EE00698EE
:100FC00087420BDC022A39D05B6E13B12046FFF753
:100FD0008CFE039B0222013E9A652FE007998F4207
:100FE00002DA761B6D422FE008998F4212DC0C99D1
:100FF00000290BDD0D9B022293FBF2F3FF1A3F1A2F
:10100000013F07FB09F002F01EF90646039B03228D
:101010009A6516E009998F4201DA2E4414E00A9984
:101020008F420EDC012A0ED05B6E13B12046FFF713
:101030005CFE039B012501369D6505E04FF0FF3501
:1010400002E0002500E01546DDF80CB00C99DBF855
:101050005C30DDF834E0069A71B102209EFBF0F0BE
:10106000381A801A013800FB09F0019302F0EBF8FE
:10107000019BCBF8600009E0DBF85820012A04BF8F
:10108000DBF84C1001F1FF31CBF8601003A801939D
:10109000FFF700FA019BA5B1BBB94FF4C87240F24B
:1010A000D241204600F034FA07462046FFF7E4F923
:1010B00002460EA840F8282D5766D565FFF7EAF9D5
:1010C00003E013B12046FFF710FE2046012100F097
:1010D000A3FA20463146FFF7BFFE1AF4807F40F0A6
:1010E000C5802046FFF7C8F90EAB856A43F8280D86
:1010F0001846FFF7CFF94FF480712046F7F796FEB8
:10110000A90740F1B3802046012174E0FFF7B4F94C
:10111000458E039003A8FFF7BDF9EA0540F1A680CC
:1011200020464FF48071F7F797FE2046FFF7A4F9A9
:10113000C36D059013B12046FFF7D7FD0EA800221E
:1011400050F8243D9D6A9A65FFF7A4F9AB0740F17A
:101150008D80204602214EE02046FFF78DF90EAB30
:10116000456D43F8240D1846FFF794F9D8F80C2084
:1011700013685268002A79DD103B122B76D8DFE81D
:1011800003F016161212757575757575757575758A
:101190007575750A0D002046294601E02046694212
:1011A000FFF781FE62E02046FFF794FE5EE02046F6
:1011B000FFF78CFE5AE02046D8F80C60FFF75CF988
:1011C0000EAD034645F8240DDA6C3068B1689042E4
:1011D000726805D15E6D8E4202D11E6D96420DD0B1
:1011E000D86459651A652046F9F747FE2846FFF787
:1011F00051F920460521F8F788FF37E0284633E00B
:101200002046FFF739F9059000282FD0D8F80C3088
:10121000C26C1A60426D9A60026D5A6023E02046EB
:10122000FFF72AF9C16D059011B12046FFF73BFE8B
:10123000059BDA6D196D002A1A6E05DD9142B4BF67
:101240000021012106DD04E09142CCBF00210121F3
:1012500000DA1A6519B12046FFF747FD03E0586E22
:10126000322100F085F905A8FFF714F94046FAF796
:101270002FFA0FB0BDE8F08F0388994213B50C46E2
:101280000ED2406850B1FFF7F7F802AB50F8244097
:1012900043F8040D1846FFF7FDF802E0044600E0AD
:1012A0000024204602B010BD13B5044640B1FFF73C
:1012B000E3F802AB048843F8040D1846FFF7EAF898
:1012C000204602B010BD2DE9F743054600283DD069
:1012D0004AB10846114602F04FFBD0F1010407461F
:1012E00038BF002401E0144617462846FFF7C4F82B
:1012F00002AEB0F8008046F8080DD0F804906846B9
:10130000FFF7C8F824BB08F101014846890002F044
:1013100081F9814618B93846FFF7E8F818E0FFF779
:10132000ABF802AB43F8040D40F828701846FFF7FD
:10133000B1F82846FFF7A0F8038800900133C0F801
:10134000049003806846FFF7A5F802E0044600E039
:101350000124204603B0BDE8F08337B5054618B335
:10136000FFF78AF800904068C0B1FFF785F80024C5
:101370000190009B1B889C4206DA019800EB8400D8
:10138000FFF7D2FA0134F4E701A8FFF783F80098D9
:101390000430FFF7C9FA009B00221A806846FFF765
:1013A00079F82846FFF7A2F803B030BD73B50E46B2
:1013B000054658B1FFF760F802AC314644F8040D19
:1013C000FFF75AFF05462046FFF764F8284602B0AB
:1013D00070BD0820FFF722BB30B585B0044610224F
:1013E0000D466846002107F017FA2046FFF73AF845
:1013F00003691BB1019400956846984705B030BD5C
:1014000070B50D4C2368132B06460D4612DCFFF712
:1014100029F803696E6043B12268284601322260D0
:1014200098472368013B236070BD2846BDE87040A3
:10143000FAF74EB970BD00BF40D9012038B5054656
:1014400000F00FF8044654B1AC4207D02046FFF735
:1014500009F8036AAB4202D01C46F4E70024204698
:1014600038BD08B5F8F72BFF18B1FEF7FBFFC069D0
:1014700008BD08BD1FB5044600216846102207F0CC
:10148000CBF9606850B1FEF7EDFF40F213134068EE
:101490000093694663680393F9F798FC04B010BDA4
:1014A00037B5054668B1FEF7E7FF02AC44F8040D16
:1014B0000068FDF767FC2046FEF7ECFF2846FFF7C3
:1014C00015F803B030BD73B5054601A8FDF7D8FB8C
:1014D0000446DCB120460121FDF7AFFC019B83B13E
:1014E00078B11846FEF7BEFF4368AB4209D12046EB
:1014F00001A9019EFDF7DCFB04463046FFF7D0FF53
:10150000E7E7204601A9FDF7D3FBE1E702B070BD94
:101510002DE9F34180460C200F461646FFF77EFA70
:101520000446F0B1FDF79EFC2246811901230F48C5
:10153000FDF7DAFB0546204685B1FEF79DFF034621
:1015400002A8C3F8048040F8043D9F601D60FEF7C8
:10155000A1FF28463146FDF749FC02E0FEF7C6FF31
:101560002C46204602B0BDE8F08100BF751401088A
:1015700013B50C4680B1FEF77FFF01901CB10068E7
:101580002146FDF733FC02AC54F8043D1868FDF722
:101590003BFC2046FEF77EFF02B010BD2DE9E7417F
:1015A0000E4690460746D0B1FEF766FF034602A8F6
:1015B000B3F90410B3F90020B3F9065040F8043D24
:1015C000B3F902308A1AED1AD243ED43164445446A
:1015D000FEF760FF384631462A46F8F71BFD03B098
:1015E000BDE8E08130B50A4D0A4C2B6854F8230061
:1015F00085B050B104A9182341F8103D6946FFF7A2
:10160000FFFE2B68002244F8232005B030BD00BF48
:101610003417022050170220F8B5094B094A044636
:1016200018680F4652F82010A14215461E4601D0F8
:10163000FFF7D8FF336845F82340034B1F70F8BD10
:1016400034170220501702203817022038B50546FB
:101650000C4641B1F8F733FE28B1A5602146BDE83C
:101660003840FFF7CDBE38BD7FB50A4A0346106843
:10167000094A52F8200048B100930E2301910293C9
:1016800002A900AB0593FFF7BBFE012007B05DF890
:1016900004FB00BF341702202417022010B50C46AB
:1016A00030B129B1FEF7DEFE034603CB2060616056
:1016B00010BD38B50546F8F78BFEFF28044603D069
:1016C000FE2808BFFF2400E0FE242846F8F7F7FDB7
:1016D0002146BDE83840F8F7B7BE02F00ABD000069
:1016E000024B1A6802601860704700BF481702205A
:1016F0002DE9F043044687B0002839D0FEF7BCFE40
:101700000346019003C804AD85E8030001A81E6AE2
:10171000D3F82890FEF7BEFE2046FFF78FFE07465F
:1017200030B32046F8F7CBFD19F0020F804604D005
:10173000284641463246F9F731FB2046FEF79CFE2B
:1017400001904046FEF798FE03903846FEF794FE5F
:10175000039B019AD96906620290116201A8DC61BB
:10176000FEF798FE03A8FEF795FE02A8FEF792FE8C
:1017700007B0BDE8F0832DE9F84FDDF828B0DDF8BB
:101780002CA005460E4690461F461446894635F85D
:10179000020BD847D047013C49F8040BF7D11F2F63
:1017A00006D8304641463A46BDE8F84F01F058BDEC
:1017B000BDE8F88F2DE9F84FDDF828B0DDF82CA052
:1017C00005460E4690461F468946044614F8010B0E
:1017D000D847D0472B1B434449F8040B002BF5D1C5
:1017E0001F2F06D8304641463A46BDE8F84F01F073
:1017F00037BDBDE8F88F00002DE9F04F9DB00646DB
:101800000F910D92002800F08683FEF735FE1CAB89
:10181000446943F81C0D1846FEF73CFE3046FAF7C3
:1018200093FF0828014602DD002C00F0C38101224D
:101830004FF0000830461B920B92CDF86880FEF7FF
:101840001BFE0368DFF80CA61B69B0F90A105B6881
:101850000E930DF1700BDAF800304BF8140D04699B
:101860004569D0F80C90B0F90870587C1291FCF7DB
:1018700033F9DAF800301090587CFCF74BF9034646
:1018800058460993FEF706FE082C51460B9A099B11
:1018900004D9102C8CBF0422022205E0012C03D1B4
:1018A00011940DF1680800E011920E98984200F032
:1018B000E2800B68587CFCF735F91390B800FFF70D
:1018C0002FF80C90002800F026833046FAF7D8F85D
:1018D0000646002D00F0BE802846FEF7CDFDDDF85F
:1018E00034B018904FF0000A129A924580F2AE8000
:1018F000189800231993836819A95B695246984781
:10190000B84205462FD10C98FEF7B6FD082C0146CB
:10191000169009D90E9A139B0092019330463A46CD
:10192000109BFFF728FF08E00E98139A0090019291
:1019300030463A46109BFFF73DFF01231098029076
:101940001CAD002200930193039255F8182D0492C8
:101950000F98CDF8148059463A46FCF7FFFA28460E
:10196000FEF798FD60E0012C5CD1002D5CD0199849
:101970000F99CDF80C90082290FBF2F2324401232B
:10198000049200F007020093084401930293069228
:1019900059462A46CDF81480FCF704FA199B18988A
:1019A0001D44836819955B6919A9524698470546F5
:1019B000DBE70C98FEF760FD082C0146169019989D
:1019C00038D90E9A0092119A139B019300FB026082
:1019D000109B2A46FFF7CFFE01230DF1700C1098E3
:1019E00000930022019302900F99039219985CF8DA
:1019F000182D049208442A465946CDF81480CDF893
:101A00002CC0FCF7ABFADDF82CC06046FEF742FDB7
:101A1000199B18981D44836819955B6919A952464A
:101A200098470546002DC4D14E440AF1010A0BF136
:101A3000010B59E70E9B0093119B139A019200FB37
:101A400003602A46109BFFF7B5FEC5E718A8FEF70E
:101A500021FD0EE001230093019304900294CDF840
:101A60000C90CDF814800F980D99129B3A46FCF714
:101A700075FA0C984DE23046FAF702F80646002D4A
:101A800000F08A802846FEF7F7FC00251890129B8C
:101A90009D427DDA189800231993836819A95B6920
:101AA0002A469847B842824624D1AA4618988368A5
:101AB0000AF1010B5B6919A95A469847B84201D14E
:101AC000DA46F3E7C5EB0A0B0D99049601230BF1F7
:101AD000010B0093019329440294CDF80C90CDF8AA
:101AE00014800F983A465B46FCF738FA09FB0B6600
:101AF00055464BE0012C27D1BAF1000F22D019989E
:101B00000F99CDF80C90082290FBF2F23244049227
:101B100000F0070208440D990692012352460093F3
:101B2000019302932944CDF81480FCF73BF9199BEB
:101B3000189853441993836819A95B692A469847F2
:101B40008246D9E74E4421E0BAF1000FFAD0199845
:101B50001199029400FB016204920D990F9ACDF83D
:101B60000C90012310440093524601932944CDF870
:101B70001480FCF7F3F9199B189853441993836860
:101B800019A95B692A4698478246DDE701357EE759
:101B900018A8FEF77FFCBEE1012300930193049097
:101BA0000294CDF80C90CDF814800F980D99129BEB
:101BB0003A4641E030460A91FEF75EFC82461CA898
:101BC000BAF80A2040F810ADDAF800401092D4F8C4
:101BD0001090BAF808709E4C13B2DAF80C200B92F1
:101BE0000993FEF757FCD9F804000E909948006855
:101BF000407C54F820402569D5F80080FBF76CFF45
